:020000040800F2
:100000000000011095C60308218A0208FDD80008E7
:1000100099C7030899C7030899C70308000000009F
:100020000000000000000000000000006D900208C9
:1000300069900208000000006590020851EF000876
:1000400099C7030899C7030899C7030899C7030804
:1000500099C7030899C70308399C0008659D0008E3
:10006000299D0008ED9C0008B19C0008E5BB000834
:10007000D5BB0008C5BB0008B5BB0008A5BB000880
:1000800091BB00087DBB000899C7030899C7030806
:1000900099C7030899C7030899C70308759C000806
:1000A00099C703086DE0000899C703087DE00008C0
:1000B0005DE000084DE0000899C703080DC4000882
:1000C00015C4000801C4000809C4000899C7030842
:1000D00099C703085191000899C70308B590000813
:1000E000FD9B000899C70308719002080DE0000805
:1000F0001DE0000899C703082DE0000869BB00084F
:1001000099C7030899C703083DE0000899C7030889
:1001100079F0000899C703088DC6010871C6010867
:1001200055BB000841BB00082DBB000819BB0008E7
:1001300005BB000899C7030899C7030899C70308B6
:1001400099C7030899C7030899C70308258A0208B5
:10015000F1BA0008DDBA0008C9BA0008DDEF0008EE
:10016000F5C30008FDC3000899C7030899C7030831
:1001700099C7030899C7030899C7030899C70308D3
:0801800099C7030899C70308A1
:1001880002020300E01F0020DC1F00200000000026
:100198000000000016000800EC1F0020F41F0020DB
:1001A8000000000024060008030001007825002054
:1001B800802500200000000000000000010104006C
:1001C800E42A00206C3E002000000000000000002F
:1001D80008020900323D0020703E002000000000A7
:1001E8001F82000806020C00A83D00207C3E00206B
:1001F80000000000DF8E000807020200DC3D00203E
:10020800883E0020000000002C06000802000C00B8
:10021800B43D00208C3E00200000000000000000DB
:10022800F70106002C3D0020983E00200000000049
:100238002E0600080A020A00682B0020A03E0020B3
:100248000000000034060008031233004B41002070
:1002580018410020000000004006000825005A0050
:1002680064400020BE4000200000000000000000A4
:10027800F6110C00584000204C40002000000000FF
:10028800740600082F001100644200203940002045
:100298000000000080060008012008005C420020E1
:1002A800BC42002000000000920600081A00080066
:1002B80040420020C4420020000000009A060008C6
:1002C80010000300F0420020F84200200000000067
:1002D800A20600081D00010014430020A8430020C6
:1002E80000000000A60600081900050000430020D1
:1002F800AC43002000000000A8060008000104002C
:100308009C430020B443002000000000AE06000813
:100318002700040034430020B843002000000000F8
:10032800B206000800020500BC4300202447002054
:1003380000000000000000001E000400FC44002033
:100348002C47002000000000B606000822000C0020
:100358007C4400203047002000000000BA06000856
:1003680004008000645A0020E45B002000000000C4
:1003780000000000F901040020620020946A0020B7
:10038800000000001182000818102C00F061002005
:10039800986A002000000000FD6F0308FB010100BF
:1003A800B4610020C46A00200000000009C50008EC
:1003B800FC01090080600020C86A002000000000DD
:1003C800D5C400080A10120054600020D46A002026
:1003D80000000000C606000806001600245D002084
:1003E800E86A0020000000006D0702081B00F40006
:1003F800086B0020A46D00200000000011630208B3
:1004080026000E00A86E0020986E00200000000054
:10041800ADB002080B2010000072002044720020CA
:1004280000000000D80600081F000E00C46F00205E
:100438005472002000000000E806000805020100D0
:10044800AC6F00206472002000000000F60600086F
:100458002300100094780020AC78002000000000F1
:1004680081E902080902010020790020787900203A
:1004780000000000F806000812100C00D9780020CF
:100488007C79002000000000FA0600080C00240017
:10049800EC780020887900200000000045BC0108A5
:1004A80005000600F27A0020FC870020000000000A
:1004B800080700080E20EA00D679002004880020EA
:1004C800000000004D070208130004000C7B002008
:1004D800F088002000000000100700080201030057
:1004E800C1790020F4880020000000006DBC0108DC
:1004F80028000C00B88B0020D88B002000000000DA
:1005080014070008290050004C8B0020E48B0020C1
:10051800000000000000000014000200488B0020CA
:10052800348C002000000000200700083400100070
:1005380050A9002024AA002000000000058203081A
:100548000D003C0014A9002034AA0020000000007F
:1005580049A0010811000C00A89D002070AA0020E5
:1005680000000000FD9F0108FA010200BC9600206F
:100578007CAA00200000000021C50008FD0124001D
:100588008896002080AA002000000000A1810008B1
:10059800FE01080074960020A4AA002000000000B4
:1005A80011C500082C00100054AD002044AD0020F7
:1005B80000000000796D03082B00240088AD00209E
:1005C80064AD002000000000496D0308F811010027
:1005D80024B40020A8B4002000000000220700086E
:1005E8002A0060000CB50020ACB400200000000018
:1005F800DD81030815007000DCAE00206CB500201A
:100608000000000000000000030106002CB60020D6
:0C06180068B60020000000002407000865
:10062400C409000019012828013C2401000000002D
:1006340000004A01B400D6010000000000000000E0
:1006440000000000000000000000000000000000A6
:100654000000000000000000000000000000000096
:100664000000000000000000000000000000010085
:100674000000000000000000000000000000000076
:100684000000000000000000000000000000E8037B
:100694006400040A00017E05EA05B4053200000185
:1006A4000500000000002801000090010000200364
:1006B400000000000100C800141E010064002C01A9
:1006C400280000300100005A0000000090012C01B5
:1006D400C80064002B21231E6400020000000100F6
:1006E4000A012900000000000000010000000005CC
:1006F400000000002E0000000001000541495234B2
:1007040000000000200003000100000008000000B9
:1007140000000001000000000000000003000400CD
:06072400040101000000C9
:10072A005001000007000000020000000000803FA6
:10073A000000803F0000803F000000000000000031
:10074A000102030406070809010100003024040815
:10075A00F8510408000000000000000040240408CA
:10076A004824040800000000012000004C2404086A
:10077A005424040800000000014000005824040822
:10078A000037040800000000012000006424040867
:10079A007024040800000000040000007424040807
:1007AA0080240408000000000400000084240408D7
:1007BA00F84A040800000000010000000201FF00DE
:1007CA000000803F09D2020879C9020859D10208FB
:1007DA0000000000B5C602089DCB02086D81020820
:1007EA00D58002080000000000000000C98002084D
:1007FA0049800208458002084180020835800208C3
:10080A00318002083D80020839800208BD80020852
:10081A00B1800208898002089D800208758002085A
:10082A00618002084D800208D4F603080508040016
:10083A0000000000801D04081C1D0408C0F60308FF
:10084A000000000000F7030805080A000000000085
:10085A00801D04081C1D04081C1F04080000000059
:10086A00FFFFFFFF0000803F010000000000803F03
:10087A00303030302D30312D30315430303A303044
:10088A003A3030000000803F0403090412010002DC
:10089A0002020040830440570002010203010000E3
:1008AA0009024300020100C03209040000010202E9
:1008BA00010005240010010524010001042402029C
:1008CA000524060001070582030800FF0904010048
:1008DA00020A000000070501024000000705810224
:1008EA00400000007DD302089DD202085DCC0208B8
:1008FA0011C702081DCA020821C702083DC702081B
:10090A00E9C60208D9C6020800000000000000007B
:10091A000100000000000101FFFF0000E841040897
:10092A000000000000000000FD9E0108A0860100F2
:10093A0004000000000000000000000000000000A9
:10094A00000000000000000000000000000000009D
:10095A00404E0408143D04080000000041590108F3
:10096A007D000000060000000000000000000000FA
:10097A00000000000000000000000000000000006D
:10098A0000000000405204080000000000000000BF
:10099A000DAA0308E803000003000000000000009D
:1009AA00000000000000000000000000000000003D
:1009BA000000000000000000485204080000000087
:1009CA00000000007508020810270000030000005C
:1009DA00000000000000000000000000000000000D
:1009EA000000000000000000000000009857040802
:1009FA00000000000DF10208C9370108204E00006E
:100A0A0005000000000000000000000000000000D7
:100A1A0000000000000000000000000000000000CC
:100A2A005C4304080000000000000000C9A4030899
:100A3A001027000001000000000000000000000074
:100A4A00000000000000000000000000000000009C
:100A5A0000000000545204080000000000000000DA
:100A6A00A1C40008E803000005000000000000001F
:100A7A00000000000000000000000000000000006C
:100A8A00000000000000000060520408000000009E
:100A9A000000000009BF0108204E0000030000000A
:100AAA00000000000000000000000000000000003C
:100ABA00000000000000000000000000705204085E
:100ACA00000000000000000015BD0108204E0000D3
:100ADA000300000000000000000000000000000009
:100AEA0000000000000000000000000000000000FC
:100AFA00805204080000000000000000D1560108DE
:100B0A00400D030003000000000000000000000088
:100B1A0000000000000000000000000000000000CB
:100B2A00000000009C4204080000000000000000D1
:100B3A005DB103081027000001000000000000005A
:100B4A00000000000000000000000000000000009B
:100B5A000000000000000000303D04080000000012
:100B6A00000000009573020810270000030000002F
:100B7A00000000000000000000000000000000006B
:100B8A00000000000000000000000000905204086D
:100B9A000000000000000000E5BA0308A08601007A
:100BAA00010000000000000000000000000000003A
:100BBA00000000000000000000000000000000002B
:100BCA00203D0408000000000000000005BA0308E8
:100BDA0050C30000010000000000000000000000F7
:100BEA0000000000000000000000000000000000FB
:100BFA0000000000985204080000000000000000F5
:100C0A006DB50308A86100000100000000000000A3
:100C1A0000000000000000000000000000000000CA
:100C2A000000000000000000A452040800000000B8
:100C3A0000000000E17B0208A0860100010000001C
:100C4A00000000000000000000000000000000009A
:100C5A0000000000000000000000000064430408D7
:100C6A00000000000000000015F10008A00F0000BD
:100C7A000100000000000000000000000000000069
:100C8A00000000000000000000000000000000005A
:100C9A00B05204080000000000000000B9B40208C5
:100CAA001027000001000000000000000000000002
:100CBA00000000000000000000000000000000002A
:100CCA0000000000C4420408000000000000000008
:100CDA002D9F0108A00F0000010000000000000085
:100CEA0000000000000000000000000000000000FA
:100CFA000000000000000000C843040800000000D3
:100D0A00000000006DD60208102700000100000054
:100D1A0000000000000000000000000000000000C9
:100D2A00000000000000000000000000083D040868
:100D3A000000000000000000ED6103081A410000F5
:100D4A000100000000000000000000000000000098
:100D5A000000000000000000000000000000000089
:100D6A00BC520408000000000000000075B003082F
:100D7A00400D030000000000000000000000000019
:100D8A000000000000000000000000000000000059
:100D9A0000000000C4520408000000000000000027
:100DAA0031B00308400D03000000000000000000FD
:100DBA000000000000000000000000000000000029
:100DCA000000000000000000CC52040800000000EF
:100DDA0000000000A9A00108A0860100030000008D
:100DEA0000000000000000000000000000000000F9
:100DFA00000000000000000000000000FF000000EA
:100E0A00010000000101000001EF020800000000DB
:100E1A00000000000100000001010100045604085E
:100E2A000E000000191B030800000000000000006B
:100E3A007C080020C85504080000000000000000DB
:100E4A000000000000000000F85104080000000043
:100E5A00000000000809002004000000545504089E
:100E6A000C000000E92003081C0D0020000000000F
:100E7A00785404080C000000B9200308100D002063
:100E8A0000000000E8550408080000000000000007
:100E9A00040D002004000000D85504080C000000CE
:100EAA00D11F0308F80C0020000000006454040855
:100EBA0003000000C5600308E00C002000000000E9
:100ECA00E055040803000000C5600308C80C0020B0
:100EDA00000000006854040801000000000000003F
:100EEA000000000000000000000000000D000000EB
:100EFA00000000000000000000000000C8550408BF
:100F0A0000000000000000000000000000000000D7
:100F1A00F851040800000000000000000809002041
:100F2A0004000000F854040803000000751F0308B9
:100F3A00B00C002008000000D85504080C0000007E
:100F4A00D11F0308F80C00200000000064540408B4
:100F5A0003000000C5600308E00C00200000000048
:100F6A00E055040803000000C5600308C80C00200F
:100F7A00000000006854040801000000000000009E
:100F8A000000000000000000000000000D0000004A
:100F9A00000000000000000000000000F0550408F6
:100FAA000000000000000000000000000000000037
:100FBA00F8510408000000000000000008090020A1
:100FCA00040000000055040803000000C56003087F
:100FDA00280D0020000000006854040801000000E9
:100FEA0000000000000000000000000000000000F7
:100FFA000D000000000000000000000000000000DA
:10100A0020700020702D72002D202D2D202D2D2DC9
:10101A002D202D2D2D2D00000000000000000000C5
:10102A0000000000000000002D202D2D202D2D2D68
:10103A002D202D2D2D0000000000000000000000D2
:10104A000000000000000000BA79002088130C1785
:10105A0001000000BC79002088130C170000000072
:10106A003C540408000000000000000000000000DA
:10107A00000000004C5404080800000000000000B2
:10108A003409002004000000585404080800000035
:10109A000000000028090020000000006454040831
:1010AA0004000000B51F0308000000000000000053
:1010BA00685404080100000000000000000000005D
:1010CA0000000000000000000D0000000000000009
:1010DA000000000000000000B879002088130C17F7
:1010EA0001000000B679002088130C1700000000E8
:1010FA00A85404080E000000711B03080000000039
:10110A0000000000400900200A7B002001000000C6
:10111A00401D0408B5790020010000004C1D040898
:10112A005EB6002002000000541D04082A5B00205D
:10113A000000000000000000285B00200000000002
:10114A0000000000265B00200000000000000000F4
:10115A00245B00200000000000000000225B002049
:10116A000000000000000000205B002000000000DA
:10117A0000000000F41D0020000000000000000034
:10118A00B479002002000000601D0408B05404086D
:10119A000000000000000000000000000000000045
:1011AA004C5404080800000000000000C409002094
:1011BA000400000058540408080000000000000061
:1011CA00B80900200000000064540408040000006C
:1011DA00511B0308000000000000000068540408C6
:1011EA0001000000000000000000000000000000F4
:1011FA00000000000D0000000000000000000000D8
:10120A0000000000C05404080000000000000000B4
:10121A000000000000000000D05404080C00000088
:10122A0059200308000A002004000000DC540408C6
:10123A000C000000951B0308F409002004000000BC
:10124A00E85404080C00000019200308E8090020EB
:10125A0000000000F454040803000000951F03086E
:10126A00D00900200800000000550408030000000F
:10127A00C5600308280D0020000000006854040817
:10128A000100000000000000000000000000000053
:10129A00000000000D000000000000000000000037
:1012AA0000000000085504080000000000000000CB
:1012BA0000000000000000001055040804000000AF
:1012CA001921030800000000000000006854040807
:1012DA000100000000000000000000000000000003
:1012EA00000000000D0000000000000000000000E7
:1012FA00000000005C550408000000000000000027
:10130A0000000000000000005C4404080C0000001B
:10131A0000000000600A0020040000006C55040868
:10132A000800000000000000540A00200400000029
:10133A00785504080800000000000000480A002050
:10134A0004000000805504080800000000000000A6
:10135A003C0A002004000000885504080800000028
:10136A0000000000300A0020040000009055040824
:10137A000800000000000000240A00200400000009
:10138A00985504080800000000000000180A002010
:10139A0004000000A0550408080000000000000036
:1013AA000C0A002004000000685404080100000030
:1013BA000000000000000000000000000000000023
:1013CA000D00000000000000000000000000000006
:1013DA00A85504080E000000611B03080000000065
:1013EA00000000006C0A0020B05504080E0000003E
:1013FA00000000000000000000000000E40A0020D5
:10140A00B85504080E0000000000000000000000AB
:10141A0000000000840B0020097B0020040000006B
:10142A006C1D0408B0790020E0150C1700000000BC
:10143A00B3790020080000001C1D0408B2790020BE
:10144A0005000000801D0408C05504080E000000B5
:10145A00000000000000000000000000D40B002083
:10146A00000101010060024010600240000000001B
:10147A00000B000000002000000000000000000037
:10148A00006002402860024000000000060C0000D4
:10149A000000200000000000000000000060024080
:1014AA004060024000000000100D00000000200013
:1014BA000000000000000000006002405860024086
:1014CA0000000000160E00000000200000000000CE
:1014DA00000000000060024070600240000000004E
:1014EA00200F0000000020000000000000000000A3
:1014FA0000600240886002400000000026100000E0
:10150A00000020000000000000000000006002400F
:10151A00A06002400000000030110000000020001E
:10152A00000000000000000000600240B8600240B5
:10153A0000000000362F000000002000000000001C
:10154A000000000000640240106402400000000035
:10155A000038000000004000000000000000000009
:10156A0000640240286402400000000006390000BE
:10157A00000040000000000000000000006402407B
:10158A004064024000000000103A000000004000E1
:10159A00000000000000000000640240586402409D
:1015AA0000000000163B00000000400000000000A0
:1015BA000000000000640240706402400000000065
:1015CA00203C000000004000000000000000000075
:1015DA0000640240886402400000000026440000C3
:1015EA00000040000000000000000000006402400B
:1015FA00A0640240000000003045000000004000E6
:10160A00000000000000000000640240B8640240CC
:10161A000000000036460000000040000000000004
:10162A0000000000000000010000000000000000AF
:10163A0000000000D05B04080E000000000000005B
:10164A000000000000000000001D0020FFFFFFFF57
:10165A00FA0000000100000001000000085504081B
:10166A000000000000000000000000000000000070
:10167A006D56040804000000071F0308000000005C
:10168A000000000068540408010000000000000087
:10169A000000000000000000000000000D00000033
:1016AA00000000000000000000000000CE5B0020E7
:1016BA000100C40900000000CC5B00200100C4093D
:1016CA0000000000CA5B00200100C40900000000FD
:1016DA00C85B00200100C40900000000C45B0020B0
:1016EA000100C40900000000C65B00200100C40913
:1016FA0000000000C25B00200100C40900000000D5
:10170A00C05B00200100C4090000000090560408D4
:10171A000E000000000000000000000000000000B1
:10172A003C0F002028B600209CFF2C01000000007E
:10173A00FA0600200A0000001C1F0408AC790020E9
:10174A00E0150C1700000000F90600200800000050
:10175A001C1D0408F806002005000000801D04086E
:10176A00AE79002002000000341F0408F87A002035
:10177A000100FF7F01000000F07A00200200000053
:10178A00401F0408CA79002003000000501F040803
:10179A00C979002003000000501F0408C87A0020FD
:1017AA000000F40101000000C67A00200000F401E4
:1017BA0001000000C47A00200000F40101000000CA
:1017CA00C27A00200000F40101000000C07A002063
:1017DA0000FF0100DC7A0020E803D0070A000000BD
:1017EA00DA7A0020006401000A000000DB7A002097
:1017FA00006401000A000000D47A0020006401009D
:10180A000A000000D97A0020006401000A000000E2
:10181A00D87A0020006401000A000000D77A00206C
:10182A00006401000A000000D37A002000FF0100D2
:10183A000A000000D27A002000FF01000A0000001E
:10184A00D27900200000F40101000000D0790020C4
:10185A000000F40101000000CE7900200000F4012C
:10186A0001000000CC7900200000F4010100000012
:10187A00CF7A002000C80100CE7A002000C80100FB
:10188A00CD7A002000C80100CC7A00200064010053
:10189A000A000000CB7A002000FF01000A000000C5
:1018AA00E77A002000C80100E67A002000C801009B
:1018BA00E57A002000C80100E47A002000C801008F
:1018CA00E37A002000C80100E27A002000C8010083
:1018DA00E17A002000C80100E07A002000C8010077
:1018EA00DF7A002000C801009856040800000000B2
:1018FA00000000000000000000000000A8560408D4
:10190A000900000000000000E00F002004000000B1
:10191A00B05604080900000000000000D40F00209F
:10192A00040000006C5A04080900000000000000CE
:10193A00C80F002004000000E85304080900000052
:10194A0000000000BC0F002004000000B856040884
:10195A000900000000000000B00F00200400000091
:10196A00C05604080900000000000000A40F00206F
:10197A0004000000C8560408090000000000000026
:10198A00980F002004000000D05604080900000047
:10199A00000000008C0F00200400000068540408B6
:1019AA00010000000000000000000000000000002C
:1019BA00000000000D000000000000000000000010
:1019CA0000000000A8570408000000000000000002
:1019DA000000000000000000B857040805000000DD
:1019EA0000000000C87900200000000068540408C4
:1019FA0001000000000000000000000000000000DC
:101A0A00000000000D0000000000000000000000BF
:101A1A0000000000C0570408000000000000000099
:101A2A000000000000000000F85104080000000057
:101A3A0000000000E808002004000000E453040845
:101A4A000C0000004D1F0308401000200000000099
:101A5A00545504080C000000C51A0308341000206D
:101A6A0000000000785404080C000000911A0308D2
:101A7A002810002000000000E855040808000000B3
:101A8A00000000001C10002004000000D8550408C3
:101A9A000C0000007D1A030810100020000000004E
:101AAA00CC570408090000000000000004100020C0
:101ABA00040000006454040803000000C560030821
:101ACA00EC0F002000000000685404080100000028
:101ADA0000000000000000000000000000000000FC
:101AEA000D000000000000000000000000000000DF
:101AFA00D4570408000000000000000000000000A5
:101B0A0000000000E45704080C0000000000000078
:101B1A005810002000000000EC5704080A000000DA
:101B2A0000000000107B002000000000F8570408A5
:101B3A000A00000000000000187B002000000000DE
:101B4A00005804080A00000000000000207B002062
:101B5A000000000008580408080000000000000007
:101B6A004C10002000000000105804080400000077
:101B7A0081230308000000000000000068540408E4
:101B8A00010000000000000000000000000000004A
:101B9A00000000000D00000000000000000000002E
:101BAA00000000001C5804080000000000000000AB
:101BBA000000000000000000305804080C0000007B
:101BCA0000000000701000200000000040580408C7
:101BDA0004000000DD2103080000000000000000EE
:101BEA00485804080C00000000000000641000209F
:101BFA00000000005C58040804000000BD2103082E
:101C0A000000000000000000685404080100000001
:101C1A0000000000000000000000000000000000BA
:101C2A000D0000000000000000000000000000009D
:101C3A0064580408000000000000000000000000D2
:101C4A0000000000785804080700000000000000A7
:101C5A00AC100020000000008458040808000000AE
:101C6A0000000000A01000200000000090580408A6
:101C7A00080000000000000094100020000000008E
:101C8A009C5804080800000000000000881000208A
:101C9A0000000000A8580408080000000000000026
:101CAA007C100020000000006854040801000000B5
:101CBA00000000000000000000000000000000001A
:101CCA000D000000000000000000000000000000FD
:101CDA00B45804080000000000000000E3080020D7
:101CEA0000000000C05804080B00000000000000BB
:101CFA001411002000000000C85804080B0000005E
:101D0A00000000000811002000000000D458040858
:101D1A000B00000000000000FC1000200000000082
:101D2A00E05804080B00000000000000F01000203A
:101D3A0000000000EC5804080B000000000000003E
:101D4A00E410002000000000F85804080B0000000E
:101D5A0000000000D810002000000000005904080C
:101D6A000B00000000000000CC1000200000000062
:101D7A000C5904080B00000000000000C0100020ED
:101D8A0000000000185904080800000000000000C4
:101D9A00B41000200000000068540408010000008C
:101DAA000000000000000000000000000000000029
:101DBA000D0000000000000000000000000000000C
:101DCA002459040800000000000000000000000080
:101DDA000000000038590408080000000000000054
:101DEA0044110020000000004459040808000000C3
:101DFA0000000000381100200000000050590408BB
:101E0A0008000000000000002C1100200000000063
:101E1A005C5904080800000000000000201100209E
:101E2A0000000000685404080100000000000000DF
:101E3A000000000000000000000000000D0000008B
:101E4A0000000000000000000000000064590408BF
:101E5A000000000000000000E00800200000000070
:101E6A00745904080B0000000000000074110020DF
:101E7A0000000000805904080B0000000000000068
:101E8A0068110020000000008C59040807000000B7
:101E9A0000000000601100200000000098590408AA
:101EAA000700000000000000581100200000000098
:101EBA00A459040807000000000000005011002087
:101ECA00000000006854040801000000000000003F
:101EDA000000000000000000000000000D000000EB
:101EEA00000000000000000000000000B0590408D3
:101EFA000000000000000000E008002000000000D0
:101F0A00BC5904080700000000000000C0110020AE
:101F1A0000000000C4590408070000000000000087
:101F2A00B811002000000000CC5904080700000086
:101F3A0000000000B011002000000000D45904087D
:101F4A000700000000000000A811002000000000A7
:101F5A00DC5904080700000000000000A01100205E
:101F6A0000000000E4590408070000000000000017
:101F7A009811002000000000EC5904080700000036
:101F8A00000000009011002000000000F45904082D
:101F9A000700000000000000881100200000000077
:101FAA00FC5904080700000000000000801100200E
:101FBA00000000006854040801000000000000004E
:101FCA000000000000000000000000000D000000FA
:101FDA00000000000000000000000000045A04088D
:101FEA000E00000000000000511C03080000000061
:101FFA00C8110020C679002017000000601F0408DD
:10200A00C57900200A320100C479002001FA0100D2
:10201A00C079002000C80100BE790020E803D0077B
:10202A0001000000414952424F544634000000006A
:10203A000C5A04080E000000671C03080000000088
:10204A0091210308A4120020145A04080E0000006B
:10205A00DD1903080000000000000000F41200204F
:10206A001C5A04080E00000061230308AD1E030871
:10207A00A91E0308D0130020245A04080E000000E9
:10208A00891C0308000000000000000084140020DE
:10209A002C5A04080E000000191D0308E91C030845
:1020AA000000000010150020345A04080E00000039
:1020BA00951D0308DD1D030800000000B01500206F
:1020CA00D07A002001030100405A04080E000000E3
:1020DA00BD1C0308991C030800000000A01600207C
:1020EA00485A04080E000000491D0308FD21030890
:1020FA00000000002C170020545A04080E000000AB
:10210A000D1E03084922030800000000CC17002016
:10211A00CA7A0020010301005C5A0408000000008A
:10212A00000000000000000000000000685A0408D7
:10213A000800000000000000F8180020000000005D
:10214A00705A04080700000000000000F018002080
:10215A0000000000805A0408070000000000000088
:10216A00E8180020000000008C5A0408070000004C
:10217A0000000000E018002000000000985A04083F
:10218A000C00000000000000D4180020000000002D
:10219A00A45A040803000000C5600308BC18002004
:1021AA00000000006854040801000000000000005C
:1021BA000000000000000000000000000D00000008
:1021CA00000000000000000000000000AC5A0408F3
:1021DA0000000000000000000000000000000000F5
:1021EA00BC5A04080A0000000000000090240408F9
:1021FA0000000000C45A04080A00000000000000A1
:10220A001024040800000000CC5A04080A00000048
:10221A0000000000E87A002000000000D45A0408F8
:10222A000A0000000000000004190020000000005D
:10223A0068540408010000000000000000000000CB
:10224A0000000000000000000D0000000000000077
:10225A000000000000000000DC5A04080000000032
:10226A00000000000000000000000000F05A04080E
:10227A0003000000C56003084019002000000000A8
:10228A00FC5A040803000000C5600308FC0600208D
:10229A0000000000045B040803000000C560030896
:1022AA0028190020000000000C5B0408030000004D
:1022BA00C5600308101900200000000068540408D3
:1022CA000100000000000000000000000000000003
:1022DA00000000000D0000000000000000000000E7
:1022EA0000000000185B0408000000000000000065
:1022FA000000000000000000245B04080700000042
:10230A0095220308F019002000000000404E04083E
:10231A0003000000C5600308D8190020000000006F
:10232A00305B040803000000C5600308C0190020E0
:10233A0000000000385B040803000000C5600308C1
:10234A00A819002000000000405B040807000000F4
:10235A0079220308A0190020000000007055040823
:10236A0003000000C560030888190020000000006F
:10237A004C5B040803000000C560030870190020C4
:10238A0000000000585B040803000000C560030851
:10239A0058190020000000006854040801000000D9
:1023AA000000000000000000000000000000000023
:1023BA000D00000000000000000000000000000006
:1023CA00645B04080E000000191C0308E11B0308E3
:1023DA0000000000F81900206C5B04080E000000E1
:1023EA007D1E03080000000000000000AC1A002057
:1023FA00785B04080E0000000000000000000000E6
:10240A0000000000381B0020885B04080E00000052
:10241A00551E0308B122030800000000C41B002057
:10242A00905B0408000000000000000000000000AB
:10243A0000000000D450040803000000C56003082F
:10244A00E81C0020000000007C5B04080300000078
:10245A00C5600308D01C0020000000009C5B040833
:10246A0003000000C5600308B81C0020000000003B
:10247A00A85B040803000000C5600308A01C002034
:10248A0000000000B05B040802000000DD5F0308E2
:10249A000000000000000000B85B04080200000011
:1024AA00DD5F03080100000000000000C45B0408AF
:1024BA0002000000DD5F03080200000000000000C7
:1024CA00000000000D0000000000000000000000F5
:1024DA000000000000FFFF0000000000AA550501EF
:1024EA000000AA5507010000AA5503009F0000003A
:1024FA0000000000010203040102030406070809A0
:10250A00AA550B010000AA550902000000000000AC
:10251A0001000000C0120000685E0C0043000000C9
:10252A0000000000000000000000000000000000A1
:10253A00000000000000000000000000430000004E
:10254A000000000000000000000000000000000081
:10255A00000000000000000000000000430000002E
:10256A000000000000000000000000000000000061
:10257A00000000000000000000000000430000000E
:10258A000000000000000000000000000000000041
:10259A0000000000000000000000000043000000EE
:1025AA000000000000000000000000000000000021
:1025BA0000000000000000000000000043000000CE
:1025CA000000000000000000000000000000000001
:1025DA0000000000000000000000000043000000AE
:1025EA0000000000000000000000000000000000E1
:1025FA00000000000000000000000000FDC9030800
:10260A003DC8030800000000BD5D040868560408C0
:10261A00994C0408994C0408994C0408994C0408EC
:10262A00994C0408994C0408994C0408994C0408DC
:10263A00994C0408FFFFFFFFFFFFFFFFFFFFFFFFAB
:10264A00FFFF000001004153434949000000000018
:10265A000000000000000000000000000000000070
:10266A0000000000000041534349490000000000F7
:10267A000000000000000000000000000000000050
:10268A0000000000000000006C1F00200000000095
:10269A000000000000000000000000000000000030
:1026AA000000000000000000000000000000000020
:1026BA000000000000000000000000000000000010
:1026CA000000000000000000000000000000000000
:1026DA0000000000000000000000000000000000F0
:1026EA0000000000000000000000000001000000DF
:1080000070B4EFF31186502383F31288436B1A6820
:10801000D20720D45D686DB9446A826A944217D051
:1080200081691144D9600ED9A21A5A608462002273
:1080300080F858201A6842F00102F1B21A6081F308
:10804000118870BC704701698A1A5A608562EEE730
:10805000012380F85830F3B283F3118870BC704765
:10806000436A8269D154436A0169426B01338B428E
:1080700028BF00234362002A2FD0EFF31182502340
:1080800083F31288436B1968C9072CD470B45E68F7
:108090006EB9456A816A8D4217D084690C44DC60F0
:1080A0000ED9691A59608562002180F85810196844
:1080B00041F00101D2B2196082F3118870BC70479F
:1080C0000469611A59608662EEE7012380F858302E
:1080D000D2B282F3118870BC7047426DD36843F00E
:1080E0008003D3607047D2B282F31188704700BF1B
:1080F000026B10B462B1836CC2684469D11A013B4F
:10810000615C5DF8044B08BF13468364C8B27047D6
:10811000016A4369C4685B5C0131A14228BF114612
:1081200001625DF8044BD8B2704700BF436B13B1D6
:1081300090F858007047836A406A181AB0FA80F0C5
:1081400040097047416A836A99420AD3CB1A416B4E
:10815000026961B14968501E0B4483420AD2C01AB9
:10816000704702691144CB1A416B0029F2D1501EAD
:10817000C01A704700207047036B43B1826C5B6884
:1081800093422FBF981AC0689B1AC0187047C269E3
:10819000036A9A422FBFD01AC0688018C01A70476D
:1081A0000A4B30B503F1180493F900205D78072AD3
:1081B000C8BF143A811804330D7313F8025C855458
:1081C00013F8012C0A76A342EED130BDCCEE0308A1
:1081D00003682DE9F041DF691FB13B46BDE8F0417E
:1081E0001847002A164611DD04460D460E4400E0ED
:1081F00023689B68204698470028F9D0236815F823
:10820000011B1B6820469847AE42F1D1BDE8F081C2
:1082100000232522027043708370C37070471523BA
:1082200003701623C370172383713A2383703B2393
:1082300043713C230372704730B4846814B12368DF
:10824000A5885D83436840F2E93001E0002832D020
:108250001D89013815F0020F80B2F7D089B29981DB
:1082600040F2E93101E0002947D01889013910F0C6
:10827000010F89B2F7D0998940F2E93100E059B392
:108280001889013910F0020F89B2F8D092B29A81A0
:1082900040F2E93201E0002A3FD01989013A11F099
:1082A000010F92B2F7D09B8914B12368A2881A8378
:1082B000012030BC704721498B4204D0A1F57441A4
:1082C0008B42D9D102201E4901EB001041890131B6
:1082D00089B241814189CFE7184A934204D0A2F57F
:1082E00074429342E0D10221154B03EB01114B89FB
:1082F00001339BB24B814B89D6E71048834203D0B0
:1083000010498B42B8D102210D4800EB0111488978
:10831000013080B248814989AEE708498B4203D0D9
:10832000084A9342C0D10222054B03EB0212538943
:1083300001339BB253815389B6E700BF003001403F
:10834000388C0020003C0040F0B484894FF6FF7662
:108350004FF47A7443B3002938D00F78013101E02B
:10836000B4421AD00589013C15F00205A4B2F7D039
:10837000BCB284814FF47A7402E0BCB2B4420CD037
:10838000058915F0010504F1FF37F6D08589ADB2F6
:108390000AB115700132013BDCE70D4B984207D062
:1083A000A3F57443984202D00120F0BC7047022527
:1083B000084B03EB05156B8901339BB26B81688910
:1083C00080B2003018BF0120F0BC7047FF27C9E71A
:1083D00000300140388C002070B50546806810B12F
:1083E00004688088608341F08001686840F2E93465
:1083F00000E0E4B10689013C16F0020FA4B2F8D007
:1084000089B2818140F2E93100E009B30489013980
:1084100014F0010F89B2F8D081890021FFF794FF91
:10842000AB6813B11A689B881383012070BD104993
:10843000884204D0A1F574418842EED102240D494E
:1084400001EB04146189013189B261816189E4E73A
:10845000074CA04203D008498842DED10221054CD6
:1084600004EB01114C890134A4B24C814989D4E751
:1084700000300140388C0020003C0040002870B5DE
:108480001EDB0928044620DD012303EB83035B0088
:10849000B0FBF3F2092AF8D87BB10E4EB4FBF3F02F
:1084A0000928CCBF57223022A6FB03E5024403FB78
:1084B0001044EB0801F8012BF0D100230B7070BDC4
:1084C0002D230B7040420131DBE7303001F8010B06
:1084D000F3E700BFCDCCCCCC884230B44FF00104E0
:1084E0002ED301FB04F4B0FBF4F58D42F9D284B134
:1084F000AAB901E0B0FBF4F5092DCCBF5722302218
:108500002A4404FB150003F8012BB4FBF1F4002C02
:10851000F0D100221A7030BC7047B0FBF4F5092D81
:10852000CCBF372230222A4404FB150003F8012B6C
:10853000B4FBF1F4002CF0D100221A7030BC70476B
:108540000546002AEBD1D7E703685A1C0260197070
:10855000704700BF2DE9F047089C2578002B804626
:1085600089460CBF4FF0200A4FF0300A661C35B325
:10857000002A29DD334601E0024698B113F8011BB9
:10858000501E0029F8D1971E60B13D46013D51466D
:108590004046C8476B1C002BF8DC257827EAE770BB
:1085A000013055B1041B29464046C847301916F81A
:1085B000015B002DF7D1BDE8F087BDE8F087002A08
:1085C00004DC2846BDE8F0870020EBE7571EDCE717
:1085D00083684268D0ED037A00EB83010133934254
:1085E00081ED040A836004BF0023836000EB8303F2
:1085F00093ED047A036870EE277A9A42C0ED037A0D
:1086000077EEC77AC0ED037A0CDA013307EE103A41
:10861000F8EEC76AB7EE007A87EEA60A036030EE7E
:10862000070A704707EE102AB8EEC77A87EE870A66
:10863000704700BF90ED057A90ED004AD0ED066AD4
:10864000D0ED014AD0ED047A90ED035AD0ED025AF4
:10865000A4EE007AB0EE406AB0EE470AB0EE667A59
:10866000A6EE247A67EEC07AA0EE457AE6EE257A89
:1086700080ED057AC0ED067A704700BFD0ED057A2F
:1086800090ED013AD0ED003AD0ED064A90ED024A65
:1086900090ED077A90ED035A90ED086AD0ED045AF8
:1086A000C0ED067AF0EE406A27EE830AC0ED056A57
:1086B000A3EEA60A80ED087AA4EE240AA5EE470AE6
:1086C000A5EEC60A80ED070A704700BFD0ED007A1C
:1086D00090ED017A30EE670AE7EE007AB0EE670AB5
:1086E000C0ED007A704700BF704700BF0A44914256
:1086F00014D030B40139551E41F2210211F8014F56
:10870000082380EA042004044CBF82EA40004000B1
:10871000013B80B2F7D18D42F0D130BC704700BF31
:108720002DE9F04FDFF8F8C1DFF8F8E1BCF80A7086
:10873000DEF80060BCF80C30BCF808A03C028BB03E
:10874000361B4FF00004CDE90034009CBCF8063025
:108750004FEA17654FF0000767EB0507B946B046CB
:10876000A4FB06670024CDE90634009C002304FB2B
:1087700009770024CDE90034AAFB0823CDE90223C0
:10878000039AF30D00930AFB09230393009B43EA2A
:1087900047230093029B4FEAD31AFB150193039BD7
:1087A0004AEA436ADDE9002344464D46CDE90845DF
:1087B000069C12F5FA62A4FB086743F1000304FB70
:1087C0000977CDE90623BCF80440039BBCF80220DE
:1087D0004FEAE31B230C059323040493340A44EA71
:1087E00007643D12DDE904674FEAC23816EB0A065A
:1087F00047EB0B0718EB0408DDE906344FEA524952
:1088000049EB0509B3F5FA6F74F10004B246BB46B3
:108810003CDADDE90067BC00B20044EA9673B418A4
:1088200047EB030522463C462B4602FB04F406FBBD
:108830000344A2FB06232344940844EA83749D1056
:108840005B104FEA3202B8EB040869EB0509BAEB9A
:10885000020A6BEB030BDDE90623304C4FF0FF35CA
:10886000A242AB412CDBDDE90856A5FB052305FB45
:1088700006F403EB4403D40F44EA4304DD17DDE9B7
:108880000623121B63EB0503CDE90623DEF8044043
:10889000A4FB082304FB0933540D44EAC3245D15EB
:1088A000B4EB0A0A65EB0B0B4FEADA3343EA4B43AE
:1088B00000B1036009B1069B0B600BB0BDE8F08FFF
:1088C00040F6AC52B4184FF0000347EB03052246C4
:1088D000A2FB022304FB05F403EB4403941843EBCF
:1088E0000305A4185D414FEA850CA6004CEA947C70
:1088F000B41A6CEB0305DF00D6006D104FEA3404A8
:1089000047EA5277921B63EB0703B8EB040869EB65
:1089100005091AEB020A4BEB030BA4E724FAFFFF4D
:10892000C88B0020D01F00204FF400638382704763
:108930004FF40063838270474FF480538382704703
:10894000BFF34F8F0549064BCA6802F4E062134338
:10895000CB60BFF34F8F00BFFDE700BF00ED00E02D
:108960000400FA05F8B5057B466903681F2D29D96F
:10897000A5F120045F682021A1400F422A4613D0B0
:108980001022A240D960DA605A68E240D10703D5CC
:10899000012202FA04F4DC6004463046FFF730FBA3
:1089A000227B23681F2A20D9A2F1200008215A68BF
:1089B0008140114200D0D9600422596882400A42A5
:1089C00021D1F8BD20211C68A9400C422A460CD0B8
:1089D0001022AA4099609A601A68EA40D207DBD553
:1089E000012202FA05F59D60D6E70821186891403A
:1089F000014200D099600421186801FA02F2024293
:108A000003D09A60F8BDDA60F8BDF8BD70B4037B9E
:108A100004681F2B08D9203B2021626801FA03F368
:108A20001A421CD170BC70472021226801FA03F35E
:108A30001A42F7D042691449582000FB02125168CB
:108A40005689CD680868296821F00101296082896A
:108A500092B222EA06028281A36070BC704742692A
:108A60000949582000FB021251685689CD680868F0
:108A7000296821F001012960828992B222EA060266
:108A80008281E36070BC70474C5D002030B4094BBC
:108A90001C786CB1084A002502EBC4041168938865
:108AA0004D628889083203439BB2A2428B81F5D183
:108AB00030BC70470C6000201060002010B4037BB5
:108AC00001681F2B09D9203B20224C6802FA03F3CE
:108AD0001C4214D15DF8044B704720220C6802FA46
:108AE00003F31C42F6D00C4A40680024147002685C
:108AF0005DF8044B22F0010202608B607047064A69
:108B000040680024147002685DF8044B22F00102F2
:108B10000260CB60704700BF0B6C0020F0B5C40052
:108B200022189200AE498B585B689D8AADB2EEB2B6
:108B3000F7070A445CD4B70732D5BFF35F8F167EC0
:108B4000F6B2012E00F0C780A64D1A8BBFF35F8FDF
:108B5000221801EB8202167E022E00F0D580221828
:108B600001EB8202167E032E00F088809A8895F928
:108B7000086092B242F480629A80221801EB82026D
:108B8000127E013296425BD1AA7A00266E72002ACA
:108B900040F09580204401EB800000234375F0BD38
:108BA00077074ED416F0400600F0C9808D4D1E8A1E
:108BB00095F908E0176AF6B207F80E605FFA8EFEC4
:108BC0000EF1010C4FFA8CFC177E85F808C00CF1F1
:108BD00003029742664600F01C81221801EB8202D4
:108BE000127E9445C9D10EF1020676B22E72C4E708
:108BF0001E887C4D26F400663604360C1E801E88C6
:108C0000B6B246F480661E80967E00272F72002E34
:108C100048D06E7A002E42D0221801EB8202012643
:108C2000127E6E72022A00F0B980221801EB8202D5
:108C3000927D42F001021A82204401EB8000037E03
:108C4000F0BD684D967E0127AF72002E73D06E7A0C
:108C5000002E7BD1221801EB8202527E002A00F006
:108C6000A3801A882E7A92B2013642F4007276B24C
:108C70001A802E721A88D205FCD47EE7927E002AD2
:108C80003FF474AF6A7A002A3FF470AF9A8895F97E
:108C9000086022F480621204120C9A806DE7D27D83
:108CA000FF2AB9D0221801EB8202967D06F0FE065B
:108CB0001E82D37DFF2BBFD0FF232B72BCE79A8887
:108CC00022F4407212042044120C01EB80009A80BE
:108CD00000234375F0BD927E424D002A3FF435AF2C
:108CE0006A7A002A3FF431AF1A8822F480621204B3
:108CF000120C1A80BFF35F8F1A8B1A88AE7292B271
:108D000042F400721A8031E7927E002A3FF427AFC6
:108D10006A7A002A3FF423AF1A8895F9086022F492
:108D200080621204120C1A809A8822F48062120463
:108D3000120C9A8021E76A7A002A8BD091E715F00D
:108D4000800F284D3AD195F9086016E7167ED2F8C3
:108D500020E01F88022E95F9086045D927F4806726
:108D60003F043F0C1F801F8AFFB20EF806701F8859
:108D7000D2F820E0BFB247F400771F80F2B21F8A1A
:108D8000561C76B2FFB20EF806709F88961CBAB2D7
:108D900076B242F480622E729A806BE71A8892B2A1
:108DA00042F400621A8040E71A8895F9086092B28E
:108DB00042F4807201271A806F725BE795F90870A0
:108DC000B7F1FF3F2CD0D669F65D1E8292F818E00D
:108DD00001377AB2964516462A727FF4CEAEA3E7E3
:108DE0003C3D0020D01F0020BFB247F400771F8019
:108DF0001F8AFFB20EF80670F6B21F8AD2F820E082
:108E0000721C52B20336FFB276B20EF802702E72A6
:108E100030E79A8822F480621204120C9A80DCE611
:108E2000D77D1F822E72957E1DB9127E002A7FF497
:108E300003AF9A8822F480621204120C9A80FBE637
:108E400070B5044682B01430E56D06236A464321AE
:108E5000A847B0B19DF804009DF800609DF801108E
:108E60009DF802509DF803209DF8053041EA062147
:108E700043EA002342EA0522A187E287A4F84030B2
:108E8000012002B070BD00BF70B5044682B008304A
:108E9000656A06236A463B21A847A8B19DF80400ED
:108EA0009DF800609DF801109DF802509DF8032088
:108EB0009DF8053041EA062143EA002342EA0522F3
:108EC000E18222836383012002B070BD50F8043C2C
:108ED000012280F84520103803B11847704700235D
:108EE000012243608360036003714370C271837227
:108EF000837043710272C3727047F8B50468C4F39B
:108F00000D0405460E4604B32F6830F0B5FD092860
:108F100040F08880454C236923F440732361236922
:108F200043F400732361236943F0010323613E602E
:108F300030F0A2FD2369092823F00103236171D1D8
:108F40002B6804332B600020F8BD394B394A93421B
:108F50002BD902F58042934226D902F580429342F2
:108F60002AD902F58042934228D902F580329342F1
:108F700026D902F50032934224D902F500329342F9
:108F800022D902F50032934220D902F500329342F1
:108F90001ED902F5802293421CD9B3F1016F1BD375
:108FA000052005F08BFAFBE7082430F065FD092861
:108FB00014D04FF0FF30F8BD1024F6E71824F4E782
:108FC0002024F2E72824F0E73024EEE73824ECE709
:108FD0004024EAE74824E8E75824E6E7134F3B69D2
:108FE00023F440733B613B6943F400733B613B698D
:108FF00023F0F8033B613B6943F002031C433C61EF
:109000003B6943F480333B6130F036FD3B6923F02C
:1090100002033B613B69092823F0F8033B613FF4FD
:1090200073AFC6E76FF00100F8BD00BF003C02401F
:1090300000400008FF3F0008F8B504460D468E18B2
:109040000027B54201D12069F8BDE368591CE160F1
:10905000234415F8012B1A720429F2D1206918B99A
:10906000A1682046FFF749FF2061E760E9E700BFFC
:1090700070B582B00446694614302BF037FDB0B1AC
:109080009DF805009DF801609DF802109DF80350C1
:109090009DF804209DF8063041EA062143EA0023AA
:1090A00042EA0522A187E287A4F84030012002B0FD
:1090B00070BD00BF38B5254B9C68236B73B1636DE1
:1090C000626BCAB1998A1A88C90592B201D5D207D2
:1090D00000D438BD4FF6F7721A8038BD636D998998
:1090E0001A88890692B2EBD59206E9D5E26ACAB12E
:1090F000988880B29047E2E799891A880D0692B263
:10910000E0D51006DED5A26A616A8A4219D0A1694B
:109110002569885C98800132B2FBF5F105FB1122CC
:10912000A262CFE79B88E2696169DBB28B54E26996
:10913000E068636D0132B2FBF0F100FB1122E261E5
:10914000BEE7DA6822F08002DA60BBE7143D002057
:1091500038B5254B1C68236B73B1636D626BCAB164
:10916000998A1A88C90592B201D5D20700D438BDB0
:109170004FF6F7721A8038BD636D99891A8889068F
:1091800092B2EBD59206E9D5E26ACAB1988880B26C
:109190009047E2E799891A880D0692B2E0D5100649
:1091A000DED5A26A616A8A4219D0A1692569885C04
:1091B00098800132B2FBF5F105FB1122A262CFE7E4
:1091C0009B88E2696169DBB28B54E269E068636D98
:1091D0000132B2FBF0F100FB1122E261BEE7DA6876
:1091E00022F08002DA60BBE7143D002003685B6A6E
:1091F00003B11847704700BF03681B6A03B11847E3
:10920000704700BF03682DE9F041DF691FB13B469D
:10921000BDE8F0411847002A164611DD04460D4608
:109220000E4400E023689B68204698470028F9D048
:10923000236815F8011B1B6820469847AE42F1D100
:10924000BDE8F08103689B69184700BF03685B694C
:10925000184700BF03681B69184700BF0368DB6835
:10926000184700BF03689B68184700BF03685B6826
:10927000184700BF03681B68184700BF014B1868F8
:10928000F8E700BF70B6002038B50C46097849B140
:10929000054601342B6828461B68984714F8011BC3
:1092A0000029F7D138BD00BF064B53F820302BB151
:1092B0001A689B8851690B4201D11383704753830D
:1092C000704700BFDC95002003682DE9F04F03F1E3
:1092D0003F4404F57E04604EA40A0125345D04F089
:1092E0001F066409032C05FA06F500F0AF80042C74
:1092F00000F0A780022C54D08588B5FA85F0C0F123
:109300001F0080B2C40803EB840400F00700266A43
:1093100080000F27874026EA07062662276A01F0A9
:10932000030602FA00F0721E3843012AC1F3810CD1
:10933000C1F300182062C1F3411137D9002422463D
:1093400001274FF0030E03E0102A04F1020426D097
:1093500007FA02F0A84302F10102F5D1D3F800C0E8
:109360000EFA04F0C04300EA0C0CC3F800C0D3F8B6
:10937000008006FA04FC4CEA080CC3F800C0D3F8DD
:109380000CC000EA0C00D860D3F80CC001FA04F05D
:1093900040EA0C00102AD86004F10204D8D1BDE8DC
:1093A000F08F2E4C666C35436564A5E700200246BD
:1093B0004FF0010E4FF0030904E00132102A00F1D2
:1093C00002003CD00EFA02F737EA0504F5D1D3F8D3
:1093D00000A009FA00F4E4430AEA040AC3F800A072
:1093E000D3F800B006FA00FA4AEA0B0AC3F800A064
:1093F000D3F808A004EA0A0AC3F808A0D3F808B012
:109400000CFA00FA4AEA0B0AC3F808A0D3F804A041
:109410002AEA07075F60D3F804A008FA02F747EAD0
:109420000A075F60DF683C40DC60DF6801FA00F437
:1094300001323C43102ADC6000F10200C2D1BDE8D9
:10944000F08F064C266B3543256355E7034C266C9D
:109450003543256450E700BFB01D040800380240C2
:10946000026802F13F4303F57E032DE9F04F9B0AAA
:10947000544DEB5C03F01F055B090124032B04FA38
:1094800005F400F09980042B00F09180022B3ED06F
:1094900001F00306731E012BC1F3810CC1F3001808
:1094A0008588C1F3411137D90024234601274FF0A5
:1094B000030E03E0102B04F1020426D007FA03F098
:1094C000A84303F10103F5D1D2F800C00EFA04F06D
:1094D000C04300EA0C0CC2F800C0D2F8008006FAC3
:1094E00004FC4CEA080CC2F800C0D2F80CC000EA38
:1094F0000C00D060D2F80CC001FA04F040EA0C0075
:10950000102BD06004F10204D8D1BDE8F08F2E4BAF
:109510005D6C2C435C64BBE7002003464FF0010EFA
:109520004FF0030904E00133102B00F102003CD09E
:109530000EFA03F737EA0504F5D1D2F800A009FACC
:1095400000F4E4430AEA040AC2F800A0D2F800B02A
:1095500006FA00FA4AEA0B0AC2F800A0D2F808A0FC
:1095600004EA0A0AC2F808A0D2F808B00CFA00FA15
:109570004AEA0B0AC2F808A0D2F804A02AEA0707B0
:109580005760D2F804A008FA03F747EA0A075760C1
:10959000D7683C40D460D76801FA00F401333C43FB
:1095A000102BD46000F10200C2D1BDE8F08F064B51
:1095B0001D6B2C431C636BE7034B1D6C2C431C641D
:1095C00066E700BFB01D04080038024010B504096A
:1095D000013C032C17D80D4B33F8142000F00F007A
:1095E00042FA00F313F001030DD0012303FA00F057
:1095F0000138104033F03AF8054A064B125D10442A
:1096000003EBC00010BD002010BD00BFDC1D04082E
:10961000D81D0408509400202DE9F04F4A484B49CA
:109620004B4B4C4C4FF0010A4FF002094FF004082D
:109630004FF0080C4FF0100E20274026802530F800
:10964000022B12F0010F03D01960A3F804A0083315
:1096500012F0020F03D01960A3F80490083312F03F
:10966000040F03D01960A3F80480083312F0080F28
:1096700003D01960A3F804C0083312F0100F03D010
:109680001960A3F804E0083312F0200F02D019602B
:109690009F80083312F0400F02D019609E8008337B
:1096A00012F0800F02D019609D80083312F4807F81
:1096B00005D04FF4807B1960A3F804B0083312F48E
:1096C000007F05D04FF4007B1960A3F804B0083385
:1096D00012F4806F05D04FF4806B1960A3F804B0CA
:1096E000083312F4006F05D04FF4006B1960A3F833
:1096F00004B0083312F4805F05D04FF4805B19602A
:10970000A3F804B0083312F4005F05D04FF4005BF7
:109710001960A3F804B0083312F4804F05D04FF459
:10972000804B1960A3F804B00833D20B04D04FF477
:10973000004219609A80083301F58061A1427FF4EC
:109740007EAFBDE8F08F00BFDC1D040800000240C2
:10975000509400200010024000286AD003682DE9D0
:10976000F04F03F13F4404F57E045F4EA40A012547
:10977000345D04F01F066409032C05FA06F559D080
:10978000042C00F0AC80022C59D08588B5FA85F005
:10979000C0F11F0080B2C40803EB840400F007008E
:1097A000266A80000F27874026EA07062662276A76
:1097B00001F003068240701E3A430128C1F3810C78
:1097C000C1F300182262C1F341113DD900242246A1
:1097D00001274FF0030E03E0102A04F1020426D003
:1097E00007FA02F0A84302F10102F5D1D3F800C054
:1097F0000EFA04F0C04300EA0C0CC3F800C0D3F822
:10980000008006FA04FC4CEA080CC3F800C0D3F848
:109810000CC000EA0C00D860D3F80CC001FA04F0C8
:1098200040EA0C00102AD86004F10204D8D1BDE847
:10983000F08F70472D4C266C35432564A5E72B4CE3
:10984000666C35436564A0E7002002464FF0010EC8
:109850004FF0030904E00132102A00F102003CD06D
:109860000EFA02F737EA0504F5D1D3F800A009FA99
:1098700000F4E4430AEA040AC3F800A0D3F800B0F5
:1098800006FA00FA4AEA0B0AC3F800A0D3F808A0C7
:1098900004EA0A0AC3F808A0D3F808B00CFA00FAE0
:1098A0004AEA0B0AC3F808A0D3F804A02AEA07077B
:1098B0005F60D3F804A008FA02F747EA0A075F607E
:1098C000DF683C40DC60DF6801FA00F401323C43B1
:1098D000102ADC6000F10200C2D1BDE8F08F034C19
:1098E000266B3543256350E7B01D0408003802405D
:1098F000002855D0026802F13F4303F57E032DE9AD
:10990000F04F9B0A544DEB5C03F01F055B090124EB
:10991000032B04FA05F444D0042B00F09780022BAB
:1099200044D001F00306731E012BC1F3810CC1F377
:1099300000188588C1F341113DD900242346012731
:109940004FF0030E03E0102B04F1020426D007FAB7
:1099500003F0A84303F10103F5D1D2F800C00EFAD9
:1099600004F0C04300EA0C0CC2F800C0D2F800803A
:1099700006FA04FC4CEA080CC2F800C0D2F80CC08D
:1099800000EA0C00D060D2F80CC001FA04F040EA02
:109990000C00102BD06004F10204D8D1BDE8F08F88
:1099A00070472E4B1D6C2C431C64BAE72B4B5D6C2F
:1099B0002C435C64B5E7002003464FF0010E4FF0E6
:1099C000030904E00133102B00F102003CD00EFA31
:1099D00003F737EA0504F5D1D2F800A009FA00F43C
:1099E000E4430AEA040AC2F800A0D2F800B006FA7A
:1099F00000FA4AEA0B0AC2F800A0D2F808A004EA6A
:109A00000A0AC2F808A0D2F808B00CFA00FA4AEA2A
:109A10000B0AC2F808A0D2F804A02AEA0707576088
:109A2000D2F804A008FA03F747EA0A075760D76894
:109A30003C40D460D76801FA00F401333C43102B5A
:109A4000D46000F10200C2D1BDE8F08F034B1D6B62
:109A50002C431C6365E700BFB01D040800380240BA
:109A600038B590F8593003B938BD04461846FFF7A9
:109A7000ADFD0546D0B1202300218371C171FFF7F0
:109A800037FF21460F4B41F8103F28462AF0C0FF10
:109A9000AB88B3FA83F3C3F11F03012212FA03F375
:109AA000E2D009490A6813430B6038BD0146FFF74D
:109AB0001FFF2146034B41F8103F2846BDE83840C0
:109AC0002AF0A6BFCD8E0008003C014038B5044600
:109AD00000F11405FFF7C4FF236E80226B21284696
:109AE0009847642005F096F9236E072268212846DE
:109AF0009847642005F08EF9236E00226B212846DA
:109B00009847642005F086F9236E01226B212846D0
:109B100098470F2005F07EF994F85320236E032A0E
:109B20008CBF1A2218221B21284698470F2005F0C7
:109B300071F9236E18221C21284698470F2005F042
:109B400069F9236E94F852201A21284698470F206D
:109B500005F060F9236E94F854201921284698479F
:109B6000642005F057F9236E1022372128469847C4
:109B70000F2005F04FF92846236E0122382198471F
:109B80000F20BDE8384005F045B900BF10B10368AB
:109B900082885A83704700BF10B1036882881A8395
:109BA000704700BF18B10368828809B95A837047AB
:109BB0001A83704710B40A4B0A4A1C780123834069
:109BC000234052F8200029B9B3FA83F149095DF81E
:109BD000044BE7E7191C18BF01215DF8044BE1E7CE
:109BE000D8950020DC95002030B1036882881B697D
:109BF0001A4214BF01200020704700BF2DE9F04138
:109C00000B4E346873691C400FD0DFF828800127A1
:109C1000B4FA84F3C3F11F0307FA03F558F82300DD
:109C200003689847AC437561F2D1BDE8F08100BF8D
:109C3000003C0140189600202DE9F0410B4E34689D
:109C400073691C400FD0DFF828800127B4FA84F331
:109C5000C3F11F0307FA03F558F823000368984778
:109C6000AC437561F2D1BDE8F08100BF003C01401A
:109C7000189600202DE9F0410B4E346873691C40A2
:109C80000FD0DFF828800127B4FA84F3C3F11F0353
:109C900007FA03F558F8230003689847AC43756149
:109CA000F2D1BDE8F08100BF003C014018960020D1
:109CB0002DE9F0410B4E346873691C400FD0DFF87A
:109CC00028800127B4FA84F3C3F11F0307FA03F5D0
:109CD00058F8230003689847AC437561F2D1BDE89A
:109CE000F08100BF003C0140189600202DE9F041B2
:109CF0000B4E346873691C400FD0DFF828800127B1
:109D0000B4FA84F3C3F11F0307FA03F558F82300EC
:109D100003689847AC437561F2D1BDE8F08100BF9C
:109D2000003C0140189600202DE9F0410B4E3468AC
:109D300073691C400FD0DFF828800127B4FA84F340
:109D4000C3F11F0307FA03F558F823000368984787
:109D5000AC437561F2D1BDE8F08100BF003C014029
:109D6000189600202DE9F0410B4E346873691C40B1
:109D70000FD0DFF828800127B4FA84F3C3F11F0362
:109D800007FA03F558F8230003689847AC43756158
:109D9000F2D1BDE8F08100BF003C014018960020E0
:109DA000084A094808B5536C43F4804353640021C2
:109DB000402234F0D6FF054B4FF0FF321A60C3F853
:109DC000032008BD00380240189600205896002055
:109DD00003685B6A184700BF2DE9F0410446184646
:109DE0000D461646984631F097FF2768E6722844DC
:109DF000A07229467D69434632462046AC46BDE8FE
:109E0000F0416047036810B504461B689847236813
:109E100020469B689847A37B0133A37310BD00BF06
:109E200010B5036804469B689847FF2301226373BB
:109E3000227310BD08B5FFF7C9FB38B12C2282711F
:109E40000022C2712021BDE8084051E508BD00BFD5
:109E500040F2E93300E0A3B10289013B12F0020FA6
:109E60009BB2F8D089B2818140F2E93300E043B17E
:109E70000289013B12F0010F9BB2F8D08089C0B279
:109E80007047094A904205D0084B984201D0FF2004
:109E900070470223064A02EB03135A89013292B239
:109EA0005A815889C0B2704700300140003C0040E0
:109EB000388C002010B5014600BF074C2368986815
:109EC000FFF764FE23685868FFF7C2FF23689868AD
:109ED000FFF762FE00BF10BDAC960020144B984205
:109EE00024D003F58063984220D0028822F04002FB
:109EF0001204120C0280028822F038031B041B0C8F
:109F000059B141F48071002991FAA1F2B2FA82F1BB
:109F100008BF4FF0FF310139C9000B439BB20380EA
:109F200003889BB243F04003038070474908DCE795
:109F30000038004010B5802104468069FFF7CEFF4D
:109F4000012004F00DFF2046FFF7C0FD10226A211A
:109F500004F11400FEF770F9642004F05BFFA069BF
:109F60000421FFF7BBFF0120BDE8104004F0F8BE5C
:109F7000F8B5464E0446FFF773FDF77ADFB104F1FA
:109F800014054FF48071A069FFF7A8FF94F85220E0
:109F90001A212846FEF750F9012004F0E1FE0421C1
:109FA000A069FFF79BFF2046FEF74AFF94F93E3079
:109FB000013362D0F8BD04F114054FF48071A0693B
:109FC000FFF78CFF80226B212846FEF735F996209B
:109FD00004F020FF032268212846FEF72DF9962081
:109FE00004F018FF03226B212846FEF725F90F2005
:109FF00004F0B6FE10226A212846FEF71DF90F2054
:10A0000004F0AEFE3A466C212846FEF715F90F2003
:10A0100004F0A6FE94F8542019212846FEF70CF906
:10A020000F2004F09DFE18221B212846FEF704F99C
:10A030000F2004F095FE10221C212846FEF7FCF8A4
:10A040000F2004F08DFE102237212846FEF7F4F889
:10A050000F2004F085FE012238212846FEF7ECF897
:10A060000F2004F07DFE0421A069FFF737FF0120D7
:10A0700004F076FE0123F37283E794F93C30013358
:10A0800098D10620BDE8F84004F018BAD01F00208F
:10A09000F8B5654C0601A7190546387A2AF014F878
:10A0A0003B7A03F01F015B090122032B02FA01F244
:10A0B0006DD0042B66D0022B5CD0A3190135187922
:10A0C000FFF784FAEDB2074610B11223C571837110
:10A0D000A3195879FFF77AFA10B11323C571837168
:10A0E000A3199879FFF772FA10B11423C57183711F
:10A0F000A5190A21EA793846FFF72EFB6879FFF7A0
:10A1000065FAEA790A21FFF727FBA879FFF75EFADB
:10A11000EA790A21FFF720FBA359444A934247D02A
:10A12000434A934250D0434A934259D0424A9342C1
:10A1300062D0424A93426BD0414A93422CD034447D
:10A14000227BE2B901200222198801F4415141F435
:10A1500045710A4302431A809A8B22F4006212046A
:10A16000120C07219A8319821A8892B242F0400297
:10A170001A80F8BD334B596A0A435A629DE70020A2
:10A180000246E1E72F4B19690A431A6195E72D4B07
:10A19000196A0A431A6290E702F564424FF400100C
:10A1A000536A43F4001353622FF00CFCA359C6E723
:10A1B00002F584324FF48050536A43F48053536263
:10A1C0002FF000FCA359BAE702F500324FF48040AB
:10A1D000136A43F4804313622FF0FCFBA359AEE7EC
:10A1E00002F5FE324FF40040136A43F40043136259
:10A1F0002FF0F0FBA359A2E702F582324FF4005092
:10A20000536A43F4005353622FF0DCFBA35996E7E3
:10A2100002F568424FF48010536A43F4801353628E
:10A220002FF0D0FBA3598AE7388C00200030014082
:10A2300000380040003C0040003401400050014024
:10A240000054014000380240427A02B9704710B50C
:10A2500004460368406804F10A01984700236372CA
:10A2600010BD00BF437A5A1C0344D2B242729972A5
:10A27000037A934200D802B9704710B504460368C8
:10A28000406804F10A0198470023637210BD00BFC3
:10A29000302827D0312827D0322827D0332827D07C
:10A2A000342827D0352827D0202827D0212827D088
:10A2B000102827D0112827D0122827D0132827D0DC
:10A2C000142827D0152827D0162805D0172808BF0E
:10A2D0000F2202D0002070470E22104B03EB4203E6
:10A2E000587E70470022F8E70122F6E70222F4E7E1
:10A2F0000322F2E70422F0E70522EEE70622ECE76C
:10A300000722EAE70822E8E70922E6E70A22E4E76B
:10A310000B22E2E70C22E0E70D22DEE7CCEE030899
:10A3200070B5448806460D46C4F30B04224600214E
:10A33000284634F016FD3369094A934209D3094A85
:10A34000934206D2224628461946BDE8704032F0B4
:10A3500087BA23B121462846BDE87040184770BD32
:10A36000240600082A070008064B07498B4202D33F
:10A370000023184670471A88C2F30B029042F8D0A7
:10A380001433F3E78801000824060008024A136822
:10A3900023EA0000106070470C7B0020F8B5174DD1
:10A3A0002B78A32B28D16B78BE2B25D102222946EE
:10A3B0004FF6FF70FEF79AF9114FAC1C22884AB194
:10A3C000A618BE4218D2052A16D92146FEF78EF9E4
:10A3D0003446F3E721460222FEF788F90222A1184B
:10A3E000FEF784F90634074B641B1C8041F60F53BB
:10A3F000C31A58425841F8BD0020F8BD004000087B
:10A4000000800008BA3E00202DE9F04FDFF84C91A3
:10A410004D4F8BB00326A7EB09071822002104A893
:10A4200034F09FFC494BCDF8109005971A69002A2B
:10A4300004DA474A5A6002F188325A6001228DF8E4
:10A440002420F322DA60434B434C1B88ADF80030E4
:10A450000222694604A8FEF7EFFD022269464FF684
:10A46000FF70FEF743F9DFF8F8A080464FF0000BCD
:10A47000544539D30AAC002524F8245D0222214634
:10A4800004A8FEF7D9FD022221464046FEF72EF928
:10A4900040BAC043ADF80800022202A904A8FEF7A2
:10A4A000CBFD079878B106ABC0F1040229461844E9
:10A4B00034F057FC089818B9069904A8FEF71DFD5A
:10A4C0000023089007939DF82430089A23B11F4970
:10A4D0000B6943F000430B61013E2DD0002A9CD153
:10A4E000FFF75CFF50B32CE065888DF80DB0C5F325
:10A4F0000B05AB1DADF808302388C3F30B02ADF894
:10A500000A201B0B062202A904A88DF80C30FEF7C6
:10A5100093FD062202A94046FEF7E8F861688046EE
:10A520002A4604A8FEF788FD616840462A46FEF7E1
:10A53000DDF8143480469BE7002AD1D0052003F0D3
:10A54000BDFF0BB0BDE8F08F00800008003C02406A
:10A550002301674504EF0308880100080040000854
:10A56000240600080378202B024600F10100F9D0F0
:10A57000092BF7D02D2B2CD02B2B03BF5378B7EE04
:10A58000000A0246B7EE000AA3F13001C8B209285A
:10A590009FED467A10D8F2EE046A07EE901AF8EEB4
:10A5A000E77A12F8013FE7EE267AA3F13001C8B24C
:10A5B0000928B0EE677AF0D92E2B4CD003F0DF03D8
:10A5C000452B0BD0F7EE007A67EE276A20EE260ABD
:10A5D00070475378BFEE000A0246D5E710B45178B1
:10A5E0002D2959D02B290ABF9178501C901C00248A
:10A5F000A1F13003092B53D8002303EB830301EBB4
:10A60000430310F8011FA1F13002092AA3F130031E
:10A61000F3D9B3F59A7F28BF4FF49A73072B42D929
:10A62000DFED236A1A46F7EE007A083A072A67EE4A
:10A63000A67AFAD803F007032BB1F2EE046A013BC5
:10A6400067EEA67AFBD124B3C7EE276A5DF8044B08
:10A6500020EE260A70475378A3F13001C8B20928CA
:10A6600002F10102AAD8F2EE046AF0EE665A07EE91
:10A67000901AF8EEE77A12F8013F87EEA66AA3F186
:10A680003001C8B2092866EEA56A37EE067AEED91F
:10A6900094E767EE276AD9E7901C91780124A7E731
:10A6A000F7EE007ACFE7F7EE007AC5E7000000008A
:10A6B00020BCBE4CB5EEC00ADFED317AF1EE10FAE7
:10A6C000CCBF30EE270A30EE670ADFED2E7A20EE9F
:10A6D000270A30B5FDEEC07A87B017EE904A0546DE
:10A6E00084EAE470002303A9A0EBE47001930093D3
:10A6F000029320F0D9F9002CACBF20232D2303A80E
:10A700008DF8003031F008FB012803A924D002287D
:10A710002DD0032805BF3023684668468DF80130E8
:10A7200034F045FB684631F0F7FA0338C4B22246EC
:10A730006946284634F099FB00232B55284631F012
:10A74000EBFA2E22431C2A540DEB0401E81834F0D6
:10A750004BFB284607B030BD302368468DF80130EA
:10A760008DF802308DF8033034F021FBDAE7302326
:10A7700068468DF801308DF8023034F018FBD1E7CF
:10A780006F12033A00007A442DE9F041064615465F
:10A790000846B6FBF2F43CB905FB1464124B1B5D92
:10A7A00000F8013BBDE8F081B4FBF2F767B90E4B4E
:10A7B00005FB174705FB1464DA5D00F8012B1B5DF0
:10A7C00000F8013BBDE8F081B7FBF2F8B8F1000FEB
:10A7D00002D04046FFF7D8FF05FB1878024B13F86C
:10A7E000082000F8012BE3E7CC23040830B402680A
:10A7F0001146531C036011F8024B0160D31C5178C1
:10A8000003609378151D05601B0443EA0123D0788B
:10A81000234343EA006030BC704700BF0368591C03
:10A820001A46016012F8021B0260587841EA0020C3
:10A83000704700BF03685A1C02601878704700BF59
:10A8400038B504460068154632F00AF822682A44F2
:10A85000226038BD036810B40A0E5C1C04601A70D4
:10A8600003680A0C5C1C04601A7003680A0A5C1C0A
:10A8700004601A7003685A1C026019705DF8044B7A
:10A88000704700BF036810B40A0A5C1C04601A70A9
:10A8900003685A1C026019705DF8044B704700BFD2
:10A8A00003685A1C026010B4197003680A0A5C1C21
:10A8B00004601A7003680A0C5C1C04601A70036858
:10A8C000090E5A1C026019705DF8044B704700BFF6
:10A8D00003685A1C026019700368090A5A1C026056
:10A8E000197070472DE9F047002488B080460F4664
:10A8F0001E46A14605AD531C0393117839B3252993
:10A9000033D1931CCDF810900393507830284ED05B
:10A910004FF0000AA0F13003DBB2092B42D96C28BA
:10A9200019D0642800F0938024D825281CD063D93E
:10A93000582876D063281BD131784046B847039A0F
:10A94000531C03931178043601340029D7D12046D3
:10A9500008B0BDE8F087039B5A1C03921B78642B58
:10A960007CD02AD8252B54D1252140460134B84724
:10A97000039AC0E7732833D044D975284FD106F124
:10A98000040E30682B4600220A217646FDF7A4FD0E
:10A99000049A0095534639464046FDF7DBFD039A7D
:10A9A0000444A8E704AA03A920F05AF8B7E7D31C87
:10A9B000039390784FF0010AACE7732B10D05BD96A
:10A9C000752B3AD0782B96D1A3F15802B2FA82F2C5
:10A9D000306852092B4610210436FDF77DFDD7E77C
:10A9E0003368049A0093394600234046FDF7B2FDD0
:10A9F00004360444039A7EE70028B9D1204608B003
:10AA0000BDE8F0876E28B3D1039A336804361C6022
:10AA100071E72AD9582BD7D0632B8DD06BE77828D4
:10AA2000A6D1A0F15802B2FA82F2306852092B4640
:10AA30001021FDF751FD0436AAE706F1040E306837
:10AA40002B4600220A217646FDF746FDA0E7331D7E
:10AA5000306829461E46FDF711FD99E7331D306821
:10AA600029461E46FDF70AFD92E7002B7FF443AF0F
:10AA7000204608B0BDE8F0876E2BC6D03BE700BF8C
:10AA80000EB400B584B005AB019053F8042B064911
:10AA9000039301A8FFF726FF019B00221A7004B060
:10AAA0005DF804EB03B07047498500080FB430B57A
:10AAB00083B006AB0A490B4853F8042B09680068B9
:10AAC0000193FFF70FFF084C05462068FEF7BEFB19
:10AAD0000028FAD0284603B0BDE8304004B07047E3
:10AAE000083D00200C3D002070B60020DFED2B7AE1
:10AAF000B4EEE70AF1EE10FA4ADDDFED296A9FEDC8
:10AB0000297A01E0B0EE670AB4EEC70AF1EE10FA56
:10AB100070EE667AF6DC9FED247AF4EEC77AF1EEF9
:10AB200010FA38D5DFED1E6A9FED207A01E0F0EED5
:10AB3000407AF4EEC77AF1EE10FA37EEA60AF6D4B0
:10AB4000DFED1B7AB4EEE70AF1EE10FA14DDDFED6B
:10AB5000137A37EEC00A60EE006A9FED166A9FED29
:10AB6000167ADFED167AA6EE867A20EE266AE6EEF3
:10AB7000877AA6EE270A7047DFED117AB4EEE70A6E
:10AB8000F1EE10FA44BFDFED087A37EEC00AE2E7D3
:10AB9000F0EE407ABFE7B0EE670AD1E7DB0F49403D
:10ABA000DB0FC940E4CB1641DB0F49C0E4CB16C133
:10ABB000DB0FC93F92E741B99730083C15A82ABE80
:10ABC000DB0FC9BF80EAE073A3EBE0738B4205DBC8
:10ABD000002801DD401A704702D1704700207047FD
:10ABE0000844704709B909E0194690FBF1F301FBED
:10ABF00013030846002BF7D1084670470146FBE7D0
:10AC0000F0EEC07AB0EEE07AB4EEE77AF1EE10FA48
:10AC1000B4BFB0EE676AB0EE476AB5EE406AF1EED7
:10AC200010FA46D0B4EEE77AF1EE10FA8CBFF0EEEF
:10AC3000675AF0EE475AC5EE866A9FED1F3A9FEDC0
:10AC40001F6A9FED1F4A9FED1F5ADFED1F3ADFED90
:10AC50001F4ADFED1F5AA6EEC36AE6EEA34AA6EE30
:10AC6000864AB7EE006AA6EE845AA6EEA46AE6EE1D
:10AC7000855AC5EE866AB4EEE77AF1EE10FA48BF5F
:10AC8000DFED147AF5EEC00A48BF77EEE66AF1EE22
:10AC900010FA48BFDFED107AB5EEC00A48BF77EE74
:10ACA000E66AF1EE10FA48BFF1EE666AB0EE660AA7
:10ACB0007047DFED076ADEE739094E3DE3B59E3E9A
:10ACC00088FA163E45FE7F3F99FB243F69A2163E57
:10ACD000A7DFA834DB0FC93FDB0F4940DFED317A36
:10ACE00030EE277AFDEEC76A16EE903A2033402BFD
:10ACF00002D99FED2D0A7047B4EEE70AF1EE10FA83
:10AD00004DDD9FED2A6ADFED2A6A01E0B0EE677A39
:10AD1000B4EEE67AF1EE10FA77EE467AF6DC9FEDC5
:10AD2000257AF4EEC77AF1EE10FA35D5DFED1F6A19
:10AD30009FED217A01E0F0EE407AF4EEC77AF1EE71
:10AD400010FA37EEA60AF6D4DFED167AB4EEE70A6B
:10AD5000F1EE10FA1BDCDFED197AB4EEE70AF1EE42
:10AD600010FA44BFDFED137A37EEC00A60EE006AD6
:10AD70009FED136A9FED137ADFED137AA6EE867AC4
:10AD800020EE266AE6EE877AA6EE270A7047DFED08
:10AD90000F7A37EEC00AE9E7B0EE670AD4E7F0EEC3
:10ADA000477ABCE7DB0FC93F00000000DB0FC9405A
:10ADB000E4CB1641DB0F49C0E4CB16C1DB0FC9BFA2
:10ADC00092E741B99730083C15A82ABEDB0F4940ED
:10ADD000FDEEC07A17EE903A2033402B51D8DFEDCC
:10ADE0002D7AB4EEE70AF1EE10FA50DDDFED2A6AB3
:10ADF0009FED2A7A01E0B0EE670AB4EEC70AF1EEE1
:10AE000010FA70EE667AF6DC9FED257AF4EEC77ADA
:10AE1000F1EE10FA38D5DFED206A9FED227A01E0DD
:10AE2000F0EE407AF4EEC77AF1EE10FA37EEA60AA9
:10AE3000F6D4DFED1D7AB4EEE70AF1EE10FA1BDC72
:10AE4000DFED1A7AB4EEE70AF1EE10FA44BFDFED57
:10AE5000147A37EEC00A60EE006A9FED156A9FED26
:10AE6000157ADFED157AA6EE867A20EE266AE6EEF2
:10AE7000877AA6EE270A7047DFED067A37EEC00A1A
:10AE8000E9E79FED0E0A7047B0EE670AD1E7F0EEF2
:10AE9000407AB9E7DB0F4940DB0FC940E4CB1641EC
:10AEA000DB0F49C0E4CB16C1DB0FC93FDB0FC9BFC5
:10AEB00092E741B99730083C15A82ABE000000006F
:10AEC00010B507EE901A2DED028BB8EE678ADFED14
:10AED000217A28EE008A044628EE278AB0EE480A36
:10AEE00031F07EFEF0EE408AB0EE480A31F0DAFD35
:10AEF000F7EE007A9FED187AF0EE675AE8EE875A7F
:10AF00000023A361B0EE676AC7EEA56A636123629E
:10AF1000E361A8EEC76ABDEC028B77EEC07AB6EEAD
:10AF2000007AF8EE005A27EE877A20EE250A27EEFF
:10AF3000267A26EE266A67EEA67A20EE260A84EDA9
:10AF4000046AC4ED017A84ED007A84ED027A84ED1E
:10AF5000030A10BD27D4D236F304353F10B44C0990
:10AF6000012250F8243001F01F0102FA01F10B43D5
:10AF700040F824305DF8044B704700BF4B0901F0E6
:10AF80001F0150F82320012303FA01F1114214BFDD
:10AF900018460020704700BF074A084B10781B78FE
:10AFA000074A834296BFC31AC3F180030020126888
:10AFB00018441044704700BFBCAB002039AB0020E0
:10AFC000448B0020064A074B10781B7883428ABFC7
:10AFD000C3F18003C01AC018C0F17F00704700BFE2
:10AFE000BCAB002039AB002030B5144C237883B0C3
:10AFF0001BB90120237003B030BD052200238DF85A
:10B0000000208DF8013000BF0D4D2B689868FEF7C9
:10B01000BDFD2B6801AA6946586829F01BF92B6809
:10B020009868FEF7B9FD00BF9DF8053003F00103F5
:10B0300083F00100237003B030BD00BFBE96002036
:10B04000AC96002070B5064C0646256803E02368E0
:10B050005B1BB34203D8FFF7C7FF0028F7D070BDD2
:10B06000109600202DE9F04F89B0B2F1000A02904D
:10B070000491039340F3B0800B46002201EB8A0158
:10B0800053F8040B8B420244FAD1039B0592002B28
:10B0900000F09A80059B002B6AD0544B059A1B68E0
:10B0A000DFF85C9100920099DAB25118B1F5807F17
:10B0B0008CBFC2F58072009A01924D4A92689A4202
:10B0C0006DD9190C1A0A4FF0020406208DF81F30B2
:10B0D0008DF81E208DF81D108DF81C40FFF7B2FF73
:10B0E0000620FEF7E7FE434A0123137000BFD9F89C
:10B0F00000309868FEF74AFDD9F8003007A9586873
:10B10000002229F05FF80024049D029E019FA346BF
:10B1100029684FEA840800220B46013471B1B94214
:10B120002AD2D9F8000031684068FDF70DF92A6885
:10B13000336813443360BF1AC5F800B0A24505F167
:10B14000040506F10406E3D1D9F800309868FEF74B
:10B1500023FD00BF254B019900981B68421A0092FD
:10B16000224A0B441360039A32B3009A002A9AD100
:10B17000059809B0BDE8F08F029CD9F8003054F86A
:10B180000810586800223B46FDF7DEF854F8082006
:10B190002B683A44DF1B44F808202F60D4E7059859
:10B1A000009C1549154A001B0590059800230B705B
:10B1B000137009B0BDE8F08F059B009A9B1A0593A8
:10B1C000059809B0BDE8F08FFFF70EFF00287FF467
:10B1D00061AF039B0593CBE7039C1CB9FFF704FF0A
:10B1E0000594C5E700230593C2E700BF448B002008
:10B1F000040F0020BE960020BCAB002039AB00201D
:10B20000AC96002070B5104D104E2B7831788B42E3
:10B2100084B016D00E4A03921A4402928CBF0C4698
:10B22000CA1A04A98CBFC3F180020024012341F88B
:10B23000102D02A802220194FFF714FF002333709F
:10B240002B7004B070BD00BF39AB0020BCAB002038
:10B250003CAB002070B5194C194D237829789942E0
:10B2600084B027D0174A03921A44029234BF0E4684
:10B27000CA1A04A934BFC3F180020026002341F892
:10B28000102D02A802220196FFF7ECFE2378184445
:10B29000C0B203062B7848BF80F080008342207044
:10B2A00002D0002004B070BD002301202B70237059
:10B2B00004B070BD012004B070BD00BF39AB0020E8
:10B2C000BCAB00203CAB002008B545F20820FFF7DE
:10B2D000B9FE0620FEF7EEFD064B0122C7201A70CC
:10B2E000FEF7E8FD04480549054A002303700B708A
:10B2F000136008BDBE960020BCAB002039AB002017
:10B30000448B00202DE9F04182B00346060C050A6B
:10B31000032406208DF80730884617468DF805600F
:10B320008DF806508DF80440FFF78CFEC0B100BFC9
:10B330000D4C23689868FEF729FC236801A958681A
:10B34000002228F03FFF23684246002158683B4610
:10B35000FCF7FAFF23689868FEF71EFC00BF38462A
:10B3600002B0BDE8F08100BFAC960020F0B5124BF2
:10B370009D6885B00DB905B0F0BDED0A14D0002769
:10B3800004AE7C196410E00210226946FFF7BAFF90
:10B390000F2809DD6B4653F8042B01320AD1B34262
:10B3A000F9D12546AF42ECDBFFF72CFF034BED0252
:10B3B0001D60E0E7671CF5E7040F0020448B0020C8
:10B3C0000C4B984213D0A3F5806398420FD003F53D
:10B3D000804398420BD003F58063984207D003F571
:10B3E0008063984203D0044B186840087047024BB2
:10B3F000186870470004014020AA0020F0B5774B80
:10B40000774A87B01968914200AF00F0DB800023D3
:10B41000744A3B607B60136843F48033136003E03D
:10B420003B68B3F5A04F09D0136803F400337B6089
:10B430003B6801333B607B68002BF1D0694B1B6894
:10B4400013F4003318BF01237B607B68012B7BD092
:10B45000654D644B654AEA606549586F654A086006
:10B46000AA605E6B644C654A654826F080065E63A0
:10B470005E6F46F080765E67196B0C431C63596BF8
:10B480005963996B9963196C41F05B5141F47B11DD
:10B4900041F41F6141F00F011964596C07F1180460
:10B4A0000A4348F2FF715A6444F8101D00262146F1
:10B4B0000123FB733E737E73BE7321F09DFF214613
:10B4C0004FF6FF734F48BB6021F096FF4FF6FF73B6
:10B4D00021464D48BB6021F08FFF21464B4821F0AB
:10B4E0008BFF21464A4821F087FF2146494821F039
:10B4F00083FF2146484821F07FFF2146474821F03D
:10B500007BFF2146464821F077FF20462EF06AFA5D
:10B51000444B454C1B68BA6844484549A4FB034367
:10B520009B09A0FB0202013B920CB3F1807F0A60F1
:10B5300007D2404AF0200721536085F82300966027
:10B5400011601C37BD46F0BD264B3B4D1A6C3B4885
:10B5500042F080521A642C684268816844F4404486
:10B560002C609C689C609C6844F400449C609C68CF
:10B5700044F4A0549C600068120642EA801242F42F
:10B580008002490842F00802013942EA01425A6049
:10B590001A6842F080721A601A689201FCD5284934
:10B5A000104A40F205700860996821F00301996023
:10B5B000996841F002019960936803F00C03082B2D
:10B5C000FAD145E700221A6062B61E4B1B6883F36E
:10B5D00008881D4B1B689847FEE700BFFCFF012051
:10B5E000EFBEADDE0038024000ED00E00005FA05D8
:10B5F0001C62002000000008FF916700335F070015
:10B60000000002400004024000080240000C02401A
:10B61000001002400014024000180240001C0240CA
:10B620000020024020AA0020D34D621083DE1B437D
:10B630001496002010E000E00070004000000020A0
:10B64000003C02400000FF1F0400FF1F08B5054B2F
:10B650001B6803B19847044B044A1A6072B6FDF7A1
:10B660006FF900BFE8740020FCFF0120EFBEADDEE3
:10B6700008B5034B1B6803B1984772B6FDF760F934
:10B68000E8740020084B10B507281B68C8BF1438A1
:10B6900018440C46007EFDF799FF20B12146BDE815
:10B6A0001040FEF77FBA10BD8496002030B50446E6
:10B6B000406D61718389A26823F400531B041B0C45
:10B6C000838185B0A379009213F0040230D04FF447
:10B6D000805213F00203ADF804205CD1ADF80630BF
:10B6E0004FF480630022ADF8083011F00103ADF88B
:10B6F0000C2028D1ADF80A3008238D07694648BFD1
:10B70000ADF80A302EF004FAA279636DD10724D483
:10B7100012F0080F9A8A1BD122F008021204120CB0
:10B720009A829A8992B242F400529A8105B030BD51
:10B7300013F00203ADF804202AD04FF4005513464D
:10B74000ADF80650CEE70423ADF80A300C23D4E759
:10B7500092B242F008029A82E3E710498B4215D078
:10B76000A1F548418B420FD001F580618B4209D091
:10B770000B498B42CCD105200121FFF783FFA27931
:10B78000636DC5E70320F7E70220F5E70020F3E744
:10B79000ADF80630A6E74FF400539FE700100140D4
:10B7A0000014014010B50446406DA160838923F464
:10B7B00000531B041B0C8381A37984B013F0040293
:10B7C000009135D04FF4805213F00203ADF80420FD
:10B7D0005CD1ADF806304FF480636279ADF8083083
:10B7E000D1074FF00003ADF80A30ADF80C3045BF7B
:10B7F0000423ADF80A3008230C236946920748BF9A
:10B80000ADF80A302EF084F9A279636DD1071FD408
:10B8100012F0080F9A8A16D122F008021204120CB4
:10B820009A829A8992B242F400529A8104B010BD71
:10B8300013F00203ADF8042025D04FF40051134655
:10B84000ADF80610C9E792B242F008029A82E8E722
:10B8500010498B4215D0A1F548418B420FD001F51C
:10B8600080618B4209D00C498B42D1D10520012146
:10B87000FFF708FFA279636DCAE70320F7E702200C
:10B88000F5E70020F3E7ADF80630A6E74FF40053E4
:10B890009FE700BF001001400014014038B50C4B79
:10B8A00007281B68CCBFA0F11404044623440546B6
:10B8B000187EFDF78BFE50B101342722C4718271CE
:10B8C00028F020FC28460021BDE83840DAE638BDE3
:10B8D0008496002070B50F4C0F4DC0EBC00004EBF8
:10B8E0008004286B26693043286382B09209667B06
:10B8F000A1600025012101A863618DF804608DF825
:10B9000005208DF806508DF807102EF0C9F802B00A
:10B9100070BD00BF440D002000380240074BC0EB53
:10B92000C00030B403EB8000054C0569236B2B434A
:10B9300023630176427630BC704700BF440D00207F
:10B94000003802402DE9F04F5B4C54F8204083B0A2
:10B95000002C00F0AC80E66D002E00F0AA8090462E
:10B96000564A35692260994604F2622204F1620364
:10B970006361A2614FF400737268A1600746E360DF
:10B9800023616265A246B5B14D4B00205A689542CD
:10B9900003F11C0376D001301028F7D100207A1C67
:10B9A000D2B20C21FFF7BAFF636DB168326922632E
:10B9B0000433A1632365F068E8B1414B00215A6864
:10B9C000904203F11C035BD001311029F7D100250F
:10B9D0007A1CD2B20B212846FFF7A0FF2346F27F44
:10B9E00038492846FFF776FF636DB168F2686263F5
:10B9F0000433E163E36494F86100FDF7E7FD054675
:10BA000094F86000FDF7E2FD8346307F00284BD1BB
:10BA100019F0080F38D118F0020F09D045B10B22E8
:10BA20007B1CAA71EB712846727F2221FDF794FEE0
:10BA300018F0010F15D1A36B7BB996F82020B17FC8
:10BA40008DF8063001A8930901228DF805308DF894
:10BA500004108DF807202EF023F8504603B0BDE8FF
:10BA6000F08FBBF1000FE6D001370C238BF8077085
:10BA70008BF806305846727F2221FDF76DFEDAE71B
:10BA8000CDB2A5E7C0B28AE70137FFB215B10B23EB
:10BA9000EF71AB7119F0100F284614BF022112216B
:10BAA000727FFDF759FEC6E728F00EFBB0E7A2460D
:10BAB000D3E7B246D1E700BF143D002008EF0308EA
:10BAC000440D0020658900080348D0F8AC3113B15B
:10BAD00000F5D27018477047440D00200348D0F895
:10BAE000903113B100F5C47018477047440D002021
:10BAF0000348D0F8743113B100F5B6701847704799
:10BB0000440D00200348D0F8583113B100F5A87057
:10BB100018477047440D00200348D0F83C3113B15A
:10BB200000F59A7018477047440D00200348D0F87C
:10BB3000203113B100F58C7018477047440D002078
:10BB40000348D0F804310BB1FC301847704700BFF0
:10BB5000440D00200348D0F8E8300BB1E03018471E
:10BB6000704700BF440D00200348D0F8CC300BB123
:10BB7000C4301847704700BF440D00200348D0F878
:10BB8000B0300BB1A8301847704700BF440D0020FB
:10BB90000348D0F894300BB18C301847704700BF81
:10BBA000440D00200248836F0BB170301847704776
:10BBB000440D00200248C36D0BB154301847704744
:10BBC000440D00200248036C0BB138301847704711
:10BBD000440D00200248436A0BB11C3018477047DF
:10BBE000440D00200248836803B11847704700BF26
:10BBF000440D0020431C00F014812DE9F04F4FEA62
:10BC0000C00808EB00039B00DFF8F4A25AF803B069
:10BC100087B00AEB0304BBF1000F00F0FF80143380
:10BC20000AEB03010022DBF804704AF803204A60A3
:10BC30008A60CA600346A56801900133D4F80C906D
:10BC4000DBB2002D00F0EE801522EB71AA71B9F184
:10BC5000000F00F00081162289F8062089F80730CD
:10BC60009BF80E0028F030FABB8823F440731B04C5
:10BC70001B0CBB802846FDF78FFF4846FDF78CFF65
:10BC800011212846FDF7ECFB11214846FDF7E8FBA2
:10BC90000826642404E00A203CB103F061F8013C6A
:10BCA0002846FDF7A1FF0028F5D02846FDF76EFFD6
:10BCB0000A2003F055F82846FDF76EFF0A2003F02E
:10BCC0004FF8013EECD14846FDF760FF0A2003F033
:10BCD00047F82846FDF75AFF0A2003F041F82846A6
:10BCE000FDF75AFF0A2003F03BF84846FDF754FFE2
:10BCF000019B08EB03040AEB84042846637C002BB9
:10BD00000CBF122132210422FDF726FD637C002B9B
:10BD10000CBF1221322148460422FDF71DFD704B55
:10BD20009F4200F0B7806F4B9F4200F0BD806E4B8A
:10BD30009F4200F0A580BB8801996C4A6C4C23F4AB
:10BD400040731B041B0CBB803B8888440AEB880AA9
:10BD50009BB243F001039AF810103B80BD8802A803
:10BD6000002918BF14462DF03DFE049A6148B2FB2D
:10BD7000F4F325F03F05A0FB02122D04900C2D0CCE
:10BD80000543BD805C4C39884FF4967202FB00F28B
:10BD900084FB02409BB2D217002BC2EBA01221F011
:10BDA000010108BF01230904013243F40043090CD7
:10BDB00092B239803A84BB833B889BB243F0010343
:10BDC0003B803B8823F4816323F002031B041B0C9C
:10BDD00043F480634FF480423B803A813B8823F0F8
:10BDE00080031B041B0C3B809BF810308DF808303F
:10BDF0000024012302A88DF80B308DF809408DF83E
:10BE00000A402DF04DFE9BF80F308DF8083002A847
:10BE10008DF809408DF80A402DF068FE07B0BDE8A6
:10BE2000F08F7047B9F1000F48D0162289F807301B
:10BE300089F806209BF80E0028F046F9BB8823F409
:10BE400040731B041B0C2846BB80FDF7A5FE48462B
:10BE5000FDF7A2FE18E79BF80E0028F035F9BB8825
:10BE600023F440731B041B0CBB802846FDF794FE93
:10BE70004846FDF791FE11212846FDF7F1FA07E744
:10BE80001E4A136A43F4000313624FF400002DF0BE
:10BE9000A1FD50E7194A136A43F4001313624FF4EB
:10BEA00000102DF097FD46E7144A136A43F480030F
:10BEB00013624FF480002DF08DFD3CE79BF80E00DF
:10BEC00028F002F9BB8823F440731B041B0C48467E
:10BED000BB80FDF761FE4846FDF75EFED8E600BF79
:10BEE0000054004000580040005C0040009F2400C7
:10BEF000804F120083DE1B43D34D62100038024096
:10BF00003C3D0020F8B54FEAC00E274F069C0EEBD3
:10BF1000000507EB85056E68002E42D04900C9B2C6
:10BF2000A9754FF0000C0121EA7585F819C0A976B2
:10BF30002B76697585F814C0B3882C629905EC617D
:10BF400014D43388DA050CD44FF4805401E0013C5A
:10BF50001ED033889B05FAD433889BB243F4807398
:10BF60003380B3889BB243F44073B3800EEB00017F
:10BF700007EB81024FF4805401E0013C08D0537D6F
:10BF8000002BFAD107EB81073C7D84F00100F8BD5E
:10BF9000064A138801339BB21380FFF72BFE20461D
:10BFA000F8BD3046F8BD00BF3C3D0020B83E002043
:10BFB00070B590F904506C1C82B00AD0032D08DCD7
:10BFC00016460A46417900962846FFF79BFF02B0C5
:10BFD00070BD002002B070BD00B50378012B83B0A6
:10BFE00004D1032301AA0021FFF7E2FF9DF80530E9
:10BFF0009DF804209DF806001B0243EA0243184303
:10C0000003B05DF804FB00BF08B5FFF7E5FF014B87
:10C01000586008BDD01F002008B5FFF7DDFF014BB9
:10C02000186008BDD01F0020F0B585B002AB0446F3
:10C030000093032206231E210120FFF763FF00283F
:10C040003CD09DF808509DF809109DF80A709DF8A5
:10C050000B209DF80C609DF80D3041EA052142EA65
:10C06000072243EA062309B212B21BB2144D06EEB0
:10C07000901A07EE102A07EE903AF8EEE66A95ED70
:10C08000035AD5ED055A95ED046AB8EEC77AF8EE75
:10C09000E77A66EE856A27EE257A67EE867AFDEE08
:10C0A000E66ABDEEC77AFDEEE77A16EE901A17EE55
:10C0B000102A17EE903A2180A280638005B0F0BD6F
:10C0C0000000002000B583B0012000920A466821DC
:10C0D000FFF718FF03B05DF804FB00BFF0B5C60022
:10C0E00033189B00254DEA585468A28A83B092B257
:10C0F0000192019A2B4412F4706F1CBF01221A7531
:10C10000019B13F4E06F07460CD1A38A3E4423F44D
:10C11000706305EB86051B041B0C0022A3826A7565
:10C1200003B0F0BD238BA38823F480631B041B0C96
:10C13000A380019B9B05E8D423889805E5D4238838
:10C14000D9050ED52388DA05FCD423889BB243F4A5
:10C150000073238023889B05FCD43846FFF74AFDF3
:10C16000D3E723889BB243F400732380A38823F48E
:10C1700040731B041B0CA380C7E700BF3C3D00209D
:10C18000F0B583B0441C8DF8073001D0032802DDE0
:10C19000002003B0F0BDC700244E3B1806EB83031C
:10C1A0005D68002DF4D04900C9B2997501240021C1
:10C1B000DA755C7699761C765C751975A9880DF12F
:10C1C00007028905DA611A6214D42B88DA050CD4C7
:10C1D0004FF4805401E0013C1ED02B889B05FAD41B
:10C1E0002B889BB243F480732B80AB889BB243F4C3
:10C1F0004073AB80074406EB87024FF4805401E0A4
:10C20000013C09D0537D002BFAD106EB87073C7D1A
:10C2100084F0010003B0F0BD054A138801339BB2DE
:10C220001380FFF7E7FC2046B3E700BF3C3D00204A
:10C23000B83E00202DE9F043322083B002F0EAFD41
:10C24000112300221E210120FFF79AFF0122104630
:10C2500060231E21FFF794FF642002F0DBFD684697
:10C26000FFF7E2FE0024DFF85481254626460A2720
:10C270000123184602221E21FFF782FF322002F01E
:10C28000C9FD6846FFF7D0FEBDF902E0BDF9041014
:10C29000BDF900208E457346A8BF0B469342A8BF48
:10C2A000134643454FF0010075440C44164479DBB6
:10C2B000FCF7FAFF013FDBD14FF001091223002206
:10C2C0001E210120FFF75CFFDFF8F0800A27012321
:10C2D000184602221E21FFF753FF322002F09AFD7A
:10C2E0006846FFF7A1FEBDF902E0BDF90410BDF9F3
:10C2F00000208E457346A8BF0B469342A8BF134645
:10C3000043454FF00100A5EB0E05A4EB0104A6EB9D
:10C3100002064ADBFCF7C8FF013FD8D107EE906A5E
:10C32000F8EEE76A07EE905AB8EEE77A07EE904A21
:10C33000DFED1F5A9FED1F5A1F4EF8EEE77A85EE8C
:10C34000A66A702300221E210120C5EE876A85EEB1
:10C35000277AB0EEC66AF0EEE66AF0EEC77A86EDAE
:10C36000036AC6ED046AC6ED057AFFF709FF0122EC
:10C37000104620231E21FFF703FF002302221E2167
:10C380000120FFF7FDFE642002F044FDB9F1000F2B
:10C3900004D14FF07E53F36033617361012003B029
:10C3A000BDE8F0834FF0000988E74FF00009B5E7DA
:10C3B00000406F4601C05E460000002001F0FFFF14
:10C3C0000378012B00D07047417990F9040058227E
:10C3D000D6E600BF0378012B00D07047417990F971
:10C3E00004004822CCE600BF134601200A4668211B
:10C3F000C6E600BF0220FCF791BB00BF02206DE63D
:10C400000120FCF78BBB00BF012067E60020FCF792
:10C4100085BB00BF002061E61549164B16480A6827
:10C4200010B48C681549B2FBF4F203FB02F303600D
:10C43000D1F88820124B134C42F47002C1F88820C6
:10C440001A68002042F001021A6098601A6822F00F
:10C45000847222F480321A605C601A684FF00064C3
:10C4600022F480221A60D8608C605DF8044B70471B
:10C470000000002040420F0020AA002000ED00E054
:10C480000038024010300024044B4FF4F0700A21B1
:10C49000022283E80700FFF7BFBF00BF00000020B3
:10C4A00038B50B4C23688BB15A68821A002A0546AE
:10C4B00004DA0CE05A68AA1A002A07DB9A6822609C
:10C4C00018461A6890472368002BF3D138BD38BD51
:10C4D000647400200B4B002210B4027203F59074B8
:10C4E000032102E0072A09DC9979890702D5197925
:10C4F000815401329C4203F11803F3D15DF8044BDF
:10C50000704700BFE41D04082E230370704700BF6E
:10C51000012332213122417042710370037170474F
:10C520002322032302704370704700BF2DE9F041BE
:10C530000B78047BDB43DEB200F1100200F138031C
:10C5400042F8044F9342FBD1DFF89CC000F1600138
:10C55000002243F8042F8B42FBD14FF0140E05212B
:10C56000002546FA01F303F00103002B1D4414BF1C
:10C570004FF019084FF00A0811F0010FEDB214BF87
:10C580002746002700220EEB02039BB200EB830339
:10C59000013242455F61F6D1013A92B2013201396E
:10C5A0000EEB02034A1C9BB201D09E46D9E715F060
:10C5B000010F14BF19250A2500215A1892B200EB69
:10C5C00082020131A9425461F7D10B449BB21A1D7A
:10C5D00000EB8202013300219BB25160ACF80030C5
:10C5E0000361BDE8F08100BFE41F0020254B5B889C
:10C5F0000B332DE9F04F8A4601F1060B1FFA83F940
:10C600004FF00108002100271AF801EB3E464C4686
:10C610000122A4F10B039BB207E001339BB2B0F8F7
:10C620000CC0C5F814C09C420AD000EB8305002A58
:10C63000F3D100EB830501339BB29C426A61F4D1D4
:10C64000231D00EB83030136092FF6B259600CD08D
:10C65000092E14D008FA07F313EA0E0F14BF0122B3
:10C6600000220C34A4B20137D3E709F17809DA4586
:10C670001FFA89F9C7D1034B5980BDE8F08F00221A
:10C68000EFE700BFE41F00202DE9F047DFF85C80F2
:10C69000B8F8043004338A461FFA83FC01F1090913
:10C6A0004FF0010E1AF8017B64460026231F0EFA94
:10C6B00006F29BB23A40BAB1818900EB830501339F
:10C6C0009BB29C426961F6D101360434082EA4B2B3
:10C6D000ECD10CF1200CCA451FFA8CFCE2D10023EE
:10C6E000A8F80430BDE8F0871146E6E7E41F002013
:10C6F00010B4037B01681F2B09D9203B20224C6812
:10C7000002FA03F31C4214D15DF8044B7047202257
:10C710000C6802FA03F31C42F6D00C4A406800246D
:10C72000147002685DF8044B22F0010202608B6015
:10C730007047064A40680024147002685DF8044B94
:10C7400022F001020260CB60704700BFA49D002070
:10C7500008B515F0D3FBFEF78BFF00BF024A034B71
:10C760001278197824F0D0BEC0220020C122002007
:10C77000038A2DE9F0478589ADB21D4029D00F46C7
:10C7800006464FF000484FF00009B5FA85F328FA45
:10C7900003F2D24391B21B3B15403182042B16D8D1
:10C7A000DFE803F03129211903007B6A002B32D026
:10C7B00003F1FF3A1FFA8AFAC7F824903C6A34B1B1
:10C7C00023682046514698476468002CF8D1002D14
:10C7D000DBD1BDE8F0873868716B036889B2984790
:10C7E000002DD2D1F5E77868B16B036889B298471C
:10C7F000002DCAD1EDE7B868F16B036889B298479C
:10C80000002DC2D1E5E7F868316C036889B298471A
:10C81000002DBAD1DDE7F36A1FFA83FACEE700BF35
:10C820002DE9F04F2DED028BA0F10A0389B00C46E3
:10C83000E72B00F23787DFE813F01C0135073507D7
:10C840003507350735073507350735073507350708
:10C8500035073507350735073507350735073507F8
:10C8600035073507350735073507800135073507A3
:10C870003507710135073507350764013507810232
:10C8800035076902350739023507310235070C02D1
:10C890003507E001350735073507DA01D3013507DC
:10C8A000C70535073507BF05350796053507350731
:10C8B000350779053507350735073507F60235079A
:10C8C000FC003507F305CF05350735073507350774
:10C8D000350735073507DD06350795063507600648
:10C8E00035070B06350720073507350735073507A8
:10C8F0002805ED04E604C502E800AB049704CF0464
:10C900008B043507540438043507350735073507D8
:10C910002D04350735070C04350735073507FE03A9
:10C92000E703AC036A033507350735075B034403A8
:10C93000350315033507350735073507350735073F
:10C940003507350735073507350735073507350707
:10C950003507280535073507350735073507350706
:10C9600035073507350735073507350735072D01F5
:10C9700035073507350735073507350735073507D7
:10C9800035073507350735073507350735073507C7
:10C9900035073507350735073507350735073507B7
:10C9A00035073507350735073507350735073507A7
:10C9B0003507350735073507350735073507350797
:10C9C0003507350735073507350735073507350787
:10C9D0003507350735073507350735073507350777
:10C9E0003507350735073507350735073507350767
:10C9F0003507350735073507350735073507350757
:10CA00003507350735079E01A901AE4E337853B17E
:10CA1000AD4F002537F8021F2046FDF759FF337848
:10CA20000135AB42F6DC012009B0BDEC028BBDE85C
:10CA3000F08FA44E3378002BF5D0A44F0025B846D4
:10CA4000236817F81520591C21601A7098F80110F6
:10CA500001EB810101EB810101F2EE2189B2204657
:10CA6000FDF736FF33780135AB4208F10208E7DC09
:10CA7000D9E7974D28462FF04FF90028D3DD2B46F4
:10CA80000544226813F8011B501C9D422060117060
:10CA9000F7D1C8E70B68DFF870C2591C9CF800207A
:10CAA00021601A709CF80030002BBCD0894E8A4D52
:10CAB0008A488B490023226816F8017F02F1010E93
:10CAC000C4F800E01770226815F8017F02F1010E2A
:10CAD000C4F800E01770226810F8017F02F1010E1F
:10CAE000C4F800E01770226811F8017F02F1010E0E
:10CAF000C4F800E017709CF8002001339A42DADC99
:10CB000091E70B68774A581C1178206019702368E8
:10CB10005278591C216001201A7085E7724D084631
:10CB20002988FDF7D5FEA9882046FDF7D1FE2046CD
:10CB30002989FDF7CDFE012076E76C4D05F1500601
:10CB400028782EF05BFA2368027A591C21601A704B
:10CB500023686A78591C21601A702368AA78591CC6
:10CB600021601A702368EA780435591CAE422160AE
:10CB70001A70E5D157E75E4D0846E989FDF7A8FE32
:10CB80002046A989FDF7A4FE01204DE7594B03F18A
:10CB9000700522681978501C20601170226859783D
:10CBA000501C2060117022689978501C2060117010
:10CBB0002268D978501C2060117022681979501CA5
:10CBC0002060117022685979501C20601170226811
:10CBD00099790733501C9D4220601170D9D122E70A
:10CBE0000B6801229918216010461A701CE708464C
:10CBF0000021FDF755FE012016E73F4D05F13807EE
:10CC000003E00835AF423FF40EAF95F902603046BD
:10CC10000DF046FD0028F4D023685A1C22601E70D7
:10CC200029882046FDF754FE2368EA78591C2160C4
:10CC30001A7023682A79591C21601A702368AA790E
:10CC4000591C21601A7023686A79591C21601A7076
:10CC5000D7E72A4B03F15A0522685979501C206006
:10CC6000117022681978501C206011702268597860
:10CC7000501C2060117022689978501C206011703F
:10CC80002268D978501C2060117022681979063307
:10CC9000501C9D4220601170DED1C4E60B68184A1A
:10CCA000591C527D216001201A70BDE6154D05F119
:10CCB000800655F8041F2046FDF7F2FDAE42F8D17C
:10CCC000B1E600BF10790020BE5B002088AD0020D7
:10CCD00064420020174500202745002047450020DA
:10CCE00037450020488B0020B43D00204C8B0020AD
:10CCF00094780020DCAE002014A9002064400020BD
:10CD0000F0610020046B002015450020AB4D05F1BB
:10CD10004006B5F880102046FDF7DAFD236895F847
:10CD20008220591C21601A70236895F883200435ED
:10CD3000591CB54221601A70EBD174E6A04D0B6806
:10CD40002A7A591C21601A70A98B2046FDF7C0FD74
:10CD5000298B2046FDF7BCFD698B2046FDF7B8FD09
:10CD60002368EA7C591C21601A70A98C2046FDF7C3
:10CD7000AFFDE98C2046FDF7ABFD2368AA7F591C67
:10CD800021601A70236895F82020591C21601A70C0
:10CD9000698C2046FDF79CFD2368EA7A591C2160C6
:10CDA0001A70E9682046FDF77BFD23682A7C591C30
:10CDB00021601A70236895F82120591C21600120F8
:10CDC0001A7031E67F4D804E9FED808ADFF8308209
:10CDD000DFED7F8A05F120070EE0FCEEE77ACDED6E
:10CDE000017ABDF8041020460435FDF771FDBD42FF
:10CDF00006F118063FF417AE717C0029F3D0754B8D
:10CE0000D5ED007A1B78012BE7D1734B1B68DB044F
:10CE100040F1EB84F5EE407AF1EE10FA40F0158522
:10CE200040F2DC51DFE70B686C4D591C2A79216018
:10CE30001A7023686A79591C21601A702988204663
:10CE4000FDF746FD2368AA79591C21601A7069888C
:10CE50002046FDF73DFD2368EA79591C2160012039
:10CE60001A70E1E50B685E4F591C3A7821601A7020
:10CE70003B78002B3FF4D7AD0025EEB2304620F0D2
:10CE8000D3FE23684278591C216030461A7020F086
:10CE9000CBFE01892046FDF71BFD3B780135AB42F7
:10CEA000EBDCC0E54F4B5049B3F9003081FB032167
:10CEB000DB17C3EBA101204689B2FDF709FD012074
:10CEC000B2E50A68494B501C19782060117022683D
:10CED0005978501C2060117022689978501C20608D
:10CEE00011702268DB78511C2160012013709BE5D2
:10CEF0003F4D0846298AFDF7EBFC698A2046FDF77D
:10CF0000E7FC2046A98AFDF7E3FC01208CE5DFF869
:10CF1000F4E00027FEB2714600232268501C206016
:10CF200016702268501C20601370226811F8010FDF
:10CF30000133551C062B25601070EED10137062FEA
:10CF40000EF1060EE6D12B4900232268501C20600A
:10CF500017702268501C20601370226811F8010FAE
:10CF60000133551C0B2B25601070EED12368134A3A
:10CF7000581C07212060197023680021581C20606C
:10CF80001970236892F8F020591C216001201A7052
:10CF90004AE50B68184A19491078124A5D1C256049
:10CFA000187023688978581C20601970236892785B
:10CFB000591C216001201A7036E500BF086B002063
:10CFC000F061002064890020645C00200000404281
:10CFD00000E08244485D0020786000205C42002030
:10CFE000E56E0020B88B002067666666FC44002072
:10CFF000245D0020EB6B002054600020947800201A
:10D00000DB9B9141C76B00200A68B14BB14918788E
:10D01000551C2560107022685878551C25601070CA
:10D0200022689B78501C206013702046C988FDF749
:10D030004FFC0120F8E4A74D08462988FDF748FC7D
:10D0400069882046FDF744FCA9882046FDF740FC8E
:10D05000E9E4A14D05F16006A9882046FDF738FCFA
:10D06000E9882046FDF734FC29892046FDF730FC8D
:10D070002368AA7A591C21601A702368EA7A591C1D
:10D0800021601A7055F80C1B2046FDF709FCAE42D2
:10D09000E2D1C8E4914952232268501C20601370E9
:10D0A00011F8013F002BF7D1BDE48D480023226821
:10D0B000056803EB4301561C6D5C26601570026821
:10D0C00025680A446E1C527826602A70026825681A
:10D0D0000A4401339278691C0A2B21602A70E6D138
:10D0E000A1E4804D0B682A68591C127821601A70DF
:10D0F0002B6822689978531C2360002311702A68DA
:10D1000021681A4401335279481C032B20600A70AD
:10D11000F5D123682A68591C127A21601A70236895
:10D120002A68591CD27821601A7023682A68591C11
:10D13000127921601A702B6820465989FDF7C8FBC7
:10D140002A682368527A591C21601A702A68DEE422
:10D15000654B08461968FDF7A3FB644B2046198808
:10D16000FDF7B6FB01205FE4614B08461988FDF727
:10D17000AFFB604B20461988FDF7AAFB5E4B226887
:10D180001B78511C03F001032160012013704BE454
:10D190005A4B0A681B785A4D511C03F00203216058
:10D1A000137023682A7D591C21601A702968204653
:10D1B000FDF776FB69682046FDF772FB298920465A
:10D1C000FDF786FBE9892046FDF782FB2046298A88
:10D1D000FDF77EFB012027E44A4D08462988FDF72C
:10D1E00077FB69882046FDF773FBB5F90430464AA2
:10D1F000D91782FB0323C1EBA301204689B2FDF7B7
:10D2000067FB012010E4084610224049FDF718FB97
:10D21000012009E43E4B9B8AB3F5006F00F2FA82CD
:10D22000B3F5806F00F20F83B3F5007F34BF0127A1
:10D230000227384D05F10C0655F8041B91FBF7F158
:10D24000204689B2FDF744FBAE42F5D1324D334F53
:10D2500005F10C06B5EC010AD7ED087A80EE270A35
:10D260002FF072FC81B22046FDF732FBB542F1D1BE
:10D270002B4D05F10C0655F8041B204689B2FDF72D
:10D2800027FBB542F7D1FFF7CEBB00258146DFF87B
:10D290009480DFF894B005950495069507950121D3
:10D2A0004FF6FF7A05E001350B2D00F0FE8118F9ED
:10D2B000011F4F1C4AFA05F3F5D0DE07F3D5BBF882
:10D2C00000302B41D807EED506A8FDF747FEEAE768
:10D2D00000430020404200200CB5002030EF03083E
:10D2E000E8780020CC420020F4710020E871002092
:10D2F0002C4400202E440020E04300202472002013
:10D3000028720020F8710020676666665489002044
:10D31000A0710020D87100206C600020688C002073
:10D32000C478002060EF03083A6C0020FDF75CFE33
:10D330002368A44D002803F101010CBF022203223F
:10D3400021601A7029882046FDF7AAFAA9682046AC
:10D35000FDF7A6FAFDF720FE01462046FDF7A0FAEC
:10D360000120FFF761BB0B68974A984D1178984AE6
:10D37000581C2060197011682046FDF791FA236847
:10D38000944A591C127A21601A7029882046FDF7A8
:10D390009FFAA9882046FDF79BFA29892046FDF7C8
:10D3A00097FA00212046FDF793FA20460021FDF769
:10D3B0008FFA0120FFF738BB084608228549FDF7A0
:10D3C0003FFA0120FFF730BB0B68834A581C917865
:10D3D00020601970FFF79BBB0B68804E01255A1C1B
:10D3E0000A601D700B68B278591921601A7025F017
:10D3F000D7FE23687A4A7B495F1927601870B1F914
:10D400000010B2F90000FDF7EDFB23685A19226005
:10D41000187031882046FDF75BFA2846FFF704BBF9
:10D420000B6800255A1C0A601D700B685A1C0A60A4
:10D430001D700B685A1C0A60204629461D70FDF7B6
:10D440002FFA20462946FDF72BFA0120FFF7ECBA08
:10D4500000212046FDF73CFA00212046FDF738FA6E
:10D4600000212046FDF734FA23685F4D00265A1C40
:10D4700022601E7023682A68591C92F82C202160B3
:10D480001A7023682A68591C92F8362021601A7095
:10D4900023682A68591C92F8372021601A70236883
:10D4A0005A1C22601E7023685A1C22601E7023685A
:10D4B0005A1C22601E702B682046598FFDF708FA0F
:10D4C0002B682046198FFDF703FA23682A68591C38
:10D4D00092F82E2021601A7023685A1C22601E7058
:10D4E0002B682046598EFDF7F3F92B682046998E5C
:10D4F000FDF7EEF90120FFF797BA3C4E0B68727901
:10D50000394D591C21601A702B682046198CFDF783
:10D51000DFF92B682046D98BFDF7DAF971892046AF
:10D52000FDF7D6F9B1892046FDF7D2F92B682046E0
:10D53000598CFDF7CDF92B682046998CFDF7C8F979
:10D54000F1892046FDF7C4F9318A2046FDF7C0F97C
:10D550002A68236892F82620591C216001201A703D
:10D56000FFF762BA214EF378002B00F047810B6879
:10D570000822591C21601A70236801229918216021
:10D580001A7023681A4D591C2A7921601A70236871
:10D59000AA78591C21601A7029882046FDF798F94D
:10D5A000E9892046FDF794F92368F279591C216036
:10D5B0001A702368EA78591C216001201A70FFF75D
:10D5C00033BA00BF040F0020488B0020B43D002078
:10D5D0000C7B0020F0610020F0420020F27A002055
:10D5E000BE890020C0890020E87800205460002017
:10D5F000245D002023F06CFFFF28064600F00C811C
:10D6000008A9002501F8125D0DF10D008DF80D50EF
:10D6100023F03EFF08A800F8115D23F02DFF08A8B5
:10D6200000F8105D23F01CFF08A820F8085D23F027
:10D630000BFF23685A1C22601E7023689DF80D2082
:10D64000591C21601A7023689DF80E20591C216016
:10D650001A7023689DF80F20591C21601A702368E6
:10D660009DF81020591C21601A702046BDF8181032
:10D67000FDF72EF90120FFF7D7B90B68924A9349BD
:10D68000D078934A5D1C2560187023684979581C2E
:10D69000206019702368D278591C216001201A700B
:10D6A000FFF7C2B90020FFF7BFB9DFF84CA2002591
:10D6B0004FF008080135C5F1200208FA02F2A5F181
:10D6C00020032AFA05F6164328FA03F31E43252DF4
:10D6D00006F001024FF000030BD01343EAD0E8B28A
:10D6E00016F0ECF90028E5D0294606A8FDF736FC2F
:10D6F000E0E7784B1B78DA0700F195800025764E3D
:10D700002F4602E00135252D0DD029463046FDF784
:10D7100035FC0028F6D0294606A8FDF72FFC002886
:10D720005ED10137EEE76D4B6D4DB3F850102046DA
:10D73000FDF7CEF86B4B1988204689B2FDF7C8F883
:10D74000694B19684B0103F02002C1F340031343F6
:10D75000C1F3800243EA4203C1F3C00243EA8203F9
:10D76000C1F3401243EAC20301F0100119432046FD
:10D77000FDF7AEF804A904222046FDF761F82368FE
:10D7800029785A4A581C2060197011886429A8BF4A
:10D7900064212046FDF79CF8B9F1960F48D000218E
:10D7A0002046FDF795F82168B7F1190348BFA7F1A6
:10D7B0001203A3F3C4034A1C226020461A460B70CE
:10D7C00005A9FDF73DF82368494A581C102120603F
:10D7D000197020461188FDF763F80120FFF724B97E
:10D7E000394604A8FDF7BAFB9BE7F4EEC87AF1EEE0
:10D7F00010FA47DA4FF47A71FFF7F5BA0B68B1788F
:10D800003C4A581C2060197023681278591C21600A
:10D810001A70B6E608270CE523685A1C226001201E
:10D820001E70FFF701B9069B43F00103069365E7FD
:10D8300023680322591C21601A7023686A78591CD6
:10D8400021601A70AFE70427F3E4F4EEC87AF1EE32
:10D8500010FA3FF5E5AAF4EEE87AFDEEE77AF1EE8C
:10D8600010FA17EE901A20D86FF4F973303903FBD1
:10D8700001F140F2E73391FBF3F101F2DB5189B2A0
:10D88000FFF7B1BAFDEEE77A40F2E73217EE903AD1
:10D89000303B02FB03F388FB0312D917C1EB622173
:10D8A00001F2E93189B2FFF79EBA40F2F313A1F514
:10D8B000836103FB01F140F2E73391FBF3F101F2E5
:10D8C000DD5189B2FFF78FBA94780020A86E00204E
:10D8D000B88B0020F1B50020E8B60020FC01002044
:10D8E000D9780020B83E002020720020BC3E0020E5
:10D8F000686C002024B4002090E33FF41C4C08B571
:10D9000001210220FCF756F9237803F00502052ACD
:10D9100029D003F00903092B08D000210120FCF7CE
:10D9200049F900210846FCF745F9FEE7114A124B78
:10D9300011681A680B68114C23F001030B601388FF
:10D94000206823F001031B041B0C138018B129224B
:10D9500000238271C37109224A21FBF7FDFE206872
:10D96000FCF714F9D9E714F05BFB2378D1E700BF8B
:10D97000103D00208C25002090250020A0250020AF
:10D98000022828BF022010B4084C094B207000EB7D
:10D990008002C0EBC20207495DF8044B013003EB83
:10D9A0004203C0B20B602DF0ABBC00BFD9780020A1
:10D9B000D6790020E878002008B522F089FEFCF72F
:10D9C00023FDBDE8084022F06BBE00BF38B5484BD0
:10D9D0005A899989914224BF00225A81198ADA8989
:10D9E000914224BF0022DA81DA78CAB1072A41497C
:10D9F0006AD091F85700404D012400210A282C706C
:10DA00009C70D9715DD00C2807D0002A6CD0DFED56
:10DA10003B7A072A0ED00A2862D0DFED397A09E076
:10DA2000344A92F857000A2856D00C285BD1D9798D
:10DA3000DFED347A344C9FED350AA278002918BF07
:10DA4000F0EE407A062A04D8314901EB820191EDCB
:10DA50000F0A217979B1013A032A0BD8F7EE007A3F
:10DA600087EE800A2FF070F82388984228BF184666
:10DA7000208038BD38BD9B781F4A07EE103A1178D8
:10DA8000B8EEC77A67EE277A07EE101AB8EEC77AB3
:10DA900027EE277AB4EEC70AF1EE10FAEADD80EE3F
:10DAA000277AFDEEC77A17EE903A102BA8BF102305
:10DAB000012BB8BF0123DBB28B4238BF0B4613707A
:10DAC00038BDDFED147AA4E791F857000A2803D097
:10DAD0000C28ACD0D9799AE7D979DFED0E7AA9E78D
:10DAE000DFED0D7AA6E7D979DFED047AA2E700BF72
:10DAF00054600020688C002024B400206F12033989
:10DB00006F12833A0AD7A339245D00206F120338BD
:10DB100030EF03085304E9380F506E3A38B50C4C17
:10DB20000C4DAC4206D2616820461434FCF7F8FB79
:10DB3000AC42F8D3084A094B094C14600022094949
:10DB40001A705A7008480860BDE8384019F0FABEEB
:10DB50008801000824060008E8780020D978002011
:10DB6000D6790020CC420020EC78002008B5FFF7E1
:10DB7000D5FF22F0ADFDFCF747FCBDE8084022F0E0
:10DB80008FBD00BFF0B50C2934D8DFE801F0893330
:10DB900033335E333333343333330700048C9689A5
:10DBA000B2F802E01788734D24F480542404240C46
:10DBB0000484038C8488818B23F4005321F4E64190
:10DBC0001B0409041B0C46EA0E06090C43EA063343
:10DBD00041EA0721A8429BB2A4B289B200F09E801C
:10DBE00005F58065A84200F0998092688480818361
:10DBF00002640384F0BD048C9589B2F802C0B2F8C7
:10DC000000E05C4F24F480742404240C0484038C0E
:10DC10008688818B23F400731B0421F073011B0C95
:10DC200045EA0C04090443EA0423090CB8429BB2F8
:10DC3000B6B241EA0E015CD04F4CA04259D0926876
:10DC400086808183C2630384F0BD048C9589B2F819
:10DC500002C0B2F800E0474E24F010042404240C63
:10DC60000484038C8788018B23F0200321F4E64190
:10DC70001B0409041B0C45EA0C04090C43EA0413B9
:10DC800041EA0E21B0429BB2BFB289B25DD03A4C9C
:10DC9000A0425AD092688780018382630384F0BDDA
:10DCA000048C9789B2F802E01688324D24F0010402
:10DCB0002404240C0484038C8488018B23F0020345
:10DCC0001B0421F073011B0C47EA0E0709043B43B8
:10DCD000090CA8429BB2A4B241EA060125D005F581
:10DCE0008065A84221D092688480018342630384C6
:10DCF000F0BDD589148A578A23F4006343EA0525C9
:10DD00004FF6FF332B40958826F440563C4343EAB8
:10DD1000052346EA04169BB2B6B290E7158A24F4AE
:10DD2000804444EA8514A4B25FE7D689158A578AED
:10DD300023F00803334324F4407496883D4323F0D2
:10DD400004032C433343A4B2CDE7D489158A568A01
:10DD500023F0800343EA04134FF6BF741C409388FA
:10DD600027F44067354344EA031347EA85079BB22B
:10DD7000BFB28FE700000140000401402DE9F84FD9
:10DD8000F02200219148924CDFF86892914D924E1A
:10DD9000924FDFF8648230F0E4FF91489149DFF858
:10DDA0005CE2DFF85CC200221359834200F0EA8093
:10DDB000B3F1804F00F0E880AB4200F0F380B34253
:10DDC00000F0F280BB4200F0F180734500F0F0807B
:10DDD000634500F0EF80434500F0EE80DFF824A2B9
:10DDE000534500F0EB800AF5806A534500F0E88067
:10DDF0000AF5806A534500F0E580AAF5983A534544
:10DE000000F0E2800AF5806A534500F097800AF539
:10DE1000806A534508BF0D2300F091801832B2F597
:10DE20009C7FC1D16A4EDFF8E0A106F59C774FF0E8
:10DE300003094FF0020803E01836B74200F0A08053
:10DE4000B379002BF8D033791C09013C032C03F083
:10DE50000F03F1D8644A32F8140040FA03F2D207F3
:10DE6000EAD5012505FA03F3013B18402EF0FEFB2D
:10DE70005E4B1B5D18441AEBC002DDD05AF83030FF
:10DE80005B4C317A03F13F4000F57E00800A205C54
:10DE900000F01F044009032805FA04F57CD004288B
:10DEA00074D0022804D14F48406C05434D48456466
:10DEB000B2F804E0BEFA8EF2C2F11F0292B2D008AC
:10DEC00003EB800002F00702046A92000F259540E0
:10DED00024EA05040462046A01FA02F222430025DE
:10DEE00002624FF0010C2A4603E0102A05F10205F8
:10DEF000A2D00CFA02F030EA0E0102F10102F4D1D4
:10DF00001C6809FA05F1C9430C401C60D3F800B045
:10DF100008FA05F444EA0B041C609C680C409C6001
:10DF20009C689C605C6824EA0000586058685860EF
:10DF3000D8680140D960D968D960D6E70C2309EBCD
:10DF4000C3034FF0010A93F85C3003F01F0B5B0929
:10DF5000032B0AFA0BFA09D0042B0CD0022B7FF406
:10DF60005DAF4B6C4AEA03034B6457E70B6C4AEA1C
:10DF700003030B6452E70B6B4AEA03030B634DE7A1
:10DF8000BDE8F88F0023DAE70123D8E71548006BD6
:10DF90000543144805638BE71248006C054311489C
:10DFA000056485E70223CAE70323C8E70423C6E71D
:10DFB0000523C4E70623C2E70723C0E70823BEE71B
:10DFC0000923BCE70A23BAE70B23B8E7C096002071
:10DFD000E41D04080004004000080040000C00405C
:10DFE0000000014000380240DC1D0408D81D040870
:10DFF000B01D040830EF0308000401400010004089
:10E0000000140040004001405094002001490248A3
:10E01000FEF7AEBB88970020001800400149024877
:10E02000FEF7A6BB609700200004014001490248AA
:10E03000FEF79EBB609700200004014001490248A2
:10E04000FEF796BB38970020000C004001490248BB
:10E05000FEF78EBB109700200004004002494FF0ED
:10E060008040FEF785BB00BFE896002001490248CA
:10E07000FEF77EBBC0960020000001400149024827
:10E08000FEF776BBC096002000000140F0B50468A2
:10E090004B4DA30AAB4276D009D94A4DAB425CD076
:10E0A0000135AB4273D03B3DAB425AD0F0BDB3F526
:10E0B000801F64D0023DAB4257D14FF0700E022654
:10E0C0004779B0004FEA970C002964D063460227D5
:10E0D000A5899F4083190CEB43032F4303F1040CE4
:10E0E000394DBFB245F8231045F82C20A781EFF336
:10E0F0001181502282F31288821905EBC202136942
:10E10000002B33D013620433821905EBC202576926
:10E1100017B11F6053690433821905EBC202976976
:10E1200017B11F6093690433821905EBC202D769E6
:10E1300017B11F60D36904330027CAB21F6082F38E
:10E140001188304405EBC000036A93B9A38923F01A
:10E1500001031B041B0CA381F0BD4FF0200E002611
:10E16000AEE74FF0E80E0526AAE7F0BD05EB0E037B
:10E17000CAE7A3899BB243F00103A381F0BD4FF02E
:10E18000480E01269CE74FF0980E032698E74FF0C3
:10E19000C00E042694E70223BF0803FA07F7A389F9
:10E1A000094D9BB223EA070387190CEB470CA381A7
:10E1B0000CF1040345F82C1045F8232097E700BF25
:10E1C0000300100040001000C096002010B5036846
:10E1D00083480139834282B089B200F0CB80A0F538
:10E1E0008060834200F0C68000F58040834200F0EA
:10E1F000B88000F58060834200F0B38000F5806055
:10E20000834200F0AE80774C188824686408B4FB21
:10E21000F2F4013CA4B282B2B3F1804F0AD072484A
:10E22000834207D000F58060834203D000F5806010
:10E23000834202D122F0700292B26C48834200F015
:10E24000A28000F58060834200F0A78022F4407233
:10E2500000F56C4092B283421A80D9621C854FD07F
:10E260005F4A93424CD001229A821A8892B242F0BD
:10E2700001021A80B3F1804F00F099805A4A93420C
:10E2800000F0978002F58062934200F0948002F5DE
:10E290008062934200F0918002F58062934200F028
:10E2A0008E8002F58062934200F08B8002F570420E
:10E2B000934200F0888002F57052934200F085800E
:10E2C00002F58062934200F0828002F58062934200
:10E2D0007FD0A2F5983293427DD002F580629342BE
:10E2E0007BD002F58062934208BF0D2215D002A8B0
:10E2F0004FF0012340F8043D2BF0D2FB02B010BDDB
:10E300000122002119869A821A88394892B242F075
:10E31000010283421A80ADD10A46364B03EBC20399
:10E3200001A893F85D408DF80440012300228DF888
:10E3300005308DF807308DF806202BF0B1FB1B2C33
:10E3400008D02E2CDAD12C4B019301A82BF0A8FB7E
:10E3500002B010BD294B019301A82BF0A1FB02B024
:10E3600010BD204C18882468B4FBF2F4013CA4B220
:10E3700082B251E71B4C18882468B4FBF2F4013CCC
:10E38000A4B282B256E701201A80D9621C85988215
:10E390001A8892B202431A8070E701201A80D9626B
:10E3A0001C8598821A8892B202431A8062E7012281
:10E3B000B3E70222B1E70322AFE70422ADE705226B
:10E3C000ABE70622A9E70722A7E70822A5E709226B
:10E3D000A3E70A22A1E70B229FE70C229DE700BFDB
:10E3E0000004014020AA002000040040001000406A
:10E3F0000000014030EF03082C0100011901000169
:10E400002C4B98423DD0B0F1804F3CD0A3F57C43DB
:10E4100098423AD003F58063984238D003F5806380
:10E42000984236D003F58063984234D003F5806378
:10E43000984232D003F57043984230D003F57053C0
:10E4400098422ED003F5806398422CD003F5806368
:10E4500098422AD0A3F59833984228D003F58063D8
:10E46000984207D003F58063984208BF0D2202D07E
:10E47000002070470C22104B03EBC20393F85C00A2
:10E4800070470022F7E70122F5E70222F3E70322B3
:10E49000F1E70422EFE70522EDE70622EBE707228A
:10E4A000E9E70822E7E70922E5E70A22E3E70B228A
:10E4B000E1E700BF0000014030EF03082DE980488C
:10E4C000013085B0C3B203938A4D8B4F8B4C8C4E79
:10E4D0000A230293DFF82C9226F002F94FF4FA7A1D
:10E4E0004FF0100C4FF47A70D9F80430C3F30803DE
:10E4F000002B40F0C180EFF31183002B40F0BC8073
:10E500002968A26800BF2B689942F9D1D7F800E0CA
:10E5100000FB0EF39B1AB3FBFEF300FB01314FF03F
:10E52000010E0191D9F80430C3F30803002B40F029
:10E530008780EFF31183002B40F082802B68A16865
:10E5400000BF2A689342F9D1D7F800B000FB0BF264
:10E55000521AB2FBFBF200FB0323019A9B1AB3F59C
:10E560007A7FDFD3BAF1010ABED1039B002B40F0C2
:10E57000BD804FF47A7ADFF88C9150464FF0100C42
:10E58000D9F80430C3F30803002B40F09280EFF376
:10E590001183002B40F08D802968A26800BF2B6892
:10E5A0009942F9D1D7F800E000FB0EF39B1AB3FBB8
:10E5B000FEF300FB01314FF0010E0191D9F8043058
:10E5C000C3F3080303BBEFF31183EBB92B68A16816
:10E5D00000BF2A689342F9D1D7F800B000FB0BF2D4
:10E5E000521AB2FBFBF200FB0323019A9B1AB3F50C
:10E5F0007A7FE3D3BAF1010AC2D1029B013B0293B5
:10E600007FF468AFFDF722F8EFF311888CF31288DE
:10E61000A1682368DB0344BFC6F800E0A1682B684B
:10E6200032685FFA88F888F31188D7F800801A44B6
:10E6300000FB08F35B1AB3FBF8F300FB0233D4E7EB
:10E64000EFF311888CF31288A1682368DB0344BFC1
:10E65000C6F800E0A1682B6832685FFA88F888F392
:10E660001188D7F800801A4400FB08F35B1AB3FB4B
:10E67000F8F300FB023370E7EFF311828CF312889A
:10E68000D4F808E02368D90303D501233360D4F814
:10E6900008E02B683168D2B282F311883A681944D5
:10E6A00000FB02F3A3EB0E03B3FBF2F300FB01311B
:10E6B00035E7EFF311828CF31288D4F808E0236871
:10E6C000D90303D501233360D4F808E02B683168FF
:10E6D000D2B282F311883A68194400FB02F3A3EB2B
:10E6E0000E03B3FBF2F300FB013164E7184625F09B
:10E6F00059FE3EE7109600201496002010E000E03E
:10E700000C96002000ED00E02DE9F047AC4FAD4E37
:10E7100021F0DEFFBE421ED2DFF83483DFF83493EF
:10E720004446258862197DB14A450DD2052D0BD985
:10E7300033886188C3F30B03994200F0EE801446DE
:10E7400025886219002DEFD1716830461436FBF729
:10E75000E7FDBE42E4D39C4A1378A3F117010229D6
:10E760000FD99A4911F83300002840F01B81D800D6
:10E770000144497829B1964911F833300BB918236F
:10E780001370944C6378022B84BF0023637023784A
:10E79000022B84BF002323708F4B9A78042A00F049
:10E7A000F88032B91A88B2F5F07F84BF4FF4F07266
:10E7B0001A808A4D8A4A2B681A40002A00F0FB8092
:10E7C000D80700F1E180590400F1D9801A0700F15F
:10E7D000D1809B0400F1C780824D2B685A8C998CA4
:10E7E000914224BF00225A84FFF7F0F81BF066FC28
:10E7F000002800F0B4804FF40070FBF7C7FD4FF421
:10E800008020FBF7C3FD4FF00070FBF7BFFD4FF01A
:10E810008060FBF7BBFD6378022B06D8724A734910
:10E8200003EB430302EB83030B602378022B07D82F
:10E8300003EB83016E4AC3EBC10302EB43032B607E
:10E8400015F0B4F9002130226A4830F08AFA2868BD
:10E850002AF0DAFB684B2D6803F1500102E0043323
:10E8600099427AD01A78002AF9D19C78D8788442D3
:10E87000F5D26249624B0A7028461D6022F07CFD89
:10E88000604B614A1E7961496148624B1160C8253D
:10E89000642212FB0652604C406B31F8061C5A6031
:10E8A000002221809A60DA601A615A619A61DA6105
:10E8B00083F8202083F8212008B121F03FFD574B39
:10E8C0009FED575A1B88574A9FED576A557B574C07
:10E8D00057495848086006EE903AF8EEE66A138900
:10E8E000C5EE265A07EE103A5389127BC4ED005A42
:10E8F00007EE903AB8EEC77A4F4BF8EEE77A1D7202
:10E900005A7227EE067A67EE867ABDE8F04783ED05
:10E91000017AC3ED007A21F0C3BE63799B077FF4CF
:10E920000EAF716894F804A03046FBF7F9FC338809
:10E93000BAEB133F04D01436BE42FFF4F1AE0AE73F
:10E9400073887068AA1FC3F30B039A4204F106018F
:10E95000A8BF1A462DF084FFEDE7012289E737486A
:10E960000BF072FB47E73648FBF710FD4020FBF742
:10E970000DFD31E73348FBF709FD2B6829E73248E5
:10E98000FBF704FD2B6821E73048FBF7FFFC2B6801
:10E9900019E79A8AB2F57A7FBFF40BAF4FF47A7217
:10E9A0009A8206E7D8000C186468002C7FF4E0AE69
:10E9B00017241470DCE643F008032B6000E700BF67
:10E9C0002406000888010008488B0020C0110408B4
:10E9D000E81F0408D9780020245D00200C7B00206B
:10E9E00009600002E8780020EC780020CC4200208A
:10E9F000D6790020742300204C8B00204801002091
:10EA0000A82300205C420020C0B600209A78002095
:10EA1000A0710020446C00202478002034430020A2
:10EA2000C0C9FB48E41F002017B7D1383843002085
:10EA3000204000203661023DFC3F002014A9002048
:10EA40000940000201600002092000020860000283
:10EA5000024000080080000808B521F039FEFBF7ED
:10EA6000D3FC21F01DFEFFF74FFE0120BDE808405A
:10EA70002CF046BC2DE9F04F013085B0C3B20393B2
:10EA80000B4602918B4C8C4E002B00F099808B4DE5
:10EA90008B4FDFF8309225F023FE4FF4FA7A4FF0D7
:10EAA000100C4FF47A70D9F80430C3F30803002B2C
:10EAB00040F0DE80EFF31183002B40F0D98029680D
:10EAC000A26800BF2B689942F9D1D7F800E000FB9B
:10EAD0000EF39B1AB3FBFEF300FB01314FF0010E66
:10EAE0000191D9F80430C3F30803002B40F087806C
:10EAF000EFF31183002B40F082802B68A16800BFE8
:10EB00002A689342F9D1D7F800B000FB0BF2521AF1
:10EB1000B2FBFBF200FB0323019A9B1AB3F57A7F49
:10EB2000DFD3BAF1010ABED1039B002B40F0BD80B8
:10EB30004FF47A7ADFF88C9150464FF0100CD9F8E8
:10EB40000430C3F30803002B75D1EFF31183002BBE
:10EB500071D12968A26800BF2B689942F9D1D7F812
:10EB600000E000FB0EF39B1AB3FBFEF300FB013148
:10EB70004FF0010E0191D9F80430C3F3080313BB21
:10EB8000EFF31183FBB92B68A16800BF2A68934299
:10EB9000F9D1D7F800B000FB0BF2521AB2FBFBF22E
:10EBA00000FB0323019A9B1AB3F57A7FE3D3BAF1F2
:10EBB000010AC4D1029B013B0293002B7FF467AF93
:10EBC00005B0BDE8F08FEFF311888CF31288A168CF
:10EBD0002368DB0344BFC6F800E0A1682B683268F5
:10EBE0005FFA88F888F31188D7F800801A4400FB90
:10EBF00008F35B1AB3FBF8F300FB0233D2E7EFF341
:10EC000011888CF31288A1682368DB0344BFC6F81F
:10EC100000E0A1682B6832685FFA88F888F31188F1
:10EC2000D7F800801A4400FB08F35B1AB3FBF8F333
:10EC300000FB023370E7EFF311828CF31288D4F8F3
:10EC400008E02368D90303D501233360D4F808E032
:10EC50002B683168D2B282F311883A68194400FBFC
:10EC600002F3A3EB0E03B3FBF2F300FB01317FE7EA
:10EC7000EFF311828CF31288D4F808E02368D903EB
:10EC800003D501233360D4F808E02B683168D2B291
:10EC900082F311883A68194400FB02F3A3EB0E03D8
:10ECA000B3FBF2F300FB013118E7184625F07AFBBD
:10ECB0003EE700BF10E000E00C9600201096002018
:10ECC0001496002000ED00E0204B5B68C3F30803BE
:10ECD00030B4BBB9EFF31183A3B91D4B1D4C1868B9
:10ECE000A16800BF1A689042F9D11B4B1C684FF411
:10ECF0007A7202FB04F3591AB1FBF4F130BC02FB47
:10ED000000107047EFF31182102383F3128811492A
:10ED10008C680B6813F4803F104B02D00120186000
:10ED20008C680B49D2B20D68186882F311880A4BBF
:10ED300019684FF47A72284402FB01F31B1B30BCA4
:10ED4000B3FBF1F302FB0030704700BF00ED00E0C1
:10ED50001096002010E000E0149600200C96002091
:10ED60002DE9F84F8046FFF7AFFF254E2549DFF824
:10ED7000A0E0254A254D844610274FF47A740120DF
:10ED8000DEF80430C3F30803D3B9EFF31183BBB942
:10ED90000B68D2F808A000BFD1F800904B45F7D11E
:10EDA000D6F800B004FB0BF9A9EB0A09B9FBFBF993
:10EDB00004FB0393A3EB0C034345E1D3BDE8F88FB9
:10EDC000EFF3118A87F31288D2F808B01368DB03D7
:10EDD00044BF2860D2F808B00B68D5F800905FFAFD
:10EDE0008AFA8AF31188D6F800A0994404FB0AF342
:10EDF000A3EB0B03B3FBFAF304FB0933DAE700BF21
:10EE0000149600201096002010E000E00C960020E0
:10EE100000ED00E02DE9F04FDFF830C1474A4849E6
:10EE2000484E494D8046102718F1FF38C0F08480C5
:10EE3000DCF80430C3F30803002B5CD1EFF311833B
:10EE4000002B58D10B68946800BF08688342F9D141
:10EE5000D6F800904FF47A7000FB09FEAEEB040E7A
:10EE6000BEFBF9FE00FB03EEDCF80430C3F308033D
:10EE70004FF47A740120FBB9EFF31183E3B90B6807
:10EE8000D2F808A000BFD1F800904B45F7D1D6F8D2
:10EE900000B004FB0BF9A9EB0A09B9FBFBF904FB71
:10EEA0000393A3EB0E03B3F57A7FBDD2DCF80430F5
:10EEB000C3F30803002BDFD0EFF3118A87F3128826
:10EEC000D2F808B01368DB0344BF2860D2F808B05A
:10EED0000B68D5F800905FFA8AFA8AF31188D6F8A1
:10EEE00000A0994404FB0AF3A3EB0B03B3FBFAF372
:10EEF00004FB0933D5E7EFF3118487F31288D2F8C6
:10EF000008901368D80303D501232B60D2F808902A
:10EF10000B682868E4B284F31188D6F800A04FF497
:10EF20007A7400EB030E04FB0AF3A3EB0903B3FBB3
:10EF3000FAF304FB0E3E97E7BDE8F08F10E000E027
:10EF400010960020149600200C96002000ED00E0A2
:10EF500030B4EFF31183102282F312880649074C74
:10EF60000A680748013200250A602560DBB20268A2
:10EF700083F3118830BC7047109600200C96002057
:10EF800010E000E00F4B1B88014643B90E4B0F4ABF
:10EF90001B7810680BB981F00101FAF703BE0C4B26
:10EFA0005A691AB118B91A68106058747047094A3A
:10EFB00018681188084A92FBF1F201210260597425
:10EFC000704700BFE8950020EA950020EC950020EE
:10EFD000F09500200896002020A1070038B5254BA9
:10EFE0005C69236B73B1636D626BCAB1998A1A88CD
:10EFF000C90592B201D5D20700D438BD4FF6F772D9
:10F000001A8038BD636D99891A88890692B2EBD54A
:10F010009206E9D5E26ACAB1988880B29047E2E7E1
:10F0200099891A880D0692B2E0D51006DED5A26A3B
:10F03000616A8A4219D0A1692569885C9880013289
:10F04000B2FBF5F105FB1122A262CFE79B88E269D2
:10F050006169DBB28B54E269E068636D0132B2FB37
:10F06000F0F100FB1122E261BEE7DA6822F08002D3
:10F07000DA60BBE7143D002038B5254BDC68236B14
:10F0800073B1636D626BCAB1998A1A88C90592B26D
:10F0900001D5D20700D438BD4FF6F7721A8038BDBB
:10F0A000636D99891A88890692B2EBD59206E9D5E3
:10F0B000E26ACAB1988880B29047E2E799891A88D3
:10F0C0000D0692B2E0D51006DED5A26A616A8A42C8
:10F0D00019D0A1692569885C98800132B2FBF5F1ED
:10F0E00005FB1122A262CFE79B88E2696169DBB26E
:10F0F0008B54E269E068636D0132B2FBF0F100FB12
:10F100001122E261BEE7DA6822F08002DA60BBE732
:10F11000143D00202DE9F04F2DED028B95B0804677
:10F120001CF0F4FE8E4B1D7825B115B0BDEC028BA2
:10F13000BDE8F08F8B4B1B685905F6D58A4BDFF87D
:10F1400080B21B686BB1894ADBF800101368CB1AD8
:10F150007C2B06D9864811600378013303701FF0B9
:10F16000F9F8844B1B78002B6DD0834C834AD4F87C
:10F170001031A8EB0303934201F2278394F818910E
:10F18000B9F1000F32D17E4F3868FAF76FF8C0B28C
:10F1900001280FD902287B4E42F013803378002BD0
:10F1A00042F00881D4F81C31A8EB0303B3F57A6F61
:10F1B00082F0CE82D4F82031002B44D094F818315C
:10F1C000BBB9714B1B689B7801211E3B00228B420F
:10F1D00084F8181184F82C2142F26C8238680221DC
:10F1E00004301FF069F894F8243110E0D4F820318D
:10F1F0004BB3D4F8283140F6B732A8EB030393425F
:10F2000021D994F82431002B01F0D9865C4F013BC1
:10F21000DBB284F82431002B01F00A84D4F8206199
:10F2200094F82C2116F8011B94F82D313868C4F895
:10F2300020610A44013384F82C2184F82D31FAF737
:10F2400019F8C4F82881514BDBF800601B7843B1F2
:10F250004F4F386828B14F4B1B78013B012B41F2CF
:10F26000F6834D4B1B786BB14C4F3B6853B1DBF8C9
:10F270000030414C03931A46D4F84431D31A632B1F
:10F2800001F29381464F3B78022B01F078863D4E88
:10F2900096F87430032B01F0B683424B1B7873B1A0
:10F2A000414D2B685BB1344CFFF70EFDD4F8503163
:10F2B000039044F61F62C31A934200F231813B4B24
:10F2C0001B78002B7ED13A4B1B7843B12A4CD4F8E3
:10F2D000A03203F5C333A033984581F03782354B14
:10F2E0001B78002B3FF421AF234E334C334D06F2F5
:10F2F000C1272068F9F7BAFF00283FF416AF20684D
:10F30000F9F7ACFF2B7880465A1E33B120682A707B
:10F31000F9F7ACFF0028F2D107E703223946781E3F
:10F320002FF005FD96F8C03296F8C12286F8C38208
:10F3300083F47F4383F0FF039B1A1FFA88F89BB284
:10F34000B8EB132FD5D196F8C222DBB29A42D0D1B6
:10F35000781E1EF0E3FC2B7818442870C9E700BF24
:10F36000EC46002078600020886F0020F0710020BB
:10F37000EC710020026D0020FC1F00203F0D0300F7
:10F3800098710020280000209C710020046D00204E
:10F39000806F00200C6D0020146D00209071002003
:10F3A000B2AC00201C6D0020206D00208C6D002070
:10F3B0009D6D0020266D00202C6D0020306D0020FA
:10F3C00010960020484C2278A2B1484B9B7A53B14A
:10F3D000FFF77AFC464B1B68C31AA3F57A73B3F5A3
:10F3E000FA6F07D82278434B43491868F9F70AFFA8
:10F3F00000232370414CD4F8983203F5C333A03373
:10F400009845FFF460AF3E4DC4F898822B78002BEE
:10F4100041F010873B4D2B78002B41F06B8694F820
:10F420009C2239498D5CEA0702F10780AF0701F1A0
:10F43000C787680701F188872A0748D5334B344EC0
:10F440000D9314AA1146A3F13D0241F8202D00208E
:10F45000A3F140020D4603F8400C0591022311214F
:10F460005170937028463168FBF7F4F928467168AB
:10F47000FBF7F0F9F389274903EBC3039B0005333E
:10F4800081FB0321DB17C3EBA101284689B2FBF7FF
:10F49000F9F9338A03EB8303590089B22846FBF755
:10F4A000F1F91D4B059D1B789B0743BF318901F581
:10F4B0007A7189B24FF47A712846FBF7E3F90C9B15
:10F4C000327D591C0C9128461A701CF0AFFC134A6F
:10F4D00094F89C321178013393FBF1F201FB123363
:10F4E00084F89C32EFE600BFF46C0020F06100204D
:10F4F0009C740020906D0020B46C0020FC1F002044
:10F50000946D0020956D0020986D0020B46C002053
:10F510002872002067666666247200209C6D0020B9
:10F5200094F85631002B41F0CB85D34B1A6802F08A
:10F530000803002B48F603414AF60B404BF60F43F5
:10F5400049F6074604BF03460E4612F0040F4FF07B
:10F55000190118BF1E46970684F8561103D546F4C4
:10F56000804646F02006C54B5F79C6F30909002F97
:10F5700042F013819B79002B42F01E821F466420CB
:10F580004FF0FF3A4FF0000E0C960D96ADF83E701E
:10F59000ADF83CE0CDF842E0CDF846E0CDF84AE0E9
:10F5A000CDF83890ADF840A08DF84E000CAE0FCEDF
:10F5B000B34F84F805E00FC796E80F0007C727F898
:10F5C000023B39464FF0010E1B0CFE261F20C822BD
:10F5D00001F81E39A670A27184F807E0E07094F873
:10F5E0006601207180F0F10383EA0313DAB2130994
:10F5F00083F0E70343EA022383EAC2031BB283EAF0
:10F600000312D2B2C3F3072383EA121343EA02239D
:10F6100083EAC2031BB283F0C80282EA0212D2B2AA
:10F62000C3F3072383EA121343EA022383EAC203E4
:10F630001BB283EA0E0686EA0616F6B2C3F3072269
:10F6400082EA161242EA062200EB0E0382EAC6069E
:10F6500007EB0E0084F86631268011F8013B7340F9
:10F6600083EA0313DBB21A0982EA162242EA032272
:10F6700082EAC3031BB29EB281422680EDD183F0A1
:10F680007C0383EA0313DBB24FEA131E8EEA162EC5
:10F690008EEA032E8EEAC30E0FFA8EFE1FFA8EFC40
:10F6A000784FA4F800C05FFA8EFE4FEA1C2C84F855
:10F6B00028C084F827E007F5C77904F1220A3868E2
:10F6C0007968BA68FB684E460FC610375745B14691
:10F6D000F5D1386830606C4E3B7989F8043006F11A
:10F6E000270784F8B5E184F8B6C116F8011F286829
:10F6F000F9F7C0FDB742F8D194F85731002B41F02B
:10F70000E4846249DBF8002009780A2084F8570174
:10F71000002901F000865E4E01293088079042F2F0
:10F72000518170880690022902F04F80B0880590C0
:10F73000032902F05E81F0880490042902F05481CC
:10F740000529308902F04C810629B6F80A9002F0AA
:10F7500044810729B6F80CC000D0F38994F86611EB
:10F760000C920F4687F0300282EA0212D2B21609DA
:10F770004849089786F07A0646EA022609882771E2
:10F7800086EAC202444EC1EB012186FB017A079E44
:10F790004FF0000E66F30F0E069E12B266F31F4E78
:10F7A0008A44059ECDF834E0C917C1EB6A2A0027C8
:10F7B00082EA0211C9B266F30F07C2F307220026DC
:10F7C00082EA111260F30F06002007926CF30F001B
:10F7D000049A8DF845A063F31F40079B109062F3D5
:10F7E0001F4769F31F464FF000090E970F968DF8DB
:10F7F000449043EA01220DF1300E82EAC106BEE8D0
:10F800000F0036B286F0C80C8CEA0C1C1C4F84F832
:10F8100005905FFA8CFCC6F307260FC786EA1C1614
:10F8200046EA0C239EE8030083EACC031BB283F074
:10F83000230247F8040B82EA0212D2B2C3F3072371
:10F84000089E83EA1213384643EA022383EAC2027F
:10F8500006F1010E20F814194FF0230C1621FE2694
:10F86000C82384F866E102372280E17084F807C07B
:10F87000A670A371114611E02072002000720020D2
:10F8800004200020FE1F00208B2100201079002082
:10F89000C05B0020386C00200308208010F8013B7A
:10F8A0004B4083EA0313DBB21A0982EA112242EACF
:10F8B000032282EAC3031BB299B2B8422180EDD180
:10F8C00083F0F40383EA0313DBB24FEA131E8EEADC
:10F8D000112E8EEA032E8EEAC30E0FFA8EFE1FFA49
:10F8E0008EF7C84E27804FEA172C5FFA8EFE84F8F9
:10F8F0001EE084F81FC07168B2683068F36806F5CE
:10F90000C7770FC730697169B26904F28F1607C7EC
:10F9100004F2AD1784F8ADC184F8ACE116F8011F0C
:10F920002868F9F7A7FCB742F8D194F85A31002BB0
:10F9300041F0DB83B44B06931B681922980684F8C8
:10F940005A2140F1EA82B14BB14E1B78990741F13F
:10F950002187337D042B8CBF03270227FFF7B4F9DF
:10F96000338A32890C9003EB83035B00ADF84A3095
:10F970004FF47A7033688DF84C700E93F18996F8D5
:10F9800014E073688DF84DE000FB02F24FF0000CBC
:10F990000CAF4FF0FF30CDF834C010920F93ADF89C
:10F9A00048101190BE46BEE80F000597994F0FC74B
:10F9B0009EE80F0007C73A46182122F81C39E1716A
:10F9C00094F8661184F805C081F0780383EA031384
:10F9D000D8B2030983F0F60343EA002383EAC003A5
:10F9E0001BB283EA0310C0B2C3F3072383EA1013E8
:10F9F00043EA002383EAC0031BB283F0C80080EA15
:10FA0000001E5FFA8EFEC3F3072080EA1E1040EA54
:10FA10000E2080EACE0000B280F0180383EA0313C0
:10FA2000DBB2C0F3072080EA131040EA032080EA2B
:10FA3000C30301F1010EFE204FF01E0C4FF0C80968
:10FA4000A0700237217184F866E1238084F803C036
:10FA500084F80690184612F8011B414081EA011112
:10FA6000C9B20B0983EA102343EA012383EAC101E7
:10FA700009B288B2BA422080EDD181F0180181EA42
:10FA80000111C9B20A0982EA102383EA012383EA39
:10FA9000C1031BB29AB25B490491DBB24FEA122C4C
:10FAA0002280079384F827C084F826300F4601F59A
:10FAB000C77A04F1220938687968BA68FB68D646C3
:10FAC000AEE80F0010374F45F246F4D13868CEF853
:10FAD0000000DFF84C919DF81C3084F8B43109F136
:10FAE000260784F8B5C1CA461AF8011F2868F9F735
:10FAF000C1FB5745F8D1FFF7E7F8069B71681B6813
:10FB00003289069113F0140F4FF47A71D6F800E0A1
:10FB100001FB02F141F00B860E4694F866A10C90B1
:10FB20008AF06A003C4B3D4FB3F90420CDF834E035
:10FB300080EA0010C0B2030983F0D50343EA002332
:10FB400083EAC0031BB283EA0310C0B2C3F30723E6
:10FB500083EA101343EA002383EAC0031BB287FB46
:10FB60000207D2174FF0000CC2EBA7020698DDF88F
:10FB700014E0109683F0C8070E900F91ADF84A205C
:10FB8000ADF844C0ADF846C0ADF848C087EA0717E5
:10FB9000FFB2C3F30726BEE80F0086EA171646EA4F
:10FBA000072686EAC7071B4E84F804A03FB20FC69B
:10FBB00087F021039EE8070083EA0313DBB2C7F353
:10FBC000072787EA13170AF1010E47EA032786E899
:10FBD000070087EAC30384F866E14FF0210A4FF07B
:10FBE000FE0E1C27C8220C3684F805C084F807A036
:10FBF00084F802E0A6F11C01E7701846A271238088
:10FC000010E000BFFE1F00202072002024720020A0
:10FC10002872002004200020F871002067666666C4
:10FC20008B21002011F8012B424082EA0212D2B24D
:10FC3000130983EA102343EA022383EAC20212B2C1
:10FC400090B2B1422080EDD182F0680282EA0212C5
:10FC5000D2B24FEA121A8AEA102383EA022A8AEA07
:10FC6000C20A0FFA8AFA1FFA8AF3D74E23804FEAA4
:10FC7000132C5FFA8AFA04F1220384F825C084F871
:10FC800024A006F5C77E0693F36830687168B268F1
:10FC900077460FC7069B10369E42BE46F4D1338886
:10FCA000CA4E3B804F4684F8B2A184F8B3C117F81E
:10FCB000011F2868F9F7DEFABE42F8D194F866E130
:10FCC000C34AC44E84F804E08EF0EB0383EA0313C6
:10FCD000D9B20B0983F0C50343EA012383EAC103C8
:10FCE0001BB283EA0310C0B2C3F3072181EA1011EB
:10FCF00041EA002181EAC0010CCA09B281F0C807BB
:10FD000087EA0717FFB24FF0000C0C92C1F30721EE
:10FD1000059A0D93CDF838C081EA171343EA0723FB
:10FD200007CA83EAC7031BB283F0310786E80700DE
:10FD300087EA0717FFB2C3F3072383EA171343EADF
:10FD4000072383EAC703277A607AA17AE27A267BBF
:10FD500084F805C01BB25F4087EA0717FFB2C3F300
:10FD6000072383EA171343EA072383EAC7031BB277
:10FD7000584080EA0010C0B2C3F3072383EA10138F
:10FD800043EA002383EAC0031BB2594081EA011011
:10FD9000C0B2C3F3072181EA101141EA002181EAD0
:10FDA000C00109B24A4082EA0212D2B2C1F307236B
:10FDB00083EA121343EA022383EAC2031BB25E40C2
:10FDC00086EA0616F6B2C3F3072383EA161343EA5C
:10FDD0000623607BA17BE27B277C94F811C083EA39
:10FDE000C6031BB2584080EA0010C0B2C3F3072319
:10FDF00083EA101343EA002383EAC0031BB259408D
:10FE000081EA0111C9B2C3F3072383EA111343EA5C
:10FE1000012383EAC1031BB25A4082EA0212D2B222
:10FE2000C3F3072383EA121343EA022383EAC203DC
:10FE30001BB25F4087EA0717FFB2C3F3072383EAC9
:10FE4000171343EA072383EAC7031BB28CEA030CA8
:10FE50008CEA0C1C5FFA8CFCC3F3072383EA1C13A7
:10FE600043EA0C2383EACC03A17CE27C5A4F1BB209
:10FE7000594081EA0111C9B2C3F3072383EA111380
:10FE800043EA012383EAC1031BB25A4082EA021209
:10FE9000D2B2C3F3072383EA121343EA022383EAAD
:10FEA000C2031BB283F0270686EA0612D2B2C3F35E
:10FEB000072686EA121646EA022686EAC20636B205
:10FEC0000EF10103B2B231204FF0FE0C0C2184F888
:10FED0006631C8234FEA122E5FFA86FA2280E0715B
:10FEE00084F802C0E170A371049E84F814A084F821
:10FEF00015E07168B268F3683068B6F810C00FC7D3
:10FF000027F803CB84F8A3E184F8A2A119F8011F14
:10FF10002868F9F7AFF94F45F8D194F85E71002FD2
:10FF200041F0DE802D4B94F866E1B3F90010B3F98F
:10FF30000220B3F904309FED2A6A677107EE103A88
:10FF4000DBF800300C938EF06A0383EA031306EEAD
:10FF5000901AD9B20B0983F0D50343EA012383EA4F
:10FF6000C1031BB283EA03115242C9B207EE902AC1
:10FF7000C3F3072383EA111343EA0123F8EEE77A78
:10FF8000F8EEE66AB8EEC77A83EAC1031BB267EE01
:10FF9000867A66EE866A27EE067A002083F0C80C21
:10FFA000CDED0E7ACDED0D6A8DED0F7A109011909A
:10FFB00012908CEA0C160DF13009F6B2C3F3072C3F
:10FFC000B9E80F000EE000BFFE1F0020AF210020A7
:10FFD00024440020042000208C210020F8710020FF
:10FFE00088C3E43A8CEA161C4CEA062C8CEAC60C50
:10FFF000D04E0FFA8CFC0FC68CF01E0799E8070054
:020000040801F1
:1000000087EA0717FFB2CCF3072383EA171343EA03
:10001000072386E8070083EAC707C8214FF00509D0
:100020004FF01E0CFE231C200EF10102A17184F87A
:100030005E9184F807C0A370E070A6F1100184F807
:1000400004E00C36278084F8662111F8013B7B40E0
:1000500083EA0313DBB21A0982EA172242EA032277
:1000600082EAC3031BB29FB2B1422780EDD183F075
:10007000270383EA0313DBB24FEA131E8EEA172E1F
:100080008EEA032E8EEAC30E0FFA8EFE1FFA8EFC46
:10009000A94FA4F800C05FFA8EFE4FEA1C2C84F82A
:1000A00025C084F824E007F5C77904F1220A3868EE
:1000B0007968BA68FB684E460FC610375745B14697
:1000C000F5D19E4E3B88A9F8003006F1240784F84C
:1000D000B2E184F8B3C116F8011F2868F9F7CAF82D
:1000E000B742F8D194F85F91B9F1000F40F0F28770
:1000F000934B1B68052284F85F219A0641F1158114
:10010000904ADFED917AD18907EE101AB8EEC77ADE
:1001100013F0140F27EE277A01F071838B4BDFED7C
:100120008A6AD3ED007AF8EEE77A67EEA67A94F859
:1001300066C1874B874AB3F90410B2F90620864E90
:1001400086488DED0D7A8CF0220383EA0313DFB22B
:100150003B0983F0590343EA072383EAC703B2F557
:10016000FA6F1BB2A8BF4FF4FA6283EA0317FFB21B
:10017000B2F57A7FC3F3072383EA1713B8BF4FF4AE
:100180007A724FF0640E43EA0723A2F57A720EFBEF
:1001900002F283EAC70786FB02E680FB01E03FB27A
:1001A000C917D217C2EBA612C1EBA0034FF0000A89
:1001B0000CA987F0C806CDED0E7AADF84220ADF857
:1001C0004030CDF830A0CDF83CA08E4686EA061629
:1001D000F6B20591C7F30727BEE80F0087EA1617A6
:1001E00047EA062787EAC606524FDEF800E084F8A1
:1001F00004C00FC736B286F04A0383EA0313DBB2AA
:10020000C6F3072181EA13113A4641EA03210CF1B2
:10021000010C81EAC303142042F810E9FE264FF0D6
:100220004A0E002184F866C14FF0C80CE0702380AC
:10023000043784F807E0A670617184F806C0184698
:1002400012F8011B414081EA0111C9B20B0983EA8E
:10025000102343EA012383EAC10109B288B2BA42FA
:100260002080EDD181F0140181EA0111C9B24FEA79
:10027000111E8EEA102E8EEA012E8EEAC10E2E4B32
:100280000FFA8EFE1FFA8EF61F464FEA162C5FFA03
:100290008EFE84F81CE084F81DC0386859689A689E
:1002A000DB68B7F818A0049726803E4607F5C777A5
:1002B0000FC73069716903C704F28F16A7F800A051
:1002C000374684F8ABC184F8AAE104F2AB1A17F8F8
:1002D000011F2868F8F7CEFFBA45F8D1204B214A14
:1002E0001B781278013B12F00100DBB214BFC02171
:1002F0004021172B03D81C4A134493F830901B4B12
:100300001A8897071ABF002341F01001012312F445
:10031000027F18BF022312F0100F18BF062312F03D
:10032000200F18BF1023002841F008824FF0030C63
:100330001EE000BF04200020FE1F00208B210020B3
:1003400020720020287200200AD7233CF47100207C
:10035000F8710020C05B0020D34D621067666666AE
:10036000488B0020F1B50020F8EF03083A6C00201C
:1003700094F866E10C938EF0460383EA0313DAB235
:10038000130983F0920343EA022383EAC2031BB2F8
:1003900083EA0310C0B2C3F3072282EA101242EAD2
:1003A000002282EAC00212B282F0C80787EA071769
:1003B000FFB2C2F3072282EA171200238DF837C07A
:1003C000032042EA072C059A8DF834908DF83530D9
:1003D0008DF836108DF8380007CA8CEAC70C0FFA72
:1003E0008CFCD04FE3718CEA0C1903C75FFA89F9D2
:1003F000CCF3072C8CEA191C4CEA092181EAC909C3
:1004000094F808C03A700FFA89F98CEA090C8CEA62
:100410000C1C5FFA8CFCC9F3072282EA1C1242EA28
:100420000C22607AA17A94F80B90637182EACC0274
:1004300012B2504080EA001C5FFA8CFCC2F3072025
:1004400080EA1C1040EA0C2080EACC0000B2414057
:1004500081EA0111C9B2C0F3072282EA111242EA0D
:10046000012282EAC10212B289EA020989EA091963
:100470005FFA89F9C2F3072282EA191242EA0922D5
:1004800094F80CC0607BA17B84F804E082EAC90286
:1004900012B28CEA020C8CEA0C1C5FFA8CFCC2F3E0
:1004A000072282EA1C1242EA0C2282EACC0212B231
:1004B000504080EA0010C0B2C2F3072282EA101254
:1004C00042EA002282EAC00212B2514081EA0111DE
:1004D000C9B2C2F3072282EA111242EA012282EA79
:1004E000C102E17B94F8109013B281EA030282EA20
:1004F0000212D2B2C3F3072383EA121343EA0223A0
:1005000083EAC2031BB289EA030282EA0212D2B270
:10051000C3F3072383EA121343EA022383EAC203E5
:100520001BB283F0320282EA0212D2B2C3F3072373
:1005300083EA121343EA022383EAC2031BB29AB28C
:100540004FF0FE0C5FFA83FB0920C8210EF1010E6B
:1005500084F802C04FEA122CE070A17184F866E1C1
:10056000228084F812C084F811B0049B186859687E
:100570009A68B3F80CA007F5C07EAEE8070007F54F
:10058000C8778EF80290AEF800A084F8A0C184F875
:100590009FB116F8011F2868F8F76CFEB742F8D132
:1005A000039BC4F85031FEF78ABEDFF898A15E4E77
:1005B000DFF8949141201DF02BFEBAF9023086FB42
:1005C0000320DB17C3EBA00080B21DF005FEBAF9D3
:1005D000003086FB0320DB17C3EBA00080B21DF0C8
:1005E000FBFDBAF9043086FB0320DB17C3EBA00048
:1005F00080B21DF0F1FD99F800103868F8F73AFE66
:1006000094F848A11AF0010600F0F784474B0693CE
:100610001B689A0673D5464B464E1B789B0741F1E3
:100620005180337D042B8CBF4FF0030A4FF0020A38
:1006300047201DF0EDFD30681DF09AFD70681DF03B
:1006400097FD3D4AF3893868A2FB0323C3F34713A0
:1006500019460493F8F70EFE069B99F800101A68E5
:10066000049B12F0140F83EA010389F8003040F074
:1006700067863389642000FB03F01DF079FD367D29
:1006800038684AEA8606F6B23146F8F7F3FD99F87B
:10069000003038685E40314689F80060F8F7EAFDBE
:1006A00094F848A1BAF1000F29D1244E4F201DF033
:1006B000AFFD30681DF05CFD70681DF059FD5046BF
:1006C0001DF056FD01213868F8F7D4FD184A99F855
:1006D00000301678386806F00106314683F00103D1
:1006E00089F80030F8F7C6FD99F8003038685E40A8
:1006F000314689F80060F8F7BDFD94F848A1039BE6
:100700000F4AC4F844310AF10103DBB2A2FB031221
:10071000D20802EB8202A3EB420384F84831FEF7D1
:10072000B1BD00BF0420002067666666207200200D
:1007300024720020287200201F85EB5124440020E1
:10074000CDCCCCCCF87100209471002094F8A43268
:10075000C24AC4F8A08202EB8302926C42B314AD89
:1007600004F2AB23BE4E45F8203D002104F2BD2328
:1007700031800D9380211523A52784F8AA322846BD
:1007800084F8A91284F8A872904728463188FAF7AD
:100790009FF80C9DB34804F52A716D1A152DA8BF5A
:1007A00015252A462CF05CF8AF4A94F8A43215704F
:1007B000AE4A013382FB0312A2EBE37202EB420268
:1007C0009B1A84F8A432FEF78ABDA94AA94BD4F833
:1007D0001411DBF800001B88D77AA74A401A4FF49F
:1007E0007A71DEB201FB07F11B0A96771675884213
:1007F0004FF00006D37753759670167180F0D18450
:100800009E4E9F4BD6F800C01B689E4E9E48DFF858
:10081000989201688068DFF894E286FB0376DB1724
:10082000C3EB661303F5FA739BB293761B0AD37678
:1008300089FB0173C917C1EBA30189FB007911770B
:10084000C0170912C0EBA90051778E4982F8200029
:100850000CF5EA43001281FB0C71303382F8210061
:100860004FEAEC701B12C0EB6110884E9EF800E05E
:1008700082F823307830864B82F824000CF1300166
:10088000307D03901EF0020F82F82210987600F05F
:100890008584D6F800E07F4AD6F804A07E48DFF8C9
:1008A00010C282FB0E194FEAEE7182FB0A72C1EB95
:1008B000A9514FEAEA79C9EBA25200FB01E900FB1A
:1008C00002A009EB490900EB40004FEA490940004A
:1008D000049207468CFB0920801405908CFB072CA2
:1008E000F089049A3689079702EB820206F5FA76B8
:1008F00000EBC00002EB8202B6B204960892059E9D
:100900008200099201EB81014FEAE972B01A01EB12
:100910008101624E06910246039906FB1292069EE1
:1009200040B2052900EB86004FEAE7714FEAAC4C74
:100930005A4E0590ACEB0100014606FB1070089E74
:10094000504FDFF870C14FEADA7A49B201EB860105
:100950004FEADE7E87FB006983F80EA087FB026A00
:10096000099F83F809E0DFF850E13E468EFB066EF2
:10097000BCF8006003969DF810605E75049EBDF89B
:1009800014C083F80AC04FEA162689B204964FEACB
:10099000E2724FEAE777424ED973C2EB6A12C7EBB5
:1009A000AE174FEA1C2A4FEA112E4FEAE070039966
:1009B000368883F80BA0C0EB691083F810E04FEA8B
:1009C00022291A739DF810209A754FEA202CC7F33C
:1009D000072A4FEA112134BF4FF0320E4FF0330E89
:1009E0009DF80C2083F80D90587483F812C0DF71C5
:1009F00083F808A0DA74197583F81BE01E77C4F831
:100A00001081FEF7BBBBDFF8B490D9F80000F8F70F
:100A10001DFC00283EF441ACD9F800000121F8F794
:100A200011FC0222002386F874203B70FEF735BCCF
:100A300094F82C1194F82D3138684A1C013384F84D
:100A40002C2184F82D31F8F715FCFEF7FABB154C74
:100A5000DFF86C904FF0000A3FE000BFF8EF0308AA
:100A6000006B00203073002045730020565555550B
:100A7000C46F0020BC6F0020346D0020E87100209E
:100A8000F47100201F85EB511472002028720020A1
:100A9000606D00206BCA5F6B806967FF40420F008A
:100AA0002E440020FC1F002067666666247200202A
:100AB00083DE1B432C440020D34D621038AD002050
:100AC000280000201B2B00F06F820D2B00F04B81C3
:100AD0004FF0010389F801303868F8F7C7FB0028A8
:100AE00039D03868F8F7BAFB83B27E2BDBF80020E8
:100AF0002AD099F801100029EED194F82E21002A6D
:100B0000E0D07D2B00F0368294F83CE1BEF1000F7E
:100B100004D080F02003DBB284F83C11511CC9B230
:100B20002244092984F82E1182F8303100F016820F
:100B30000829D1D8B4F83A21134403EB132303F066
:100B4000FF03A4F83A31C7E784F82EA184F82FA157
:100B500089F801A0C0E794F83D3133B194F8313100
:100B600084F83D01302B00F0C18594F82F21C54B4E
:100B7000C549DFF850A3DFF850E391464A46002A02
:100B80003EF46FABDBF80020921B012A24D894F8C6
:100B90003E21002A40F01E8294F83FC133F81C0029
:100BA000F8B94FF0010284F83F210A689706E5D5AD
:100BB0009AF800209007E1D5B44EB549F2894FF478
:100BC000F36303FB02F381FB0321DB17C3EB61112A
:100BD0004FF403601DF056FB002384F82F31FEF71D
:100BE00040BB0CF1010C5FFA8CFCB0F5E06F84F8AF
:100BF0003FC100F098801BD8B0F5047F00F023813E
:100C000035D8B0F5887F00F0CD80B0F5007F00F0DA
:100C1000B380B0F5807FB1D10A685207AED59D4B45
:100C200019681DF02FFB002384F82F31FEF719BB44
:100C3000B0F5026F00F05A816AD8B0F5E46F00F0A9
:100C40008180B0F5006F00F0D680B0F5E26F95D1ED
:100C5000914BDA6B998A642303FB02F393FBF1F166
:100C60001DF010FB002384F82F31FEF7FABAB0F51F
:100C7000826F00F05181B0F5C06F00F02781B0F5B0
:100C8000806F7FF47BAF94F840310133DBB2032BEC
:100C900000F2AD8142F2107184F8403101FB03F1A2
:100CA0007E4B1B88002B40F0A08101317C4B1B78D0
:100CB000DB077C4B1B8848BF0431DF0748BF0A3184
:100CC000980748BF14311A0648BF2831DF0548BFCE
:100CD0002831580748BF64311A0748BFC8319F05FB
:100CE00048BF01F5C871980648BF01F57A71DA0668
:100CF00048BF01F5FA615F0648BF01F57A614FF41C
:100D000080601DF0BFFA002384F82F31FEF7A9BAE6
:100D1000B0F5046F1AD0B0F5116F52D0B0F5036F73
:100D20007FF42CAF41E75C4B91469A6B998A642320
:100D300003FB02F393FBF1F11DF0A4FA84F82F9169
:100D4000FEF78FBA544B91461A6CEFE7564BB3F946
:100D5000041001EB8101914649001DF093FA84F8DB
:100D60002F91FEF77EBA4FF0010184F82E1184F81E
:100D70003031A4F83A21AFE69EF80620002A3FF46D
:100D8000FDAE4A4B4A491B6881FB0321DB17C3EBCD
:100D9000A1014FF400701DF075FA002384F82F3183
:100DA000FEF75FBA0A6852077FF5E8AE414B4FF491
:100DB000887019681DF066FA002384F82F31FEF759
:100DC00050BA9EF80520002A3FF4D8AE3A4A10786F
:100DD00000283FF4D3AE394B1B8803EB8303590043
:100DE00091FBF0F14FF411601DF04CFA002384F8F0
:100DF0002F31FEF736BA0A6897067FF5BFAE9AF82C
:100E0000002090077FF5BAAE1CF0010F1F4E20495D
:100E100000F05C84726882EAE273A3EBE27303EB96
:100E20005303A1FB0331C908002AACBF41F00041C4
:100E300041F040414FF400601DF024FA002384F893
:100E40002F31FEF70EBA9EF80520002A3FF496AE29
:100E5000194A107800283FF491AE194B5B7B002BA8
:100E600000F09484154B1B8893FBF0F000EB80009E
:100E700041004FF404701DF005FA002384F82F316F
:100E8000FEF7EFB9F8EF0308207200202872002067
:100E90001F85EB51F4710020A0710020686C0020C8
:100EA000F1B500203A6C0020F87100201472002087
:100EB00067666666E8710020D26F0020BC6F002074
:100EC000C46F002024720020007200209EF80620CB
:100ED000002A3FF453AEC34B4FF4C06099681DF035
:100EE000D1F9002384F82F31FEF7BBB90F68BF0694
:100EF0007FF544AE9AF800C01CF0020F3FF43EAEFE
:100F0000B94E33896421914601FB03F11DF0BAF912
:100F100084F82F91FEF7A5B90A68900640F1F18098
:100F2000B24BB14E1878317D00F00203002B0CBF9C
:100F300000234FF47A7340F6B83208BF4FF4FA62D8
:100F400010F0010F18BF134619444FF482601DF0D2
:100F500099F9002384F82F31FEF783B9B4F83A21C8
:100F6000C2F1FF0293427FF4B3AD4FF0010384F866
:100F70003D31ADE54FF0010384F83C31ACE5FDF7C0
:100F8000A3FE9B4B1B68C01A40F6B833984200F290
:100F90001E81DFF89CA29AF804303A2B00F0BA8246
:100FA00000233B70FEF779B93868F8F75FF900283D
:100FB0007FF48EAD4FF0010384F82F318CE5C4F837
:100FC000203184F818318B4F1DF0AAF994F82431A0
:100FD000FEF71DB9884906201CF026FF002384F87F
:100FE0003E0184F82F31FEF73CB902315EE6012361
:100FF00084F8403142F2107152E6804B1B88D805CC
:1010000013D4D90600F17A839A0600F1F1835806C9
:1010100000F1F383190700F1F983DA0700F1148472
:1010200013F0020F0CBF04260C26754B754A1B7873
:10103000D27803F001030AB143F002035320049372
:101040001DF0E6F8704A128802EB820202EB82027F
:10105000900080B21DF0C0F800201DF0BDF86B4A72
:101060006B4912883868C2EBC212520081FB023110
:1010700011444FEAE27ACAEB612A5FFA8AFA5146D2
:10108000F8F7F8F899F80020049B38681E438AEABC
:10109000020A002189F800A0F8F7ECF83146386818
:1010A000F8F7E8F899F8003038687340DBB2194671
:1010B00089F80030F8F7DEF894F848A1FFF7F2BAA3
:1010C000013B84F85631FEF717BB013B84F85731DA
:1010D000FEF72BBC09F1FF3984F85F91FFF760BA86
:1010E000013F84F85E71FEF7FDBF013B84F85A3181
:1010F000FEF713BF47493A201CF096FE2870FEF712
:10110000E2B8454A1268120600F1FA82434A127B9D
:10111000002A3FF433AD94F84111032900F28A8389
:10112000DFE801F0322819023D4B1B6859799A79A2
:10113000DB7901F1407101EB022101EB0341002356
:1011400084F841314FF482601DF09CF8002384F84C
:101150002F31FEF786B8334B1A68137A507992789C
:101160001B0403EB002313444A1C84F8412103EBC6
:101170000161E7E72B4B1A68D379107952781B0489
:1011800003EB00231344EFE7264B1A689379D078DA
:1011900012781B0403EB00231344E5E72D22DA76D3
:1011A0002DE4214BDBF800101B78C4F81411013B2F
:1011B000012B3FF625AB1021022391701371FFF72D
:1011C0001FBB1DF09DF801233370FDF7F3BF174AD5
:1011D000B2F84A3100210133A2F84A313970FEF7E2
:1011E0005CB800BF14720020287200202472002016
:1011F000B8AC0020987100207DE202083A6C002013
:10120000F1B50020446C0020BC6F0020386C002039
:10121000030820808DBE020878600020C46F002083
:10122000CC420020E8780020406C0020FC1F002009
:10123000A0AC0020A64EA74B00930024A6F13F01CE
:10124000A54BA64A0A9106F8404CA5490B960CA856
:10125000F9F716FC0A9E731C0A9334700A9B292224
:10126000591C0A911A700A9BEA22591C0A911A7099
:101270000A9BC822591C0A910CA81A702AF04CFD2E
:10128000471C0CA93A460A982BF0EAFA0A9AD31995
:1012900001330A93D4550A9B5A1C0A921C700A9B6C
:1012A0005A1C0A921C700A9B5A1C0A921C700A9BB8
:1012B0005A1C0A921C700A9B5A1C0A921C700A9BA8
:1012C0005A1C0A921C700A9B5A1C0A921C700A9B98
:1012D0005A1C0A921C700A9B5A1C0A921C700A9B88
:1012E0005A1C0A921C700A9B5A1C0A921C700A9B78
:1012F000FF22591C0A911A700A9B0122991814A8FE
:101300000A911A7050F8283D9B1B33701AF08EFD1D
:101310002C70FDF7D8BF8C4689460846049105918C
:10132000069107910B46FEF719BA9FED6E7A13F0FE
:10133000140F08BFF0EE477A7EF4F0AEFEF7F7BE6A
:10134000694B1868FFF799B9684A614B12680D93A9
:10135000A3F14007002103F8401C2123D100BB70FA
:1013600040F13A8262490326624B1B885A0500F11C
:101370002982D80700F13E8203F002035E4A002B67
:101380001CBF03261146DFF88891324648462BF0F1
:1013900067FA06EB090314A80133A9F1020140F82A
:1013A000203D00225B1A06F809207B701AF03EFDF2
:1013B000FEF742B8C4F81C8186F80090FDF7FABE2B
:1013C000434A4E4B0D9214AEA2F13D0046F8200D5B
:1013D00019884B4FA2F1400300204FF00A0E02F88B
:1013E000400C082283F801E030469A70F9F74AFA77
:1013F0003B684449DA1781FB0313C2EBA30399B29C
:101400003046F9F73FFA0BF0A9FEBF680C9B3A0C87
:10141000591C0C911A700C9B3A0A591C0C911A70A9
:101420000C9B5A1C0C921F700C9B5A1C0C9218702F
:1014300030461AF0FBFCFDF7FCBF334F9FED338ABB
:10144000B7F9022022480D9007EE902AF8EEE77ACD
:1014500014AE67EE887AA0F13D01FDEEE77A46F81A
:10146000201D00F8403C0823CDED037A00F83F3CF6
:101470001E23BDF80C1000F83E3C3046F9F702FA86
:10148000B7F9003007EE903AF8EEE77A304667EEAB
:10149000887AFDEEE77ACDED037ABDF80C10F9F706
:1014A000F1F9B7F9043007EE903AF8EEE77A3046F2
:1014B00067EE887AFDEEE77ACDED037ABDF80C1081
:1014C000F9F7E0F930461AF0B1FCFDF7AFBF00BF05
:1014D000B46C0020DF7800201024040818240408CD
:1014E0002424040800000000F4710020AC890020CE
:1014F000FC2304083A6C00200C240408BC6F002074
:101500001472002067666666F871002058A08B414F
:10151000776C00209AF80240C4B1013CE4B2013477
:1015200054445146002211F8013B534083EA03130F
:10153000DBB2120ADE0042EA03228C4286EA13136F
:1015400082EA0302EFD1002A7FF42AADC04AC14EDD
:10155000C14B1288C149C24CF261DFF838931A6856
:1015600009689B68F262B4F84A21F066F364D9F81E
:101570000000F163F265F6F7FFFD039000287DF4AB
:1015800087AE0221D9F80000F7F75CFE94F84C31E1
:101590009AF803200492642B4FF0040286F874201A
:1015A00040F07C8194F84D31072B04BF9DF80C303E
:1015B00084F84D3194F84D31079306EB031ADAF8AD
:1015C0000410039108462AF0A7FBDAF808100691E8
:1015D0005FFA80FA08462AF09FFBC0B205900AEB3A
:1015E0000002079B9F48039903900832C27123F0C1
:1015F0000F0286468272059803F00F0300EBCA00C3
:101600008EF80D3052468EF80E000EF10F002BF0C2
:1016100027F9954B059A06990AF1090018442BF011
:101620001FF90398C37903F1010ACBB1013B5FFABB
:1016300083FC0CF1080CDFF860E2844400230730DF
:1016400010F8011B59408B00CA0883EA410302F0DD
:1016500018024B404EFA02F253408445DBB2EFD100
:10166000814A04980AF8023016F04EFF94F84D3182
:101670000022013384F84D3184F84C21039BDDF8BE
:101680000CA09B785BB11AF80510D9F80000F7F7A9
:10169000F1FD01359AF80230EDB2AB42F3D894F87F
:1016A0004C310322013384F84C3186F874203A70AF
:1016B000FFF7ABB902213868F7F7C4FD94F824317D
:1016C000FDF7A5BD4FF0010AFEF7B2BF326882EA0E
:1016D000E273A3EBE27303EB5303A1FB0331C908ED
:1016E000002AB8BF41F08041FFF7A4BB5F49881FC3
:1016F0001CF03EFC84F83E01FFF737BA342694E430
:1017000010230026042218460CA98DF830308DF8DD
:1017100031208DF832608DF833608DF834608DF8AB
:1017200035601CF08FFD84F82F61FDF79ABD4B4B9F
:101730001E6806EB86067600FEF7EFB94C4AD278B3
:10174000002A0CBF4FF0040C4FF0050CFEF710BE42
:10175000012338683370F7F781FD06463868F7F7DC
:101760007DFD72067DF426AD8A2851D08E287DF449
:1017700021AD94F81831002B7DF438AD3D4BC4F801
:1017800020312D2384F82431FDF71BBD304B188800
:10179000FFF76CBB0127FEF7E1B82D499A790B885A
:1017A00003EB830303EB83039F00BFB2002A00F027
:1017B0001181294B1B680FFA83FA0BF0CFFC40B262
:1017C000FDF7E0BE03262C49DDE59C469946184608
:1017D00004930593FDF7C2BF284B294A1B6829498A
:1017E00003F48003002B16BF114604260326BBE535
:1017F00024261AE424490426C5E5102615E4138995
:1018000007EE903AF8EE677AFEF791BC20260CE4DA
:101810001E4B1B689B067DF5CDAC94F81831002B50
:101820007DF4E4AC1A4BC4F820312D2384F8243124
:10183000FDF7C7BC4B1CDBB2042B84F841314FEAE7
:1018400001613FF47CAC7DE40826FFF7EEBB00BFEE
:10185000BC6F00202800002014720020F4710020CA
:10186000FC1F0020D8570020DE5700203421002024
:10187000446C0020346D00200024040878600020AF
:10188000FC230408F4230408042404082072002024
:10189000606D002038AD00200007090E96F875A095
:1018A000574905951AF00F0F04BF0AF1010A5FFAB4
:1018B0008AFABAF1070F28BF4FF0010A4FEA0A1C53
:1018C00006EB0C03187C4F4B03930A18002392F885
:1018D00024104C4A93725FFA8CF31A464A4B964690
:1018E00006EB0C024EEA000001291870D26803F1E1
:1018F00001000CD90239C9B28D1C1D44034603F8FE
:10190000012BAB424FEA1222F9D101310844B44411
:1019100022F060030AF1010A9CF811205FFA8AFAAA
:101920001343BAF1080F037000F1010340D04FEAEE
:101930000A1C06EB0C01344A087C314901449A1A0E
:1019400091F8241055180EF1100E132D5FFA8EFE2B
:10195000C6DD059D0398DFF8BCE0D2B2931DDBB273
:1019600043F04001C17103F1010CCBB10532D3B298
:101970000833C31805930EF10100002310F8011B72
:1019800059408B0083EA4103CA084B401F4902F0CB
:10199000180241FA02F25340059A8242DBB2EDD1BD
:1019A00004980CF80E3086F875A016F0ADFD65E6CB
:1019B000154A059D9A1ACDE7154B6420B3F900A08E
:1019C000FDF7E0BD9C46994618460493059306939F
:1019D000FDF7C4BE4FF0FF33EDE69C46FDF7BEBEFB
:1019E0009C469946FDF7BABE9C4699461846FDF7B7
:1019F000B5BE9C46994618460493FDF7AFBE00BF9E
:101A0000F8EF0308D8570020E55700200007090E1B
:101A100014720020DE5700202DE9F04F95B0B0F988
:101A200008500D81EDB2442D00AF0C46904600F0F9
:101A30003182064643D9812D00F0728200F29880EF
:101A4000542D00F0CC8040F2BD816E2D00F0F0816D
:101A5000802D40F0D080AA4B93F800A00AF1020A32
:101A60001AF0FF0A00F09780A64BDFF8D482A64E4A
:101A7000DFF8D0B29A4403F101090A2516E0322DAD
:101A800000F00C83A5F13C00C0B2132840F20C8397
:101A900000232268511C216015702268D14502F193
:101AA00001012160137076D019F8015B0A2DE6D18F
:101AB000BBF80030FF2BA8BFFF23DBB2E9E7052D01
:101AC00000F0D68120D8022D00F0818040F267819D
:101AD000032D00F0A381042D40F08D808B4920461A
:101AE0002A46F8F7ADFE00212046F8F7F1FE2268FD
:101AF0000021531C0125236028462B4654371170C2
:101B00006381BD46BDE8F08F242D5ED040F2D980C0
:101B1000282D00F0C781382D6DD10A687C4B012536
:101B2000511C216015702268052150192060117028
:101B300022680A2150192060117022680021501972
:101B40002060117022681978501920601170226885
:101B500059785019206011702268997853192360C0
:101B60002B461170284654376381BD46BDE8F08F7F
:101B7000A02D18D040F2E880B82D00F0CF81FE2DC6
:101B800039D1644D05F1080635F8021B2046F8F7F7
:101B90009FFEAE42F8D101252B462846543763817B
:101BA000BD46BDE8F08F5C4B08461968F8F778FE33
:101BB0005A4B20461968F8F773FE594B19682046AE
:101BC0000125F8F76DFE2B46E7E7564BF6E70422B2
:101BD000554920460125F8F733FE2B46C2E70B682E
:101BE00000215A1C226019702268012553192360B4
:101BF0002B461170B6E721462846FAF711FE034638
:101C00000028C8D1742D00F0FB80772D0DD13268EB
:101C1000716891421EBF531C33601178434A08BF5C
:101C20001946204629F096F9B5E7F52D01F0AB836A
:101C3000762D00F0DD81472D00F0888271683368D1
:101C4000292DA1EB030200F0558340F25D82392D6E
:101C500000F03E83532D40F06F83591C316019789A
:101C6000032900F2E0854B1E314D3248DBB203EB15
:101C7000430305EB430301705D7800298BD0531EAD
:101C8000DBB2AB4240F0CF850022C0F80620C0F89E
:101C9000022082725BB1591C33680144421C01333B
:101CA000336013F8010C02F8010F8A42F7D1224B7E
:101CB0001B78002B3FF46FAF012523F08BFE2B46E2
:101CC00050E7202D97D10B681C4D591C6A78216074
:101CD0001A7023682A78591C21601A702368AA7820
:101CE000591C21601A7029892046F8F7F1FD2368F4
:101CF0006A79591C21601A702268A979F9E600BF37
:101D0000E56E00204CF00308FC2A0020DF7800205C
:101D1000C1790020086F0020107AFF1F147AFF1F7E
:101D2000187AFF1F0C7B002090240408BDA4030830
:101D3000B8F40308A89D0020F03D002000720020A8
:101D400067666666242B0020822D7FF454AF0B68F3
:101D5000BB4ABC4D1178BC4A581C206019701189CF
:101D60002046F8F7B5FDB94B22681B88FF2B02F11E
:101D70000101A8BFFF2321601370A96881F310013E
:101D800089B22046F8F7A4FD296801F30F0189B252
:101D90002046F8F79DFDAE4B22681978A9E6012D83
:101DA0007FF429AF0B680022591C21601A70236848
:101DB0005A1C22601D7022682421531C23602B466C
:101DC0001170CFE6522D7FF416AF0A68A14D531C57
:101DD0000321236005F10C0E11702B460620012112
:101DE0002268561C266011702268734502F10101B9
:101DF0002160107000F0DD809979D8790633EFE723
:101E00003268716891421EBF531C33601178924A48
:101E100008BF1946204629F09DF8BCE60B685A1CFD
:101E20000A601D700B680222591C21601A705EE660
:101E3000864B0A681B88834DFF2BA8BFFF23511CCC
:101E400021601370A96881F3100189B22046F8F768
:101E50003FFD824B20461988F8F73AFD296801F3C7
:101E60000F0189B220460125F8F732FD2B4679E6AD
:101E70000B227B492046F8F7E3FC082279492046EB
:101E8000F8F7DEFC0125072277492046F8F7D8FC51
:101E90002B4667E6002A3FF47EAE744B13600125A3
:101EA0002B465FE60B68DFF8E891714E591C022261
:101EB00021601A7023684FF006085A1C226083F8CC
:101EC000008023680A22591C21601A7023680125AA
:101ED0005A1922601D70B9F800102046F8F7F8FC76
:101EE000B9F802102046F8F7F3FC23685A1922606B
:101EF00083F8008023685022591921601A702368E2
:101F00000022591921601A7031882046F8F7E0FC48
:101F100071882046F8F7DCFC2B4623E6554B4DE64E
:101F2000554B1E78033616F0FF063FF434AE534B84
:101F3000DFF860811E4403F1010A4FF00A0920E036
:101F4000B9F1500F00F0A880B9F1320F00F0C18054
:101F5000A9F13C00C0B2132840F2BE8000252946FA
:101F600023685A1C2260204683F80090F8F7B0FCE2
:101F700029462046F8F7ACFC56453FF40CAE1AF85B
:101F8000019BB9F10A0FDBD13D4B9D68196805EB48
:101F900085054FF6FF736D009D42A8BF1D4699420F
:101FA000A8BF194625EAE57521EAE171ADB289B20B
:101FB000D6E7344B21681A78481C20600A70002A42
:101FC0003FF4E9AD013AD2B202EB420205EB420224
:101FD0005578002D3FF4DFAD01351D4401332268F3
:101FE00013F8011F501C9D4220601170F7D1D2E5FB
:101FF0003268511C31601278002A01F0A682102A42
:1020000007BF214B93E842001E46314625686B1CF2
:10201000236020462A70F8F743FC31462046F8F743
:102020003FFC1A4B20461968F8F73AFC204600217D
:10203000F8F74EFC00212046F8F74AFC57E500BFB0
:10204000D26F00201472002000720020BC6F0020AC
:10205000406C0020B8F40308F5AD0308386C00208C
:1020600098240408A4240408B024040851C70008D4
:10207000E42A002058400020E56E00205CF00308B0
:10208000B02A0020A89D0020AC2300202843002077
:102090009C430020F42A0020A24B76E73388FF2BD4
:1020A000A8BFFF23DBB2F4E41BF0BEFD00283FF421
:1020B000EFAC03780A2B25D8B0F9023088FB031265
:1020C000DB17C3EBA2039BB2FF2BA8BFFF23DBB23E
:1020D000DFE498E822005AE71BF0A6FD00283FF451
:1020E0003DAF03780A2B3FF639AFB0F90430B0F9B1
:1020F000061003EB830383F3500521EAE171ADB2CF
:1021000089B22DE70023E2E7212D40F015811A4620
:10211000591C3160844D12F8021B697032605A7884
:102120002A70DA1C32609B78AB703046F8F776FB89
:1021300033682881591C1A46316012F8021B6971F4
:1021400032605B78AB7101252B460BE57268356810
:102150007B623046551BF8F749FB052D38627B6AD8
:1021600001F2D0818026B346012594E80600521A78
:10217000103AB242B8BF1FFA82FB6C4A396A9268C1
:102180003A61521A9345396A7B622046FA6088BFE9
:102190001FFA82FBF8F784FB7B6A002B01F0918128
:1021A000002D41F04D812368C7F800D05D71C0B0AB
:1021B0000533C7F808D0FB61BBF1000F01F02682A0
:1021C0003B6A3A69934281F02682AA463E6A7D6262
:1021D0007C6080255446FB681C1B544BB4F5807F03
:1021E00028BF4FF480749B6832199A4288BF9C1BA9
:1021F000F9F708F82246BC6830462146F9F782F81C
:10220000F969B86104EB000C0B787B6164452ED250
:10221000DFF81C910CF1FF3C04F1FF3E1EF8013F7A
:1022200009EB830219F823405688ECB100234FF4E0
:10223000004204F1FF3816424FEA520202D00878F9
:10224000284308706D0806D10AF1010A4D701FFA83
:102250008AFA01318025D34503D8F44532D8984510
:1022600030DC01339C42E6D1F445D7D1F9617B6A79
:10227000BA6913449BB2D3457B6206D97B6A3A6A3A
:102280001C46D6183B699E42A5D37C68802D1CBF96
:102290000AF101031FFA83FA0AF1020189B220460A
:1022A000F8F716FB2368796A01255A19226020463F
:1022B0001D70F8F70DFB2368534423602B46D7F8B5
:1022C00000D04FE4FB697C681A463B7D1370DDE764
:1022D0005A1C32601A780A2A01F028813046F8F731
:1022E000A9FA3046F8F7A6FA01253046F8F7A2FA1F
:1022F0002B4637E45A1C32601B780A2B01F00F8101
:10230000502B41F038803046F8F788FADFF8248007
:10231000A8F800003046F8F781FA0125A8F8020075
:102320002B461FE4E82A002000720020040F002042
:102330006CF00308E42A00200B3DEF2D00F27382BD
:1023400001A050F825F000BFA12F0108272801089F
:10235000272801082728010827280108272801081D
:10236000272801082728010827280108272801080D
:1023700027280108272801082728010827280108FD
:1023800027280108272801082728010827280108ED
:1023900027280108272801082728010827280108DD
:1023A0002728010827280108FB2F010827280108F2
:1023B000D92F010827280108772F010827280108AD
:1023C00027280108272801084F2F0108272801087E
:1023D000FB31010827280108C93101082728010815
:1023E000A331010827280108913101082728010895
:1023F0003931010827280108B930010827280108C8
:10240000272801082728010827280108971B010809
:102410002728010869300108272801082728010812
:102420004F300108272801082D330108272801080B
:102430002728010827280108272801082133010837
:10244000272801082728010827280108A3320108A6
:1024500027280108553201082728010827280108E4
:10246000E332010827280108272801082728010846
:1024700027280108272801082728010827280108FC
:102480007B2E010827280108072E010827280108AC
:10249000952D010827280108A72C010827280108E5
:1024A0007F2C0108452C010827280108272801084E
:1024B00027280108272801082728010827280108BC
:1024C00027280108272801082728010827280108AC
:1024D000272801082728010827280108272801089C
:1024E000272801082728010827280108272801088C
:1024F000272801082728010827280108272801087C
:10250000272801082728010827280108272801086B
:10251000272801082728010827280108272801085B
:10252000272801082728010827280108272801084B
:10253000272801082728010827280108272801083B
:10254000272801082728010827280108272801082B
:10255000272801082728010827280108272801081B
:10256000272801082728010827280108272801080B
:1025700027280108272801082728010827280108FB
:1025800027280108272801082728010827280108EB
:1025900027280108272801082728010827280108DB
:1025A00027280108272801082728010827280108CB
:1025B00027280108272801082728010827280108BB
:1025C00027280108272801082728010827280108AB
:1025D000272801082728010827280108272801089B
:1025E000272801082728010827280108272801088B
:1025F00027280108272801081B2C01082728010883
:10260000632C01082728010827280108272801082A
:10261000272801082728010827280108272801085A
:10262000272801082728010827280108272801084A
:10263000272801082728010827280108BD2B0108A1
:102640006B2B0108392B010827280108972A01085C
:102650007D2A0108112A010827280108F729010805
:102660008B2901086329010851290108F52801086F
:1026700027280108C528010827280108272801085C
:102680009B2801086D2801085928010831280108F4
:1026900009280108DF270108B32701089B27010843
:1026A00027280108272801082728010827280108CA
:1026B00027280108272801082728010827280108BA
:1026C00027280108272801082728010827280108AA
:1026D00027280108272801087B2701082728010847
:1026E000272801082327010827280108272801088F
:1026F000272801082728010827280108272801087A
:102700002728010809270108C84B1B78DB0700F1BF
:102710008A800125FBF750F9FBF7F6FF2B46FFF700
:1027200021BA5A1C32601A780F2A7CD8991C316061
:10273000C2EBC202BE4958788854D81C30600A44A3
:1027400099785170191D3160D9789170591D316097
:102750001979D170991D316059791171D91D316084
:102760009979517103F108013160DB799371012589
:1027700026F0D2F92B46FFF7F5B93046F8F74EF8B8
:10278000DFF8BC82A8F80E003046F8F747F80125BC
:10279000A8F80C002B46FFF7E5B93046F8F73EF8ED
:1027A000A44A00EB80004300012513802B46FFF76D
:1027B000D9B919465A1C32609F4A11F8020B1070A1
:1027C000316059785170D91C316099789170191D18
:1027D0003160DB78D37001252B46FFF7C3B9304653
:1027E000F8F71CF8DFF88482A8F810003046F8F7F4
:1027F00015F8A8F812003046F8F710F80125A8F8E7
:1028000014002B46FFF7AEB91A46591C316012F876
:10281000020B3260DA1C597832609A7819F0D8FECF
:1028200000287FF4B8A94FF0FF352B46FFF79AB97F
:102830001A46591C3160814912F8020B0870326047
:102840007F495A788A70DA1C32607A4A9B78937092
:1028500001252B46FFF786B97A4B7B4918684E2233
:10286000012529F0FDFF2B46FFF77CB919465A1CBC
:102870003260764A11F8020B10703160597851704D
:10288000D91C31609B7893703046F7F7C7FF704BC7
:102890000125D8802B46FFF765B93046F7F7BEFF14
:1028A000DFF8AC81A8F800003046F7F7B7FFA8F8CA
:1028B00002003046F7F7B2FF0125A8F804002B46C6
:1028C000FFF750B9DFF8A89199F80030002B3FF4DA
:1028D00062A9DFF8A08100253046F7F79FFF0FF0CF
:1028E0008BFA99F80030A8EC010A01359D42F3DB20
:1028F000FFF751B90D2A96D15A1C32601D78072D69
:1029000091D8DFF8749130464FF00C08F7F786FF46
:1029100008FB05F809EB0805A8803046F7F77EFFAD
:10292000E8803046F7F77AFF336828811A46591C49
:10293000316012F8021BA97232605B78EB7230468C
:10294000F7F754FF012549F808002B46FFF70AB9AD
:102950003046F7F763FF3F4B012518802B46FFF702
:1029600001B95A1C32601878060600F1BD862F4B5B
:102970001B78DD073FF50FA9032828BF002001259C
:10298000FAF7FEFF2B46FFF7EDB85A1C32603046CF
:1029900093F800A0F7F72AFF81463046F7F726FFA5
:1029A00005463046F7F722FF80463046F7F736FFF8
:1029B0003046F7F733FF3046F7F73CFFBAF1000F28
:1029C00000F07B86BAF1100F7FF4E5A8224BC3F824
:1029D00000905D60B8F1000F02D0204BC3F800807A
:1029E0001F49204B0222081F01251A701EF062FCAD
:1029F0002B46FFF7B7B80D4B1B78D8073FF5CBA890
:102A00000125FBF7B3F8FBF77FFE2B46FFF7AAB8CB
:102A1000064B1B78DA073FF5BEA8134A1378012549
:102A200043F0040313702B46FFF79CB8F1B5002068
:102A3000DCAE0020B88B0020FC4400205460002055
:102A400094780020E878002048060408004300201D
:102A500040420020F8440020AC23002028430020FE
:102A6000B0230020E243002024720020245D0020D7
:102A7000E56E0020944100200CB50020B74B1B7878
:102A8000D9073FF588A8B64B4FF4C87201251A80C4
:102A90002B46FFF767B8092A7FF7C5AEDFF8EC824F
:102AA0001A46591CD8F80050316012F8021B2970E0
:102AB00032605A78AA70DA1C32609A78642A03F17C
:102AC0000401A8BF64226A713160DA78642A03F1D4
:102AD0000501A8BF6422AA7131601A79EA719A1DB2
:102AE00032605A79642A03F10701A8BF64222A726E
:102AF00031609A79EA7003F108023260DB792B7158
:102B00003046F7F78BFE726833686881D11A002966
:102B10000CDD591CD8F800003160521A002A1978CF
:102B2000417203DD9A1C32605B784370012511F01D
:102B30003DF82B46FFF716B88A4A1068DA1C0146A2
:102B40002133951E356012F8035C0D70551E3560FB
:102B500012F8025C4D70326012F8015C8D70033225
:102B6000934201F10301ECD1F3E05A1C32601A7870
:102B70007D49002A00F053850A7842F00202981C31
:102B80000A707A4D30605B782B753046F7F72EFE71
:102B900028603046F7F72AFE68603046F7F73EFEB9
:102BA00028813046F7F73AFE714AE881137801250B
:102BB00043F0020313702B46FEF7D4BFC2F3470560
:102BC000122D3FF630AEC5B107F1500307F12A09C7
:102BD00003EB450AC846AAF1260A3046F7F71EFE5F
:102BE00028F8020FC245F8D1624B39F8022F23F8BA
:102BF000022FC845F9D1112D09D85F4A6B00023B5D
:102C000013440021223223F8021F9A42FBD15B4A6F
:102C100001231D461370FEF7A5BF1A46591C3160EB
:102C200012F8025B3260DA1C587832609978002D15
:102C300000F02185012D7EF4AEAF09F035FD2B4665
:102C4000FEF790BF454A127812F001017FF4EBAD18
:102C50005A1C32601878012509F068FC2B46FEF7F3
:102C600081BFDFF82C8100233046C8F80030F7F729
:102C7000BDFD0125C8F800002B46FEF773BF1A46BC
:102C8000591C31603E4912F8020BC87032603D4950
:102C90005A784A71DA1C32603B4A9B78D37001251E
:102CA0002B46FEF75FBF3046F7F7B8FD3046F7F723
:102CB000B5FD3046F7F7B2FD3046F7F7BBFD336898
:102CC000284D1946581C2A68306011F8020B82F80A
:102CD0002C003160597882F83610D91C31609B780D
:102CE00082F837303046F7F7A5FD3046F7F7A2FDFA
:102CF0003046F7F79FFD3046D5F80080F7F78EFD98
:102D0000A8F83A003046D5F80080F7F787FD336819
:102D10007268A8F83800D11A01290ADD591C2A68FE
:102D200031601B7882F82E303046F7F783FD336828
:102D30007268D31A032B0BDD3046D5F80080F7F705
:102D40006DFDA8F8320030462E68F7F767FDB086B3
:102D5000286826F0CDFAFEF71EBF00BFF1B50020AF
:102D6000EC420020E8780020247200202872002025
:102D7000E0430020BEAB0020C0AB0020E4AB00204D
:102D800094780020A86E0020B88B0020CC42002050
:102D9000584000205A1C3260BA4DDFF810831B786F
:102DA00088F805303046D5F80090F7F737FDA9F8D8
:102DB00020003046D5F80090F7F730FD7268336890
:102DC000A9F81E00D11A072900F35B84D11A032940
:102DD00000F34384D21A002A05DD591C2A683160A9
:102DE0001B7882F82630FAF7F1FD16F055FDA64B58
:102DF00028681B68002B00F01784012525F020FFB0
:102E00002B46FEF7AFBE1A46591C3160DFF89C8294
:102E100012F8021B88F8021032609C495A780A7036
:102E2000DA1C32609A4D9A782A711A1D3260DB786A
:102E3000092BA8BF09233046AB70F7F7EFFC3368C6
:102E400072682880D11A012905DD3046F7F7E6FCC3
:102E500033687268E8819A4240F05184FAF7B6FD0F
:102E6000336872689A423EF496AE5A1C32601B7800
:102E7000EB7001252B46FEF775BE3046F7F7CEFC0A
:102E800005461EF025FBFF283EF485AE3F2D00F2DF
:102E9000A78307F15009002309F8243D4FEAD5081C
:102EA000494607F12B0087F82B3008F101081EF086
:102EB000EFFA97F82B305FFA88F805F007054345DD
:102EC00005F1010503D197F82C30AB4203D0294618
:102ED00040461EF0E9FA33687268D21A012A7EF77A
:102EE0005AAE5A1C07F15000326000221D7800F8DB
:102EF000252D1EF0C1FA97F82B30AB420AD0654B56
:102F00001B683BB19A79AA4204D31B681B690BB1B9
:102F10002846984733685A1C3260484600221D787C
:102F200087F82C201EF09CFA97F82C30AB423EF428
:102F300032AE584B1B68002B3EF42DAE1B685B690C
:102F4000002B3EF428AE28469847FEF724BE581CB6
:102F50003060514A1D781570091A00297EF71BAEA2
:102F6000991C31605B78003318BF01230125537031
:102F70002B46FEF7F7BD3046F7F750FCDFF83081FF
:102F8000C8F800003046F7F749FCC8F8040030469E
:102F9000F7F744FC0125C8F808002B46FEF7E2BD10
:102FA0003E49102A13464FF0000228BF10230A6042
:102FB0004A608A60CA600A74002B3EF4ECAD326845
:102FC000013913440132326012F8010C01F8010F8B
:102FD0009A42F7D1FEF7DFBDDFF8D8800023C8F8AA
:102FE00000303046F7F702FCD8F8003001250343E3
:102FF000C8F800302B46FEF7B5BD5A1C32601D786C
:10300000132D3FF610AC9A1C326058787B6227F083
:10301000DBFF00283FF407AC7B6A214A017802F805
:103020002510D91C316002EB850299785170191D69
:103030003160D8789070581D306012491B79D37078
:103040000868012510F040FD2B46FEF78BBD154AA0
:1030500003F108010133336013F8010C02F8010F8A
:103060008B42F7D1FEF797BD591C1A4631600E49C5
:1030700012F8020B887032605B784B7001252B468A
:10308000FEF770BDE8780020408B002024B40020BB
:10309000245D00201C790020488B00206442002021
:1030A0004C8B0020EF610020F04200205460002093
:1030B000B43D00200C7B00200721B2FBF1F1C1EBF5
:1030C000C100121A7FF4AFABC9B201F1FF385FFA49
:1030D00088F800293EF45FAD08F1010815465A1C36
:1030E000326093F900A0504608F0A4FB01358146F8
:1030F00000283FF498AB80F802A03046F7F78EFB2B
:103100003268A9F800001346511C316013F8021B05
:1031100089F803103360537889F80430D31C336086
:10312000937889F80630131D3360D27889F805202A
:10313000A845D4D1FEF72FBD5A1C32601A780E2A4A
:103140003FF671AB991C31605D78032D3FF66BAB98
:10315000C748062101FB02F1421803F1030E557125
:10316000C6F800E09D784554191D3160D97851703A
:10317000591D316019799170991D31605979D1705B
:10318000D91D31609B79137101252B46FEF7EABCEE
:103190005A1C3260B74A1B78537501252B46FEF73F
:1031A000E1BC591C31601D781F2D3FF63CAB052A50
:1031B0007FF439AB3046F7F719FBAF4B43F82500E6
:1031C00014F0C0FBFEF7E7BCAB4D05F140083046FC
:1031D000F7F724FB3368A5F88000591C1A463160C4
:1031E00012F8021B85F8821032605B7885F8833014
:1031F0000435A845EBD1FEF7CEBC5A1C32609D4D7C
:103200001B782B723046F7F709FBA8833046F7F797
:1032100005FB28833046F7F701FB32686883531CAF
:1032200033601278EA747268D31A032B00F38E822B
:103230003368D11A052900F37982D21A002A7EF761
:10324000AAAC5A1C32601B7885F8213001252B4628
:10325000FEF788BC5A1C326093F80080B8F1110F59
:103260003FF6E1AA9A1C3260844D5B7805F818306D
:103270003046F7F7D3FA40F6CA039842A8BF18467B
:1032800040F2EE23984205EB4801B8BF18460125ED
:10329000A0F2EE222B46192092FBF0F24A70FEF7C4
:1032A00061BC1A46591C764D316012F8021B297117
:1032B00032605B786B713046F7F7B0FA336828807C
:1032C0005A1C32601B78AB713046F7F7A7FA3368A7
:1032D00068805A1C32601B78EB7101252B46FEF783
:1032E00041BC684A1278012A3EF655AC18465A1C71
:1032F0003260DFF8B08110F8022B88F80220DA1C67
:10330000891A306001295878326040F302823046D1
:10331000F7F784FA0125A8F800002B46FEF722BC37
:103320000125F7F7D1FF2B46FEF71CBC5A1C326073
:10333000554A1B78DFF8708113700023C8F80030FD
:103340003046F7F753FA3368D8F8002049494F4D13
:1033500010435A1CC8F8000032601B780B723046CC
:10336000F7F75CFA28603046F7F758FA686030469D
:10337000F7F754FAA8603046F7F750FA3046F7F7F7
:103380004DFAFEF708BC336872689A4240F0E2805A
:103390003F4BFF221A704FF0000A3E4D08F0B8FE76
:1033A000514620223C4885F800A02BF0DAFC87F833
:1033B0002CA097F82C30072B00F21081DFF8EC904E
:1033C000354E524697F82C3003EB430309EBC30309
:1033D0005B7CE3B197F82C3003EB430309EBC303A9
:1033E00020215B699BB197F82C3003EB430309EB79
:1033F000C303586946F82200F6F77AFA2B7856F894
:103400002300F6F7C9FB2A780132D2B22A7097F866
:103410002C300133DBB287F82C3097F82C30072B97
:10342000D0D92368591C21601A70B8F1000F3EF4FE
:10343000B2AB1A4BC8F8003001252B46FEF792BB01
:10344000174B3A6A9B68D4F800905A449A4200F2AB
:10345000B480F7F7D7FE5A464946386AF7F752FF65
:1034600023680344236086427EF795AB002120E069
:1034700064400020F0610020086B002088AD00202F
:103480005C420020EF7A0020488B0020B43D0020F1
:10349000C0220020BBAD0020BCAC00205984030832
:1034A000040F0020F27A00200C7B0020645C0020D6
:1034B000236801305A1CB04222601970F8D1FEF71F
:1034C0006ABB002DBCD159462046F7F701FA2368A4
:1034D0005A1C22601D70AD4B26689D683B6A0BEB41
:1034E0000302954280F0AB803B6AED1AF7F78AFE43
:1034F0002A463146386AF7F705FF236803442360FC
:10350000FEF749BB3046F7F789F9326871687B6A84
:103510009142834647D106461D46FEF726BE3046F9
:10352000F7F77CF9DFF89C82FEF7F2BE9A1C326056
:10353000974A59781170D91C316099785170191DCA
:103540003160DB789370FEF726BB924B93E8420024
:10355000FEF75CBD5A1C194632608F4811F8022BE9
:10356000027031605B784370042A03D9FF2A7EF42D
:10357000BEAA10E789490978994205D8022A7EF443
:10358000B6AAFF2B7EF4B3AA236801255A1922603C
:103590001D70B8F1000F3EF4FEAA814BC8F8003050
:1035A0002B46FEF7DFBA511C316012781D46131C02
:1035B000064618BF0123FEF7D8BD3A6AA3EB0208FE
:1035C000F7F720FE42464946386AF7F79BFE236824
:1035D00003442360002D3EF4DEAA44E7524620E770
:1035E00007F12C0948461DF02FFFBB8DAB423FF47D
:1035F00072AC6C4B1B68002B3FF46DAC1B689B6975
:10360000002B3FF468AC2846984764E4DA46C7F8D4
:1036100024B0FEF741BE7D62AA46FEF73DBE0A78A1
:1036200002F0FD02FFF7ABBA5F486049604A614BA8
:10363000036001250B6013602B46FEF793BAF7F782
:10364000E1FD5A463146386AF7F75CFE23680125EA
:10365000034423602B46FEF785BA3046F7F7DEF8C1
:10366000A8F80E003046F7F7D9F833687268A8F862
:103670001000FFF7AFBB012525F0AAFC2B46FEF793
:1036800071BA3046F7F7CAF8A8F80A003046F7F7DB
:10369000C5F8A8F80C003046D5F80090F7F7BEF84A
:1036A000A9F822003046D5F80090F7F7B7F833684C
:1036B0007268A9F82400FFF789BB364B1020C3F8C5
:1036C00000905D6027F034FE3B4A137843F001031D
:1036D0001370B8F1000F3EF45EAA384B0125C3F811
:1036E00000802B46FEF73EBA00F07F00032828BF7B
:1036F0000020012508F0F4FF2B46FEF733BA5A1CD0
:1037000032601B78003318BF012388F80730FFF7B9
:10371000A5BB2B4A99781288012512FB00F22B4693
:1037200092FBF1F2A8F80020FEF71CBA5A1C326096
:103730001B78EB723046F7F759F83368E8605A1C8B
:1037400032601B782B743368726876E53046F7F781
:1037500065F8A8843046F7F761F833687268E88442
:10376000D11A03297FF765AD1A46591C316012F84A
:10377000021BA97732605B7885F820303046F7F776
:103780004DF833687268688453E500BF040F002069
:10379000C179002024440020C0220020E56E0020D2
:1037A0005DC700081C790020CCAF002020B00020AD
:1037B00020B40020E986000824720020284300205D
:1037C000BE8900209C4300202DE9F04F724B734AC4
:1037D0001C7893B000F59C4120318146079111601F
:1037E000002C00F027856E4A1268904240F2278232
:1037F0006C4A6D491768DFF8E8B10492013C1C700F
:103800006A4C039107F48057002F40F02582039BF8
:103810005B7D002B40F09B84049B1B681D0400F122
:103820007787634B9945A37800F27383002B40F0B0
:103830007383604B0693049B1F6817F4805940F014
:10384000FA83039BBBF906605B8B9E42B4BF0026E4
:103850000126594B1B6813F0805300F00782069A2B
:10386000127812F0010200F0088203985349408C4C
:1038700091ED037A07EE900AF8EEE77AB4EEE77A74
:10388000F1EE10FA81F20A80002E40F0FD814C4DDD
:1038900095F8A010002940F0F7814A484A49056888
:1038A00095F82D5000200860486088604749002D39
:1038B00040F0EB810D70002A40F0EC81444B1A7807
:1038C000002A50D10399BBF900E04F8B898BBBF9DB
:1038D0000200BE45CCBF8025002545F040038E4543
:1038E000A8BF2B469B0843F08005B842C8BF2B46B3
:1038F00043F040058842A8BF1D46BBF904E0BBF970
:103900000600AD0845F08003BE45C8BF1D4645F022
:1039100040038E45A8BF2B469B0843F0800E284DE0
:10392000B842C8BF734643F0400E95F8A270884273
:10393000B8BF73469F4201F04081A5F8A42085F8E6
:10394000A620244985F8A2300F78002F01F0B1801D
:103950005F2B01F018816F2B00F0F887069B1B7816
:10396000D90740F1BA87049B1B4A1B68059203F0F4
:103970000403002B40F04A850DF14008174D002349
:10398000C8F8043005F15009109340F6330A19279E
:1039900040F2833629E000BFA87800204874002058
:1039A000A478002078600020F0610020446C0020A2
:1039B000404B4C00F1B50020AC890020D46F0020B2
:1039C000C4220020E8780020108900203025002043
:1039D000B1AA002048010020207200204C8B00205A
:1039E000C05B002004354D4520D0AA78EB789A4280
:1039F00017FB0261F6D26A78043217FB03633BF9C6
:103A000012205245A8BF5246B2F5617FB8BF4FF4AD
:103A100061729142E6DA9A42E4DC29782429E1D8FD
:103A200040460435F7F79AFA4D45DED1B04B98E899
:103A300003001F78AF4B83E80300002F00F03C84A5
:103A40000121AC48F7F79AFA002840F09A81E37810
:103A5000002B40F09681A84C23881DB225F001056B
:103A6000AEB2B342268000F0B286A44D02270E20EB
:103A70004FF014094FF0FF082F7085F8019085F87A
:103A8000028027F025FB39469A482688F7F776FA10
:103A9000002841F0458026F002039BB2B342238008
:103AA0000AD0964B1421FF2202250E201D7059705A
:103AB0009A7027F00DFB2688DFF884A2904B9AF8C5
:103AC000001058680393B50708BF81F00201C1F3E5
:103AD0004001F6F767F824218648F7F74FFA30B926
:103AE000069A1378590744BF23F004031370059B0B
:103AF0001B6813F00A0F1DD005217E48F7F73EFA28
:103B0000002800F0988625886F0740F1B58779482E
:103B10000621F7F733FA002800F07A866E0640F1A6
:103B2000888707217348F7F729FA002840F0308387
:103B3000059B1B689D0600F13B8327886D480C217F
:103B4000F7F71CFA002800F0388147F48073BB4275
:103B5000238009D0694B02251421FF220E201D70FD
:103B600059709A7027F0B4FA664B1B78082B00F056
:103B700030810E2B00F02D81049B1B685E0544D51F
:103B8000614B1B79002B00F0E18014215948F7F7B5
:103B9000F5F9002840F0DF8018F0B8F9012007F0AF
:103BA00085FE90B3DFF89C8100254FF0CC0902E040
:103BB000DDB2022D29D809FB05F76B1C58F8076008
:103BC000002EF5D1C378514A90F9020052F8233003
:103BD0000196032200920121324606F0CFFD0346F2
:103BE00005EB450000EB0010049353B1314608EBA0
:103BF0008000CC222BF0B5F8049B48F80730013543
:103C0000EDB221F009FF0028D3D1069B1B78DD0718
:103C100040F1F2803E493F4A01230B701370039B31
:103C20009AF80010186801F00101F5F7BBFF059B39
:103C30001B685A0700F1508113B0BDE8F08F364B76
:103C4000364A1F68049307F480570392DFF8F8B0F0
:103C5000334C002F3FF4DBAD00212648F7F78EF9F7
:103C600000287FF4D4AD0AF0ABFED0E578023FF532
:103C7000F6AD069A127802F001022A4D002185F86D
:103C8000A010002E3FF409AE274901200870002A39
:103C90003FF414AEF9067FF511AE244A1278D2062D
:103CA0003FF50CAEB9F1000F7FF408AE002B7FF4A6
:103CB00005AE7B023FF502AE1D4B1B78002B01F0D9
:103CC00021841C4B9B78002E41F059843BB11A4A49
:103CD0001A4B12681B689B1A002BC1F28B841020B0
:103CE000104D27F0F5F9012385F8A130E6E500BF76
:103CF000EC460020AC8900203A6C0020784200207D
:103D0000DC950020488B0020C46F00208818040830
:103D1000F2B500203C43002078600020F0610020D4
:103D2000446C0020C4220020302500202472002092
:103D300048010020F042002010960020B03E0020F4
:103D4000D895002000580020C05B0020069B1B78FF
:103D5000D8077FF521AF3C2014F01EFA00283FF46D
:103D600054AF06F0F3FC3C2017F03EF800283FF477
:103D70004CAF06F0EBFC3C2017F036F80028F0D1F1
:103D800043E7059B1B689A077FF565AEBF4C268805
:103D9000F3073FF580AE46F001039E4223803FF4D7
:103DA0007AAEBB4B1421FF2202250E201D705970E4
:103DB0009A7027F08DF926886DE627F480739BB200
:103DC000BB4223807FF4C6AEB24B1B78082B7FF436
:103DD000D0AE228822F040039BB29A4223803FF467
:103DE000CBAEAB4B02251421FF220E201D70597063
:103DF0009A7027F06DF9BFE6A74B93F80090B9F1E0
:103E0000000F5FD1DFF8E482A44F18F8030C3E786E
:103E10004146A8F103050FF027FE002800F0F083CB
:103E2000002E40F0428405F1080168790FF01CFE75
:103E3000002841F0E9819A49A87A0FF015FE002880
:103E400000F0F183022E41F0E3819649E87B0FF008
:103E50000BFE002841F0E0819349287D0FF004FE1D
:103E6000002800F0F183042E41F0DA818F49687E4A
:103E70000FF0FAFD002841F0D7818D49A87F0FF09F
:103E8000F3FD002800F0F183062E41F0B981894945
:103E900095F823000FF0E8FD002840F05887864988
:103EA00095F828000FF0E0FD002800F0F183082EBF
:103EB00040F03787814995F82D000FF0D5FD002897
:103EC00040F0F1837E4B01221A7010F050F8059BF0
:103ED0001B685A077FF5B0AE03200FF0EFFD0028F6
:103EE00000F06686238813F008047FF4A5AE08204E
:103EF00027F036FA7348744D7449754A754BBBF810
:103F0000066000682E80086014601C6013B0BDE875
:103F1000F08F0BB90123A3706F4B06931B201F7802
:103F200094F821600FF0CAFD012E07F001098246C6
:103F300000F0258607F00203059394F82030DFF89F
:103F4000B081664D052B69D8DFE813F05B004F00A8
:103F50000600DC00FF008D00012E04BF052384F85D
:103F60002030B9F1000F00F05281039B5C4FB3F990
:103F70001810B8F80030002261F30F0263F31F42FB
:103F8000002361F30F0361F31F43CBF8042039686A
:103F90006269CBF800308A42C0F06784012E41F09C
:103FA000FE82032294F820300592CBE70FF0B2FD99
:103FB000012807D14A4FB8F802303A68642101FB62
:103FC00003232361BAF1000F04D098F80630002BC8
:103FD00040F09080012E21D0414F22693B689A42E7
:103FE000C0F03186012384F82030012E3BD098F8B0
:103FF0000730012B00F014810EF028FC94F82030DB
:10400000A0E7B9F1000FD1D14FF48060BAF1000FF1
:1040100000F0FB8327F0A4F900232361059B002B0C
:104020003FF409AC059827F053F8049B1F6817F478
:1040300080593FF406AC1D212A48F6F79FFF00285F
:104040007FF4FFAB284A039BD2881B8BBBF9066029
:10405000991A8E4240F3018613449E42B4BF002653
:104060000126FFF7F6BB1E4F3A68B8F8023064210C
:1040700001FB03234FF480600022236184F8202099
:10408000E27027F055F994F820305BE73A6C002095
:1040900078420020488B0020F2B500209E000020CE
:1040A000584100205D41002062410020674100200E
:1040B0006C41002071410020764100207B410020AE
:1040C0003C430020F47100201C43002028430020C2
:1040D0002043002018430020F1B50020686C002028
:1040E00010960020AC890020404200204E41002064
:1040F0005C4200200EF0AAFB03224FF47A7384F88E
:104100002020E361A74F2B8843F002032B800AF0A5
:1041100057FC3A68E36913440422A36184F8202021
:10412000012E40F09D853B68A2699A42BFF476AFAC
:104130009D4B187820B90FF0C1FC00287FF46EAFBA
:104140002B8823F002032B808EE7964FE8E7039A33
:10415000013BD27D3BF91330002A40F08183A3F567
:104160007A73B3F57A7FA8BF4FF47A7323EAE373C7
:1041700007EE903A9FED8D7AF8EEE77A67EE877A50
:104180008B4AFCEEE77A17EE903A1380FFF749BBB3
:10419000884B894AB3F90430884982FB0302DB1754
:1041A000C3EBA202059B0A801B689D067FF5C5AC88
:1041B000834B1B78980704D5824E337D042B00F285
:1041C0005585278817F0300F3FF4B8AC102027F042
:1041D000AFF8202027F0ACF87B4B278800221A701C
:1041E0007A4A7B487B4E7C4D002111607B4A3160CE
:1041F0000023296041608161036083604361C36182
:1042000013605160936053619161D36196E4654F8F
:104210003B6847F230520323E26184F8203072E7B2
:104220000EF014FB032240F6B83384F82020E3613B
:104230005C4F68E76A4F3B78002B00F09887694B2A
:10424000DFF8B481DFF8B4B1DFF8B4A103934546D9
:104250005E46049099460EE019F804109847032C26
:1042600028DC88B93B782AF8020F01349C4205F11A
:10427000040580F2EF80072CE1B23046DBF8043011
:10428000EADD984700B2EDE738F824206B88801A01
:104290004FF47A719B1A01FB00F040F6CA0290FBC2
:1042A000F3F00844904240F2EE23A8BF1046984233
:1042B000B8BF184600B2D5E7DFF848A1DFF848815B
:1042C000494D0AF15A064FF0010951461AF8010CFE
:1042D0000FF0CAFBF8B19AF804009AF802309AF885
:1042E00003E000EB400105EB8101013BD1F8B42074
:1042F00003EB4303434493420DD095F8E02081F84B
:10430000B0E009FA00F022EA0000C1F8B430C1F8C8
:10431000B87085F8E0000AF1060A5645D5D1334950
:10432000204A334B334D09681B78D2F8009008912E
:104330000793A5F1B00A00266B685BB31F784FB3F3
:10434000AA68A9EB0202002A0ADB9AF8E020012100
:10435000B14022EA010209F5FA718AF8E020A96069
:10436000079ABAB12A7859780432D2B2002940F0BB
:104370009B8203993BF91220098B01F1C80082420C
:1043800040F333849AF8E0109A7841FA06F3D8079C
:1043900040F1C2840136042E05F10C05CCD1FFF7A3
:1043A0004FBB00BF1096002048010020AAF1823FB9
:1043B000386C0020F87100206766666610430020A4
:1043C0002472002028720020E2430020D8440020FC
:1043D000884400200425002098430020B044002099
:1043E0003CAD0020F0610020C4220020CC4200201F
:1043F000056C00207423002054AD002010790020AB
:10440000C22200206540002070F40308A84D95F8F2
:10441000AA3053B1069B1B78DE0706D5039BBBF978
:1044200006205B8B9A4200F34D841121A148F6F7D8
:10443000A5FD002800F0208295F8AE302BB995F844
:10444000A83013B93223A5F8AC30012385F8AE307B
:10445000FFF792BADDF81090974A04921146974AF6
:104460000968A2FB092A42F201020A404FEA9A1A9D
:10447000059200F0FD81924D9248934C934A95F835
:1044800000E0007884F800E01070BEF1000F04D066
:104490008E4A92F800E08EF0010E854D0F2085F8CF
:1044A0002400002B00F01283894B039E0C931B7891
:1044B000B6F826C00B931C463B78B78C039E854A02
:1044C000368B0E962646A2FB0442520802EB4202AD
:1044D000B21AD2B2CDF824C001F48051089295F8F6
:1044E0002580DFF808B2DFF824C20A900AF5967238
:1044F00076460F9105F1280400200692CDF83490FD
:10450000AE46002E00F037823EF910201FFA82F9E5
:10451000B9454FEA400103D3099DA94540F26F8296
:104520005CF82020924580F02F823BF90120059D08
:10453000002D40F04382013098422BF8012004F115
:104540000604DEDB0A98644ADDF834908EF8258094
:104550000F280CBF012100218EF82400117000F0FB
:10456000BC825E4C5E4E5F4F35883868A1686268D9
:10457000E06045F00405401A9042524F3580534D9B
:104580004FF0010188BF00223970297088BF84F87C
:104590002120002B00F0B382049A03991768524E31
:1045A000B1F824C0B1F818E0504817F480573546E8
:1045B00040F0C78239460EE06A7802EB820202EBD5
:1045C000820202F2EE2292B201318B4220F8022BDB
:1045D00005F102050ED016F81120002A00F0138212
:1045E000022AE9D00131028820F8022B8B4205F122
:1045F0000205F0D10C9A137801331370FFF704B958
:1046000008F1050168790FF02FFA00283FF413AC88
:10461000012E40F0F98505F10D01A87A0FF024FA7A
:10462000002840F0F5853249E87B0FF01DFA00289C
:104630003FF412AC032E40F0EF852E49287D0FF099
:1046400013FA002840F0EC852B49687E0FF00CFA35
:1046500000283FF412AC052E40F0E6852749A87FDC
:104660000FF002FA002840F0CB85254995F8230089
:104670000FF0FAF900283FF412AC072E40F06783E0
:10468000204995F828000FF0EFF9002840F0498301
:104690001D4995F82D000FF0E7F900283FF412AC02
:1046A000092E3FF40FAC4FF009094B463CE300BF25
:1046B000C4220020AC89002078600020D34D621015
:1046C00024740020E4060020056C0020E50600208C
:1046D000E9AC0020ABAAAAAA22470020446C002023
:1046E000686C00201096002088AD0020C05B002080
:1046F0005D41002062410020674100206C410020A4
:1047000071410020764100207B410020ECAC00206C
:10471000CC4DD5F88830A9EB0303002BFFF681A818
:10472000C94A95F88C30517C079AC5F88820013326
:10473000C64A039E32F81120B17D03F00F0385F8BD
:104740008C302B4492B292FBF1F283F8902095F8D2
:10475000901095F8912095F8923095F89C000A44B5
:1047600095F89310134495F89420194495F89530D2
:104770000A4495F89610134495F89720194495F833
:1047800098300A4495F89910134495F89A201944E2
:1047900095F89B300A44134495F89D1095F89F2096
:1047A000184495F89E3001440B441A4442F30B120E
:1047B000642AF17DA8BF642213B209B1C2F1640377
:1047C00007EE903A9FEDA27AF8EEE77AD6E402215E
:1047D000A048F6F7D3FB00283FF45DA92580B70772
:1047E0003FF56AA946F00203B34223803FF464A96F
:1047F000994B02201421FF2218700E2059709A70D4
:1048000026F066FC2688FFF757B926F091FD03E4F1
:1048100025F040039BB2AB4223803FF482A98E4B2C
:1048200002251421FF220E201D7059709A7026F067
:104830004FFCFFF776B9238823F00405ADB2AB42F5
:1048400025803FF464A9844B02251421FF220E2009
:104850001D7059709A7026F03BFC2588FFF757B9F8
:10486000C3F53B6308331BB279E403230593D0E41B
:104870007A4A92F800E008E695F8A830002B3FF459
:104880007BA8069B1B7813F001037FF475A8012217
:1048900085F8A83085F8A920FFF76EB8694D012189
:1048A00085F8A010FFF7F0B9012900F002849AF80A
:1048B000E0200123B34001361343042E8AF8E03090
:1048C00005F10C057FF438ADFFF7BAB8069B644AD2
:1048D0001B781060DF0700F1038295F8A61000290D
:1048E0007FF441A8B5F9A430322B7FF73CA895F8A6
:1048F000A2200120572A85F8A60000F09984049B85
:104900001B6813F0040302D05A2A00F0E8855D2AE0
:1049100000F0E6845B2A00F026855E2A00F06C85B4
:10492000562A00F0CD85972A00F08785A72A40F007
:104930009E844C49049B0A781B6842F004020A706A
:10494000494A059203F00403FFF713B8B2F5FA7F62
:10495000FFF609A895F8A620002A7FF404A8069B74
:104960001B780121D80785F8A61000F1C48409F04E
:10497000B9F9FEF7F8BF002F3FD05CF82020924530
:104980004FEA4001FFF4D1AD384A384D525C05EB97
:104990000109002A00F0B880022A47D199F80120C5
:1049A00002EB820202EB820202F2EE2292B20328B2
:1049B00033DD059D12B2002D3FF4BDAD089D24F8F6
:1049C0001520B8F1000F03D10B9D022D7FF6B3AD7A
:1049D0002288B4F80290B4F804804A449044244AEF
:1049E0000FFA88F882FB0852224DA2EBE87225F8F4
:1049F000018012B24FF001089DE53A464100069D44
:104A00004CF8205093E5CAB2022A04D9032A7FF455
:104A1000E9AD6246D8E57246D6E5012505FA00F90A
:104A20000A9D25EA090512B20A9580E53BF80120A6
:104A3000BDE745F04003AB4223807FF4F0AEFFF7C3
:104A400070B800BFC4220020609600207C96002031
:104A500014AE2341AC89002078420020056C002070
:104A6000B43E0020247200202072002088AD002077
:104A7000565555553423002045F004039D422380AC
:104A80000AD0B54B02251421FF220E201D7059704B
:104A90009A7026F01DFB2588B04BB14AB3F904305B
:104AA000B04982FB0302DB17C3EBA2030B80FFF7C5
:104AB0002EB83946AC48F6F761FA00283FF406AF45
:104AC00085F8A77009F00EF9FEF748BFA749A84A74
:104AD0000C91DFF8C0B2012111701B21A24805938F
:104AE000F6F74CFA059B00287FF43BADA14CA24F92
:104AF000E2683B68A3609B1AC82B00F25A83049BB0
:104B00001F6807F4805775E5C2B2022A40F2CF82CF
:104B1000032A8BD10E9A0F9D002D08BF3A4646E717
:104B200026F001039BB2B34223803FF458AE0E201F
:104B30002F7085F8019085F8028026F0C9FA268842
:104B40004DE600210FE06A7802EB820202EB82025E
:104B500002F2EE2292B20131994220F8022B05F1C5
:104B600002053FF447AD16F811201AB1022AEAD027
:104B70000288F0E7CAB2032AFAD87246EBE70023AC
:104B80000593FFF7DAB9B2F5FA7FFEF6ECAE95F8C9
:104B9000A630002B7EF4E7AE069B1B7801210B406C
:104BA00085F8A61000F0E78209F00AFFFEF7DBBEE9
:104BB000082026F0BDFBFFF73FB8704A7049106827
:104BC000B5F9A420C76981FB07018911FF17781A7D
:104BD00000F5FF407F3082423EF7B3AEC91B0A4466
:104BE00012B2A5F8A420FEF7ACBEC8398A425CDA3E
:104BF0009AF8E0109A7841FA06F3D9073FF5CAAB64
:104C000052420120099226F07BFB7B1E099A162B4B
:104C100000F24281DFE813F0E301F901CA01220248
:104C20000F0236029D01880171015A0143014001C2
:104C30002202300136029D0188011A010401EE00B2
:104C4000B201D600C0000DF001FE032240F6B833D9
:104C500084F82020E361FFF756BA0126FEF7F9BD7C
:104C60003A68E3691344A361FFF7D8B90A200EF04C
:104C700025FF27888046002800F05882F90640F179
:104C80004483404D95F8F080B8F1000F7EF456AFA4
:104C90000D2026F01DFA012385F8F0302788B8F1A1
:104CA000000F7FF49DAAFEF749BF9AF8E030012279
:104CB000B24023EA020309F5FA728AF8E030AA60EA
:104CC000FFF768BB00212848F6F758F900287FF461
:104CD000ACAB322385F8AA00A5F8AC30FFF7A5BB32
:104CE000294B1B78002B3EF43EAEE378002B7EF47C
:104CF0003AAE95F8A7300133DBB2032B85F8A73025
:104D00007EF631AE214B5B7813B9002E7EF42BAECC
:104D100009F056FEFEF722BE002A0CBF0120022039
:104D200070E74FF008094B4603EB83031D4487F8F7
:104D30000090A97868781CF0B7FB069B144A1B7892
:104D400001211170D9077FF5C0A8FEF768BF4FF0A9
:104D500007094B46E8E700BF78420020F8710020C1
:104D600067666666F8440020AC890020E9AC002044
:104D700022470020446C002010960020BC6E0020CA
:104D8000D34D6210C4220020056C0020F0420020A8
:104D90003C430020C05B0020DAF8E400DFF81C8709
:104DA00090F8361098F8023011446429A8BF6421A5
:104DB00021EAE17180F83610002B40F04B8424F09A
:104DC00097FA74E5DAF8E400DFF8F08690F8371027
:104DD00098F802301144FE29A8BFFE2121EAE171B2
:104DE00080F83710002BEAD016200EF0C5FEDAF856
:104DF000E400E4E7DAF8E400DFF8C08681781144E3
:104E0000C829A8BFC82121EAE171817098F8023051
:104E1000002BD4D014200EF0AFFEDAF8E400CEE779
:104E2000DAF8E400DFF8948641781144C829A8BF75
:104E3000C82121EAE171417098F80230002BBED000
:104E400013200EF099FEDAF8E400B8E7DAF8E4008F
:104E5000DFF8688601781144C829A8BFC82121EA73
:104E6000E171017098F80230002BA8D012200EF0EA
:104E700083FEDAF8E400A2E7DFF84086089898F8A5
:104E80000230417911446429A8BF642121EAE1710B
:104E90004171002B40F09383DAF8E4008FE7DAF8F1
:104EA000E400DFF81886017A98F802301144C82926
:104EB000A8BFC82121EAE1710172002B3FF47FAF46
:104EC0000B200EF059FEDAF8E40078E7DAF8E40097
:104ED000DFF8E885C17998F802301144C829A8BFE5
:104EE000C82121EAE171C171002B3FF468AF0A20AB
:104EF0000EF042FEDAF8E40061E7DAF8E400DFF8E9
:104F0000BC85817998F802301144C829A8BFC8210E
:104F100021EAE1718171002B3FF451AF09200EF0BD
:104F20002BFEDAF8E4004AE7DAF8E400DFF88C85D3
:104F3000417998F802301144C829A8BFC82121EA54
:104F4000E1714171002B40F04183112F7FF456AF86
:104F500035E7DAF8E400DFF86485017998F8023083
:104F60001144C829A8BFC82121EAE1710171002BB1
:104F700040F07483102F7FF457AF20E70898DFF8D4
:104F80003C8541781144B1F5967FA8BF4FF49671E6
:104F900021EAE171417098F80230002B3FF47CAFB8
:104FA00015200EF0E9FDDAF8E40008E70899DFF8CB
:104FB0000C850F791744642FA8BF642727EAE77789
:104FC0000F710EF0F3FD98F80230002B3FF464AF40
:104FD000032039460EF0D0FDDAF8E400EFE6089839
:104FE000DFF8D88401781144FA29A8BFFA2121EA10
:104FF000E171017098F80230002B3FF44DAF0120B1
:105000000EF0BAFDDAF8E400D9E60898DFF8AC84CF
:10501000817811446429A8BF642121EAE17181707B
:1050200098F80230002B3FF437AF02200EF0A4FDB9
:10503000DAF8E400C3E60898DFF88084C17998F8CC
:105040000230114481F30801C171002B3FF424AFF9
:1050500005200EF091FDDAF8E400B0E6089BDFF8D9
:105060005C84997998F8020011446429A8BF6421EE
:1050700021EAE1719971002840F0B0820D2F7FF490
:10508000FDAE09E7DAF8E400DFF83084C17898F87B
:1050900002301144C829A8BFC82121EAE171C170BA
:1050A000002B40F084820F2F7FF4D4AE87E60E9A57
:1050B0007DE43BF912209978B2F5617F4FF4966355
:1050C00093FBF1F34ADB40F633019142A8BF11464E
:1050D0000C2FA1F5617191FBF3F100F08381182F82
:1050E0007FF4E5ABC9B2C8290B46A8BFC823DAF8DC
:1050F000E400C27DDFB297423FF4D9AB9A1ADFF8E1
:10510000BC83C77548BF0732D71098F80230013703
:10511000FFB23BB9002F3FF4CAAB384626F0F0F897
:10512000FFF7C5BB18200EF027FDF3E7FA0600F1E4
:105130004F810B200EF0C2FC002840F01881BB0606
:1051400000F15281C34D95F8F030002B3FF4A0AD33
:10515000B8F1000F7FF444A8FEF7F0BC0C2F00F06C
:10516000EA80182F7FF4A3AB00210B46BFE7BA4AB1
:105170000392FFF771B9B949096811F4003140F0A1
:105180003F810B46B648C65C0F2E03F10C031ED0C0
:1051900001311529F7D1049BB2491B680591FA3AF0
:1051A000A5F8A420002203F0040385F8A620FEF74A
:1051B000E0BBAD4A049B1F68138823F004031380EF
:1051C000012307F4805784F82130FFF713BAA74E64
:1051D000D6F800E04B00BEF1000F07D05F1800EBDF
:1051E00087079EF801E07F787745D4D20B44A04F23
:1051F000A04900EB8300002330603B800B60CAE7CE
:105200004FF006094B468FE54FF001094B468BE501
:105210004FF002094B4687E54FF003094B4683E503
:105220004FF004094B467FE54FF005094B467BE5FF
:10523000914B92491A684FF47A73B3FBF2F3C3EBC4
:10524000431203EB8203049A1268DB001206A1F8F2
:10525000B43000F1E580834B05931B685F0700F1D4
:10526000D680049B1B6803F00403FEF782BB002179
:10527000BB2A109100F08081B72A00F07981BE2A04
:1052800000F07481BD2A00F04D81792A00F0DB81A5
:105290007A2A00F0D1819E2A00F0C8819D2A00F070
:1052A000BE81AE2A00F00182AD2A00F0F781EF2A1C
:1052B00000F0EE81FD2A00F0E581FB2A00F0DC81A0
:1052C000FE2A00F0D381F72A00F08E817B2A7EF43B
:1052D0004AAB4FF4FA61022007F028F9FEF743BB0E
:1052E000674B00220120674D67492A700B6026F04A
:1052F00007F8FEF738BB049B64491B680A60594AEB
:10530000059203F00403FEF734BB102026F028F8C2
:10531000202026F00DF85E494E4D081F1BF0CAFFF5
:105320005C4B02221A7095F8F030002B00F03B81A4
:105330002788FEF755BF00273946524B09915B7805
:10534000BB423FF4B4AADFF87481384607F0C8F9CD
:1053500098F8023009991BB1C9B20C200EF00CFC70
:105360000137FFB2D6E64C4B01220220BBE74B4A85
:105370004B4B528993ED007A07EE902AF8EEE77ACC
:10538000B0EEC77AB4EEE77AF1EE10FA7FF5D7AE59
:1053900093ED017AB0EEC77AF4EEC77AF1EE10FA27
:1053A0007FF7CDAEBB063FF5CDAE2A4D202025F0D0
:1053B000D7FF29467268336841F8EC2F05F1E80001
:1053C000C5F8E8301BF076FF324B01221A70AAE7CD
:1053D000102025F0ADFF2F4B278883F800804FF079
:1053E0000108A6E6CFB2A8E7202025F0A1FF294BAF
:1053F000184D00221A7096E72A4B0222032072E70A
:1054000029490978032900F0C5801946BAE6049BAA
:10541000264A1B680A21118003F00403FEF7A9BA8B
:10542000234B1B789B077FF516AF224B1B7D042B6C
:105430007FF611AF1BF0C8FE0DE7049B1E4A1B68E8
:105440004FF4C8711180074A059203F00403FEF778
:1054500090BA00BFC4220020F06100205840002014
:10546000880B040820720020686C0020DC240020D7
:105470007A2500207C25002068600020688C0020B0
:10548000D6790020D9780020E8780020B43E0020AA
:1054900028440020E2430020247A00207C4400209D
:1054A000D46F0020727A0020406C0020EA42002075
:1054B0002472002028720020EC420020F27A0020A2
:1054C0001BF006F9F4F7A0FF1BF0EAF8F9F71CF956
:1054D000012025F015FF95F8A220FFF724BA95F8D2
:1054E000A820002A40F0938095F8AA3083F00103A9
:1054F00085F8AA30002B40F085800C2025F0E8FDCF
:10550000FEF731BA002E3EF4EAAB6B4D95F8A130B0
:10551000002B3EF4D3A925F0BFFD002385F8A13070
:10552000FEF7CCB94FF6FE73644A6548968905903C
:10553000D089334401449381D1811BF0C9F8F4F739
:1055400063FF1BF0ADF8F9F7DFF8012025F0D8FE76
:10555000049BB5F8A4201B68FA3A0021A5F8A42002
:1055600003F0040385F8A610FEF703BA0223DBE775
:105570000B464FF6FE71D7E70B460221D4E7002B0E
:10558000C3D05049504A09684FF47A7000FB0313A6
:105590001360BAE725F080FDB5F9A420FBE50323ED
:1055A0000593FEF73FBD4FF00108FFF771BB0F20D9
:1055B00009920EF0E1FADAF8E400099A73E50E2098
:1055C0000EF0DAFADAF8E400FFF7F9BB11200992DD
:1055D0000EF0D2FADAF8E400099AB6E40D20099246
:1055E0000EF0CAFA099A49E50021042006F09EFF50
:1055F000FEF7B9B9304D09F0E3F9002385F8A13081
:10560000FEF75CB90B2025F063FDFEF7ACB92C4A20
:1056100085F8A81085F8A9000592FEF7AAB900211F
:10562000FF2027F0D3F895F8A2203AE6012027F0D2
:10563000CDF895F8A22031E6244A137A43F001030D
:105640001372FEF790B9214A137A23F00103137203
:10565000FEF789B917200EF08FFA1DE41020099289
:105660000EF08AFADAF8E400099A83E400210320B4
:1056700006F05CFFFEF777B90021022006F056FF26
:10568000FEF771B90021012006F050FFFEF76BB95B
:105690000021084606F04AFFFEF765B9FF21002009
:1056A00027F094F895F8A22001E60121002027F0C8
:1056B0008DF895F8A220F7E5C42200209478002008
:1056C0002072002010960020B03E002008470020E5
:1056D0002DE9F0478C4B1B78DB07074644D58B4BF5
:1056E0008B4D1C788B4E012C59D01CD3022C07D12A
:1056F00089498A4A09881288914201D901241C707B
:10570000EB7AE3B12B89D3B1854B1B78BBB107F0A2
:1057100025FD002800F09B802B7B83422CBF0121BC
:10572000002131700CE07C497E4A098810886A7B30
:10573000801A8842E2DAEB7A0024002BE2D1317839
:105740002A79632A06D8022C774E00F0BA80337883
:10575000002B5DD1754AAB7A8C4238BF0C46147071
:10576000002B4CD1BDE8F0876B4B694D19885B88E5
:10577000E878CB1A83EAE3728142A2EBE3721DD38D
:105780002B788B421AD3614B1C78E01E012861D91B
:105790006749097802294FD0012C5E4EA5D15F4A96
:1057A0005D491288687B0988121A914239DD5D4A89
:1057B00012888A42A4D200241C70A1E7B1EB400FEA
:1057C000E1DC524B1C78E11E012940F29480022A50
:1057D000DEDC57494F4E0878DFF84481DFF844C1DA
:1057E000DFF838E100210324022834701C7088F8A7
:1057F0000010ACF80010AEF8001081D11FE0012CB1
:1058000071D0022C0BD10720BDE8F04725F060BC19
:105810007068381A474B984258DD72709AE7BDE8B5
:10582000F08702241C706BE7022AD2DD4049097818
:1058300002294FF0040464D13949364E09783E48B4
:10584000022ACCBF00220122C28081804BE70221C4
:10585000317075E7022A9BDC95F800C091FBFCFCD7
:105860000CF1010CBCF1080FDFF8B4A0304EA878A1
:1058700095F801E096F800802A4CDFF8A090254EBC
:10588000A8BF4FF0080C8AF800C01FFA8CFA10FB72
:105890000AF01EFB0AFE80B2DFF88CA02080A9F877
:1058A00000E000244FF0640EB8F1020F34701C7059
:1058B000CAF804408AF801E07FF439AF0FFA8CF19E
:1058C000BDE73078A0B9012377603370C2F164027C
:1058D0001A4B00FB02F083FB0023C017A0EBA35080
:1058E0006430707036E70820BDE8F04725F0F0BB63
:1058F0007368F81A8EE7032C96D10D4909780229AE
:105900009AD0044EFCE600BFF1B500204C2B0020DD
:1059100000720020522B0020BC6F0020502B002072
:10592000D26F00204E2B002008430020406C002046
:10593000046F00207F969800086F00206BCA5F6B91
:105940002DE9F04F2DED0A8B404B1B7893B0012BC6
:10595000039001F0C4803E4C94F80021002A41F0ED
:10596000CF80072B01F0D6804FF0000ADFF8ECB0B3
:10597000DBF8043058469847002800F06F81BBF8E8
:10598000B46000228BF85520002E40F06887BBF9E8
:105990003C50DBF82410BBF93E00DBF82820BBF9B3
:1059A0004030691ACBF830102A490191821ADBF88D
:1059B0002C00CBF834200D461B1A9BF85610CBF860
:1059C00038300BF130001AF03BFC2B68990040F1A5
:1059D000E980DBED0D5ADBED0C7A1F4A94ED416A4C
:1059E000D4ED426A94ED437AD4F810311268B8EEDF
:1059F000E58ADBED0E5AF8EEE77AF8EEE58A013338
:105A000077EE867A38EE268A78EE878A9342C4ED5E
:105A1000417A84ED428AC4ED438AC4F8103101F022
:105A2000FD820A4B1E78142E02F0B1840023D4F8B4
:105A300018510293062D00F2A880DFE815F0071335
:105A4000F6121B128B1211003114CA13046F0020BE
:105A5000B823002078600020EC740020688C0020BF
:105A6000D74B1A78D4F81C71DFF8BCE39FEDD57AD8
:105A7000F8000EEB000383ED007A002A7AD0D249B9
:105A8000B0EE476AF0EE476A0023F1EC017A013389
:105A900067EEA77A05EE903AB4EEE77AF1EE10FAE7
:105AA000F8EEE55AB8BFB0EE677A9A4276EEA76A8A
:105AB000A7EEA56AE9D1F5EEC06A0EEB0003F1EEA0
:105AC00010FA83ED007A55DDC6EE265ABF4BC04A68
:105AD0001288F7EE007A75EEE75AD3ED007A65EE9C
:105AE000A77AFDEEE77A17EE903A812B43F32783EE
:105AF0009342A8BF134607EE903AF8EEE77AB54B0B
:105B0000C11903EB810393ED057AD3ED003A93EDD0
:105B1000066A93ED014AD3ED046AD3ED034A93ED8F
:105B2000025AA3EEA77AA4EE276A66EEC76AA7EE2A
:105B3000646ABDEEC77AE5EE276A17EE101A81296E
:105B400083ED056AC3ED066A43F3F6828A42A8BF75
:105B50000A4607EE902AF8EEE77AFCEEE77ACDEDFA
:105B6000047ABDF810300EEB0002938017B9132EA3
:105B700003F0B687152E42F0CF817044DFF8AC8277
:105B8000838828F81730D4F81851934B013583FBDC
:105B900005235A19EB17C3EBA203C3EBC303ED1A9A
:105BA000C4F818518D4B1B78002B01F0EF808C4D01
:105BB000CDF808A0DFF87882DFF87092DDF804A055
:105BC00005F2DC670026874BDBED087A1B78172B84
:105BD00001F04E8495ED007AB8EEC78A082B28EEC6
:105BE000278A07D1B0EE480A019326F0ADFF019B4A
:105BF00029F81600DAF8002092000BD5002E04F0E8
:105C00000081B0EE480ADBF8783707F1700098475A
:105C1000B0EE408AB0EE480ADBF89836A7F1700083
:105C20009847DBF80837384698476E4B1B78032BAC
:105C3000B0EE408A01F0FB83D5F85C06DBF8B830A3
:105C4000B0EE480A98470136032E07F12407A8EC66
:105C5000010A05F10405B6D1DDF808A0614B1F78F3
:105C6000072F00F0BC8694F828310493002B40F0F5
:105C7000C4865D4B5B79002B40F0EB850123594ACC
:105C800084F828311278072A01F0848600230693CD
:105C9000564B94ED4C9A93ED007A554BDFF8948176
:105CA000D3F800A0534B0293F7EE007A37EEC9BA4F
:105CB00008F11C032BEE07BA0025B4EEE7BAF1EEAB
:105CC00010FA0593D4ED4BBA4B4BDFF86CB1DFED16
:105CD0004B8A9FED4BAADFED3BAADFED4A9ADFF836
:105CE0005C91494F019388BFB0EE67BA2E46474B8F
:105CF00098ED008A2B44D3ED007AF5EE407AF1EE70
:105D000010FA17D0424B2B44D3ED006A38EE667A76
:105D1000B0EEC76AF4EEC67AF1EE10FA08D5B5EE29
:105D2000C07AF1EE10FACCBF37EEA68A36EEE78ADB
:105D300083ED008A374B1A88930700F08180022E8A
:105D40007ED0354B9AF82E1033F9163007EE103A04
:105D5000059B07EE901A2B44F8EEE76AB8EEC77A77
:105D6000D3ED007A4B42A6EEA77A700007EE903A88
:105D7000F8EEE77AB4EEE77AF1EE10FA0AD407EE1D
:105D8000901AF8EE677AF4EEC77AF1EE10FA88BF4F
:105D9000F0EE477A214B22490344085EB3F90C30F8
:105DA000C01A07EE100AB8EEC77AD007E7EE687A95
:105DB00040F12B861B4B93ED008A27EE888A3FE04B
:105DC000F274002000000000B8230020F4740020CA
:105DD000F07400202877002093244992E574002075
:105DE000988C0020046F00205460002078B40020BC
:105DF000E87800206860002004890020CDCCCC3DEC
:105E0000AE47813F0000C842108900206CB40020DA
:105E1000F82400203A6C002004250020947800200B
:105E2000F871002054B4002010770020086F002083
:105E30006C600020EC240020C8AF00201C890020EA
:105E4000029B94F868212B44D3ED01CA38EE6CCA4A
:105E5000002A3DD0D34BD4F86C2103991B688A1AD1
:105E60009A4235DD9AF84830022B01F0CA85022E9D
:105E700003F06787CC4B1B68990740F16E87CB4BCB
:105E8000CB49DFF8A0E331F916C09EED008ADFF8B8
:105E900098E3C7ED00AA03EB460028EE288AB0F984
:105EA0000C00A0EB0C0007EE900AF8EEE77ADEF8A3
:105EB000000027EE888A904238EE6CCAC1F28380D7
:105EC000F7EE007AB4EEE79AF1EE10FA01F15280A3
:105ED000B84B2B4493ED000A019B2BEE800A022E57
:105EE00020EE0C0AA3EC010A019303F04487B24BA5
:105EF0009BED007AD3ED007AB04BD7ED006A93EDBD
:105F0000006AAF4B67EE277A2B4427EE8B7AD3EDEE
:105F1000007A67EE277AF0EE665AECEE275AB1EE79
:105F2000467AF4EEC75AF1EE10FA08D4F4EEC65AE7
:105F3000F1EE10FA8CBFB0EE467AB0EE657A94EDD1
:105F40004C6AF7EE007AB4EEE76AF1EE10FAACBFF5
:105F50000123002343B1F0EEE66AF0EEC77AF4EED7
:105F6000E67AF1EE10FA01D587ED007A022E03F001
:105F7000E186944A944B52F826001B68B0EE6C0AF6
:105F80009847924A924B52F826001B6898479AF815
:105F9000373023B18F4B1B88002B00F0C085B0EE4B
:105FA0006A8A8D4B9BED007A38EE400A2B4493EDC4
:105FB000008A83ED000A9AF8483030EE480AC0EEB5
:105FC000077A2BB3854B1B78DB0721D5B7EE007A18
:105FD000B4EEC79AF1EE10FA04DB94F86831002BA6
:105FE00000F06F87D4F86C31039AD31A6D4A1268A7
:105FF0009A420DDD7A4B93ED007AB0EECCCAB4EE46
:10600000C7CAF1EE10FA40F1FA87002384F868312C
:10601000744B94F878212B4493ED007A2BEE877A19
:1060200067EE277AC9ED007A32B9019BC7ED00AA65
:1060300043ED01AAC9ED00AA0136032E08F10408B8
:1060400009F1040907F1040705F104057FF44FAED7
:10605000654B1B78072B01F02182012B01F09F84F7
:106060000023029394F88031002B40F0A1855F4B10
:106070005F4A1B68126813F4805C92F82C2040F091
:10608000AE865C495C4891ED006A408B5B4984EDCB
:10609000646A91ED007A5A4984ED657A07EE900AB8
:1060A000F8EEE76AD1ED037A564984ED626A37EE7D
:1060B000467A77EEE67AD1ED006A84ED617A0121C5
:1060C00084F89811C7EEA65A4F48504990ED005AEF
:1060D0004F489FED506A90ED004A4F48DFED4F6A00
:1060E000D0ED004A91ED007A35EE045AF7EE007AD1
:1060F000F4EEE75A35EE245AF1EE10FA88BFF0EECE
:10610000675A25EE065AF4EEE65AB1EE476AF1EE0A
:1061100010FAB4EEC65AB8BFF0EE665AF1EE10FAB5
:10612000C4ED675A01F10780B4EEC75AF1EE10FAD8
:1061300088BFB0EE475A3449DFED366AD1ED017AB7
:10614000334991ED014A344977EE847AD1ED014A21
:1061500077EEA47A67EEA67AB4EEE76AF1EE10FA6B
:1061600008DCB4EEE77AF1EE10FA8CBFB0EE676AA5
:10617000B0EE476A2449DFED276AD1ED027A24495F
:10618000D1ED024A264977EEA47A91ED007A67EEC6
:10619000A67AB1EE473AF4EEC37AF1EE10FA4ED495
:1061A00044E000BF80B400202072002094780020DA
:1061B000F871002028B40020A00000209CB400202A
:1061C00034B40020D0AF0020CCAF002024B0002099
:1061D00020B000203A6C002028250020F1B50020D6
:1061E0008CB4002040B40020046F002078600020B0
:1061F000E8780020C4890020F061002034420020AB
:10620000D46F00204842002004890020A0B4002060
:10621000108900206F12833A1C89002000000000C2
:10622000A4B4002054B400207CB40020F4EEC77A5B
:10623000F1EE10FA8CBFB0EE473AB0EE673AED4996
:10624000497809B9B1EE433A002A41F04B82F7EEA2
:10625000003ADFF8C8B39BF80020002A02F045821C
:10626000E549DFEDE66AD1ED024A91ED017AD1ED23
:10627000037A66EE244AE5EE074AE3EE274A63EE28
:10628000A44AF4EEE64AF1EE10FAB4BFB0EE664A64
:10629000B0EE644A98BFF0EE646A012ACDED0A4A76
:1062A00002F0448291ED067AD1ED052AD1ED077A0C
:1062B00026EE077AA5EE227AA3EE277A23EE877AD6
:1062C000B4EEE67AF1EE10FAB4EEC47A8CBFF0EEDA
:1062D000667AF0EE477AF1EE10FA98BFF0EE676A50
:1062E000B4BFF0EE447AF0EE477A022A8DED0B7AD5
:1062F00000F0DE8091ED0A7AD1ED092A91ED0B4A8A
:1063000026EE077AA5EE227AA3EE047A23EE877AA8
:10631000B4EEE67AF1EE10FAB4EEE77A8CBFB0EEA6
:10632000664AB0EE474AF1EE10FA98BFF0EE446AC2
:10633000A8BFF0EE477A032A8DED0C7A00F0B88002
:1063400091ED0E7AD1ED0D2A91ED0F4A26EE077AE6
:10635000A5EE227AA3EE047A23EE877AB4EEE67AEB
:10636000F1EE10FAB4EEE77A8CBFB0EE664AB0EE0A
:10637000474AF1EE10FA98BFF0EE446AA8BFF0EE7B
:10638000477A042A8DED0D7A00F0928091ED124A41
:10639000D1ED112A91ED137A26EE044AA5EE224A98
:1063A000A3EE074A23EE844AB4EEE64AF1EE10FA71
:1063B000B4EEE74A8CBFB0EE667AB0EE447AF1EE06
:1063C00010FA98BFF0EE476AA8BFF0EE447A052AAB
:1063D0008DED0E4A6CD091ED164AD1ED152A91ED56
:1063E000177A26EE044AA5EE224AA3EE074A23EEC8
:1063F000844AB4EEE64AF1EE10FAB4EEE74A8CBFF6
:10640000B0EE667AB0EE447AF1EE10FA98BFF0EE94
:10641000476AA8BFF0EE447A062A8DED0F4A47D0AE
:1064200091ED1A4AD1ED192A91ED1B7A26EE044A14
:10643000A5EE224AA3EE074A23EE844AB4EEE64ACA
:10644000F1EE10FAB4EEE74A8CBFB0EE667AB0EE29
:10645000447AF1EE10FA98BFF0EE476AA8BFF0EE6A
:10646000447A072A8DED104A22D091ED1E7AD1EDA3
:106470001D2A91ED1F4A26EE077AA5EE227AA4EE98
:10648000037A27EE237AB4EEE67AF1EE10FAB4EE50
:10649000E77A8CBFB0EE666AB0EE476AF1EE10FAAA
:1064A0008DED117A98BFF0EE466AA8BFF0EE477AFC
:1064B00077EEE67AF7EE006AF4EEE67AF1EE10FA9D
:1064C000C4ED4C7A43F3A88286EEA77A022ADDED6A
:1064D0000B7A67EE244A67EE877ACDED0A4ACDED56
:1064E0000B7A2DD0DDED0C7A67EE877A032ACDED9D
:1064F0000C7A25D0DDED0D7A67EE877A042ACDED92
:106500000D7A1DD0DDED0E7A67EE877A052ACDED86
:106510000E7A15D0DDED0F7A67EE877A062ACDED7B
:106520000F7A0DD0DDED107A67EE877A072ACDED70
:10653000107A05D0DDED117A27EE877A8DED117A8C
:106540002F49096811F0805800F0A387F6EE005A31
:10655000C4ED675A002A02F0BF8094F99801D4ED87
:10656000654A284D284994ED646A284E284FDFF883
:10657000B0E0B5F81AA0C978B6F9069097ED005AC0
:106580009EF800E0D4ED616AD4ED627A07EE100A5D
:10659000FDEEE44A1F4814EE905A0078FDEEC64A1C
:1065A00003F0100603F4800300F00107B8EEC77A89
:1065B00014EE900A0193002941F0D4800E49002E78
:1065C00040F0898791ED006A9DED0A5A124B25EE45
:1065D000866AA5EE076AB0EE675AA6EE265ABDEEA9
:1065E000C56A16EE10EA16EE106AAE45A8BF2E4632
:1065F00018E000BF488B0020B441002000000000DC
:10660000AC890020F0610020446C0020C05B0020B9
:1066100090410020F1B5002064890020E56E002043
:10662000485D00207045C8BF064606EE106AB8EE09
:10663000C66A012A83ED006A00F0DC8091ED046AED
:106640009DED0B5A25EE866AA5EE076AB0EE675AF5
:10665000A6EE265ABDEEC56A16EE10EA16EE106AD0
:10666000AE45A8BF2E467045C8BF064606EE106A66
:10667000B8EEC66A022A83ED016A00F0BB8091ED94
:10668000086A9DED0C5A25EE866AA5EE076AB0EE03
:10669000675AA6EE265ABDEEC56A16EE10EA16EE49
:1066A000106AAE45A8BF2E467045C8BF064606EE26
:1066B000106AB8EEC66A032A83ED026A00F09A8077
:1066C00091ED0C6A9DED0D5A25EE866AA5EE076ADE
:1066D000B0EE675AA6EE265ABDEEC56A16EE10EA6F
:1066E00016EE106AAE45A8BF2E467045C8BF0646D6
:1066F00006EE106AB8EEC66A042A83ED036A79D002
:1067000091ED106A9DED0E5A25EE866AA5EE076A98
:10671000B0EE675AA6EE265ABDEEC56A16EE10EA2E
:1067200016EE106AAE45A8BF2E467045C8BF064695
:1067300006EE106AB8EEC66A052A83ED046A59D0DF
:1067400091ED146A9DED0F5A25EE866AA5EE076A53
:10675000B0EE675AA6EE265ABDEEC56A16EE10EAEE
:1067600016EE106AAE45A8BF2E467045C8BF064655
:1067700006EE106AB8EEC66A062A83ED056A39D0BD
:1067800091ED186A9DED105A25EE866AA5EE076A0E
:10679000B0EE675AA6EE265ABDEEC56A16EE10EAAE
:1067A00016EE106AAE45A8BF2E467045C8BF064615
:1067B00006EE106AB8EEC66A072A83ED066A19D09B
:1067C00091ED1C6A9DED115A65EE865AE7EE055A69
:1067D000E6EEA57AFDEEE77A17EE901A8D42A8BF95
:1067E0000D468842C8BF054607EE905AF8EEE77A94
:1067F000C3ED077A2FB922B19200D649D64826F0C8
:106800002FF8D64B1B68002B40F0AE84D44B1B787E
:1068100093B19BF8000060B1CF4ED24F0025E8B293
:106820003B68B6EC010A98479BF8000001358542A9
:10683000F5DBCD4B1B689847CC4B1B78072B00F042
:106840004286012384F8003113B0BDEC0A8BBDE809
:10685000F08FC74B1B78013BDBB2FFF710BAC54B7B
:1068600002934FF47A751B68B5FBF3F3C3EB431542
:10687000C149DFF8388391F80190BC49B8F90600A6
:106880000F7803EB8503DD00ADB2AE4201F09386D5
:10689000DBF88810BBF93CE0DBF86C304A1C07EEF3
:1068A00090EA7344012ACBF88820CBF86C30F8EEDC
:1068B000E77A01F08D86DBED1E5ADBED206A07EEEC
:1068C000102A37EEE56AB8EEC75A012E86EE057A31
:1068D00037EE257A77EEC77A8BED1F7AE7EE866A78
:1068E0008BED1E7AF0EE667ACBED216ACBED206A55
:1068F00002F05E80DBF89C10BBF93EE0DBF8703004
:106900004A1C07EE90EA7344012ACBF89C20CBF88E
:106910007030F8EEE77A01F07686DBED235ADBED96
:10692000256A07EE102A37EEE56AB8EEC75A012E3F
:1069300086EE057A37EE257A77EEC77A8BED247AE4
:10694000E7EE866A8BED237AF0EE667ACBED266A67
:10695000CBED256A02F05580DBF8B010BBF940E0C2
:10696000DBF874304A1C07EE90EA7344012ACBF836
:10697000B020CBF87430F8EEE77A01F05F86DBEDFB
:10698000285ADBED2A6A07EE102A37EEE56AB8EEE0
:10699000C75A012E86EE057A37EE257A77EEC77A4A
:1069A0008BED297AE6EE276A8BED287AF0EE667A8F
:1069B000CBED2B6ACBED2A6A02F04C80A8F80600DA
:1069C000BBF8B430694A013B1778ABF8B430029990
:1069D0000023072F4B608B60CB607FF444A9F8F74E
:1069E00073F9DFF8C88194F828310493A0EB0A000A
:1069F000A8F80000002B3FF43CA9013B84F82831A3
:106A000013B0BDEC0A8BBDE8F08F94ED577AB1F965
:106A10000000D4ED586AB1F902E0584AF4EEC76AB2
:106A200080EAE0738EEAEE71A3EBE073F1EE10FA08
:106A3000A1EBEE71B4BFB0EE476AB0EE666A8B426E
:106A4000B8BF0B4607EE103A1378B8EEC77A27EEB8
:106A5000287A002B40F00682494BD3ED005AF4EE21
:106A6000CA5AF1EE10FA40F19087B7EE005A75EE6F
:106A7000654ADFED446A9FED445A444B36EEC77ACF
:106A800024EE855AD3ED006AE7EE055A65EEA65A64
:106A9000F5EEC05AF1EE10FA40F2F784C9EEA56A9D
:106AA000B7EE007AF0EE475AE6EE665AF0EE656A07
:106AB000F4EEC76AF1EE10FA88BFF0EE476AF5EE21
:106AC000C06AF1EE10FAB8BFF0EE6A6A304B93ED8F
:106AD000007A67EE877AA7EEA68AFFF7B1B92D4B49
:106AE0002D4C19682D4ADFF8C48094F80031C9692B
:106AF0001288A8F80010A8F80220002B3EF434AF4A
:106B00000DF05AFB002384F80031184B1B78072B3B
:106B10007EF42AAFF8F7D8F88246FEF727BF204B5D
:106B2000204A2B4493ED007AD2ED007A1E4B67EE9B
:106B3000277AF7EE006AF4EEE67AF1EE10FA93EDBA
:106B4000007A88BFF0EE667A67EE877A27EE888A49
:106B5000FFF727BA9441002064890020C0AF0020CD
:106B6000506000203C5D0020445D0020046F002048
:106B700024B40020686000205460002060B400202D
:106B800068B4002000003443610BB63B5CB40020C5
:106B900058B40020BC6E0020B8230020BC3E00206A
:106BA0001425002050B400204CB40020086F0020B1
:106BB000D94BDFF8B8B31B789BF80020DD077FF5D1
:106BC0001AAE002A3FF41DAED4ED583A94ED574A60
:106BD000D24BD4ED627A93ED005A94ED617AD4ED04
:106BE000555A94ED546ACE49CE4BF4EEC43AF3EEC6
:106BF000046AF1EE10FA77EEA64A00F15B8791ED98
:106C0000026A26EE656AB0EE674AA6EE074AB4EE5F
:106C1000E44A34EE666AF1EE10FA48BFB0EE456A17
:106C2000012A83ED006A3FF4ECAD91ED066A26EE91
:106C3000656AB0EE674AA6EE074AB4EEE44A34EE5F
:106C4000666AF1EE10FA48BFB0EE456A022A83ED9B
:106C5000016A3FF4D6AD91ED0A6A26EE656AB0EEA0
:106C6000674AA6EE074AB4EEE44A34EE666AF1EEED
:106C700010FA48BFB0EE456A032A83ED026A3FF47A
:106C8000C0AD91ED0E6A26EE656AB0EE674AA6EEDB
:106C9000074AB4EEE44A34EE666AF1EE10FA48BFF1
:106CA000B0EE456A042A83ED036A3FF4AAAD91ED84
:106CB000126A26EE656AB0EE674AA6EE074AB4EE9F
:106CC000E44A34EE666AF1EE10FA48BFB0EE456A67
:106CD000052A83ED046A3FF494AD91ED166A26EE21
:106CE000656AB0EE674AA6EE074AB4EEE44A74EE6F
:106CF000666AF1EE10FA48BFF0EE456A062AC3ED67
:106D0000056A3FF47EADD1ED1A6A66EEE56AB0EE33
:106D1000674AA6EE874AB3EE046AB4EEE44A74EE1C
:106D2000466AF1EE10FA48BFF0EE456A072AC3ED55
:106D3000066A3FF466ADD1ED1E6A66EEE55AE5EEF1
:106D4000877AF4EEE74A77EEC67AF1EE10FAC8BF1A
:106D5000F0EE457AC3ED077A53E5734BC7ED00AA11
:106D60001B689342BFF6ACA8704B1A88002384F8C6
:106D70006831002A41F015846D4A6E4B117818680D
:106D800081F00101F2F70EFFFFF7A2B86A4EDFF8BB
:106D9000E08106F24C7506F5F767F6EC017A9BED9B
:106DA000080ADBF87837F8EEE77A284627EE800AFB
:106DB0009847A5F1E000DBF898369847A5F17000F8
:106DC000DBF808379847D6F85806DBF8B83098470C
:106DD0002435AF42A8EC010ADFD1FEF73FBF4E4990
:106DE0000978C80703D45549098BA4F88C11544974
:106DF0005448098890ED037A07EE901AF8EEE77A86
:106E0000B4EEE77AF1EE10FA40F20C864E480088B4
:106E100007EE900AF8EEE77AB4EEE77AF1EE10FAB0
:106E2000C0F2D08549484A49D0ED006A91ED006A28
:106E30004848C4ED646ABCEEC75A76EE665A15EE51
:106E4000101AC4ED626AC4ED615A84ED656AA4F853
:106E50008C110121D0ED006A84F8981177EE677AE1
:106E6000FFF730B93C4B93ED005AB5EEC05AF1EE46
:106E700010FA40F30A83394BD3ED006AF5EEC06A8D
:106E8000F1EE10FA40F3018336EEC77A66EE695AE6
:106E900087EE266AC5EE856AB7EE007AB4EEC76A59
:106EA000F1EE10FA88BFB0EE476AB5EEC06AF1EEB7
:106EB00010FA76EE876AB8BFB0EE6A6A66EE266AA6
:106EC000F6E5274A92ED007AF0EEE76AF4EEC76A3B
:106ED000F1EE10FA7FF786A8224A92ED007AF0EEE2
:106EE000CC6AF4EEC76AF1EE10FA7FF77BA81E4A6F
:106EF00098ED007AD2ED006AB0EEC77AB4EEE67A89
:106F0000F1EE10FA7FF56EA801220399C4F86C1116
:106F100084F86821FFF76AB8F1B50020904100209D
:106F2000B4410020648900207CB40020E895002052
:106F3000EA950020EC950020988C0020F06100205C
:106F40004C420020D46F00204E42002038420020E6
:106F500034420020544200205CB4002064B400207D
:106F600090B400208CB4002094B40020E56E002082
:106F70006C6000200299724BD1ED017A93ED007A9A
:106F8000F0EEE77AF4EEC77AF1EE10FA7EF5A0AFF4
:106F9000D1ED027AF0EEE77AB4EEE77AF1EE10FA8C
:106FA0007EF796AFD1ED037AF0EEE77AB4EEE77AAA
:106FB000F1EE10FA7EF78CAF624B1B689A077FF5F3
:106FC000D3AE6149614BB3F90C20B1F900E06048E0
:106FD000AEEB020E00688EEAEE72A2EBEE72824217
:106FE000BEF676AFB3F90E30B1F90220D21A82EABA
:106FF000E273A3EBE27398427EF76AAFB4E6554BB7
:1070000098ED007AD3ED006AB0EEC77AB4EEE67A76
:10701000F1EE10FA7EF7FCAFFEF7F7BF07EE103A7D
:107020004D4BDFF840811B78C4F81061B8EEC77A89
:10703000F7EE006A132B86EE879AB8F90400B4F8CD
:1070400014519BED080A01F03882444B444A93EDF9
:10705000001A93ED053A93ED122A93ED176AD3EDDA
:10706000091A93ED0E4AD3ED015AD3ED063A93ED8A
:107070000A7A93ED0F5AD3ED132AD3ED186AD3EDA4
:10708000044AD3ED030A67EE897A69EE288A29EE6D
:10709000088AA1EE273A02EB85060021A2EE286AB3
:1070A000C4F80411C4F80811A1EE884AE5EEA73A25
:1070B000A7EE085A93ED167AD3ED0D5A93ED021A06
:1070C000D3ED0C1A86ED003AE2EEA86A64EEC34AEC
:1070D00027EE467A93ED0B2AD3ED152A86ED204A4A
:1070E000E0EEC33A65EEC45A93ED143AC3ED053AA7
:1070F000E1EE274AF0EE477AA1EEC45AE2EE085AD2
:10710000E2EEC66AE3EE287AC3ED064A83ED0E5A34
:10711000C3ED0F5A86ED406AC3ED176AC3ED187AC6
:10712000C4F80C11013505F01F05A4F81451A8F896
:107130000400FEF776BCB0EE465AFEF7FCBF00BF77
:1071400088B4002020720020F8710020947800207C
:1071500084B4002094B40020046F002094770020B1
:1071600010750020086F0020B44B1B78192B07D82E
:107170000121B34A01FA03F31A40002A41F078844E
:10718000B04BB14EB14F01931B689D061CD5FB7AE5
:10719000FF2B04D0AE4A12789A4201F2F380B7F97D
:1071A0000880FB7DA6F80080FF2B04D0A84A127847
:1071B0009A4201F2E280B7F91450758008200CF071
:1071C0007DFC002840F03586B7F90600B6F900C00E
:1071D000B6F902E0B7F91210B7F91E20B6F904505B
:1071E000B7F90430B6F906806045A8BF604671451E
:1071F000A8BF7146AA42A8BF2A469C45A8BF03461D
:107200003380B7F91030B6F908009E45B8BF19466B
:10721000B7F92A307180B7F91C10B7F934E043454B
:10722000A8BF43468D42B4BF0D461546B7F9362078
:10723000B580B7F92850B6F90A108242A8BF0246B5
:10724000A845ACBF9846A846B7F94230B6F90C50ED
:10725000A6F806808B42A8BF0B467045ACBF10460F
:107260007046B7F94E203081B7F94000B6F90EE00C
:10727000AA42A8BF2A468842C8BF0346B7F95A00A7
:10728000B7F94C1073817045B7F95830714FA8BFEA
:1072900070469E45A8BF0346A942D8BF1146B1819A
:1072A000F381BB892BB3DFF8BC81DFF8BCA1DFF829
:1072B0009C9108F11005B8F9023000EE103A5046E2
:1072C000B8EEC00AF1F7B6F925F03EFCB9F9043082
:1072D000B9F9062000B298420AF1240A09F10C0912
:1072E00003DB82421346A8BF034628F8023FA845A5
:1072F000E1D1524B1B78013B182B74D8DFE813F017
:1073000061007300730019007300730073007C0840
:10731000730073007300730073009C0873007300A4
:1073200073007300730019008A08730073009C08CF
:107330006100494BB6F908101A6802B111609B69E7
:10734000B6F90A2003B11A60019B1B689A0601F185
:10735000ED8602220492D9027FF558AAFE7B112EF7
:107360003FF654AA3D4BDDF810901D4633F9163018
:1073700000EE103A4846B8EEC00A06F1010806F1E0
:107380000E0707F0A7FD4B465FFA88F89E1BFFB279
:10739000A94600E0A84608F1010508EB0600B8F18F
:1073A000120FEDB2C0B23FF431AA39F9183000EE35
:1073B000103AB8EEC00A07F08DFDBD42EAD1FFF7E2
:1073C00025BABB7B002B42F07B80254B1B7813F04A
:1073D000010342F07580204A1268002A02F04F84AF
:1073E000136001230493019B1B68980603D4134A7E
:1073F0001278052AAFD1049A13460233551CDBB22A
:107400001046EDB20493B6F9003000EE103AB8EE33
:10741000C00A07F05FFDB6F9023000EE103A2846C8
:10742000B8EEC00A07F056FD019B1B6893E725F0F4
:107430008BFB29F81600FEF7FFBB00BFC4AF00208E
:107440003241300378600020548900200CB50020C0
:107450001079002050A9002060A90020C05B002006
:10746000F1B5002052890020BCAD002000000000D2
:1074700095ED007A0BEB4602B8EEC78A928F29F899
:10748000162028EE278AFEF7B5BB5FED086AFFF7E6
:107490001DBB59023FF55AA8FFF75CB8F7F714FC7B
:1074A000A94B069A1B78DFF8A482801A012BA8F852
:1074B000020000F07682072B7EF4D2ADF7F704FCD1
:1074C0000290FEF7CFBDF7F7FFFB029A9F4B801AA1
:1074D000D880FFF7B6B9002F41F0628191ED006AC4
:1074E0009DED0A5A9A4B25EE866AA5EE076AB0EE24
:1074F000675AA6EE265ABDEEC56A16EE107A16EE4B
